:10C000006F00823A00000000001801180028012883
:10C0100002280328002901290229032904290529C6
:10C02000062907290829002A012A022A032A042AA4
:10C03000052AA62A04CB02003ADE0000F002002006
:10C0400076030020C00200208E0200201C02002087
:10C0500042E000008AE0000030E20000BCE40000A2
:10C06000AAE5000098DC000056DB000018DC0000A8
:10C07000A8DB00009AEB00000C05002018E000008F
:10C0800066E800002E820200268402009E840200E0
:10C090009C430200D0430200FCF901003CEF010088
:10C0A000087C02009CE80000EC4A0200E88A0100DB
:10C0B000768B0100CE8B01002AF4000076F400009C
:10C0C000E0F2000010470100CA410100A650010043
:10C0D0007654010022580100FE3301009C33010018
:10C0E000843701004A34010072330100F633010045
:10C0F00024330100CE34010026350100D63401007E
:10C10000DA340100743501002E350100603501007C
:10C11000783A01007C3A0100CA340100D2340100AF
:10C12000723501007A3A010022360100EA3B010033
:10C130006A660100E8660100266701007449010093
:10C140008C490100C8490100D62D0100F42E0100E0
:10C150006A2F010000130100A60D0100EC2301006D
:10C16000240E0100501F01004CAC0200A2A40200EA
:10C170007EA90200AEBF020094BE020020C20200EF
:10C1800010C2020018C2020058C20200BC9602008F
:10C19000000000000000000000000000000000009F
:10C1A000C8C2020090BC020026BC020000000000D1
:10C1B000000000000000000000000000000000007F
:10C1C0009265020056530200DC560200B45402008D
:10C1D0000A5F0200B07C0200A67B0200F09602001B
:10C1E00028ED00000C450200CC4A0200C44B0200BE
:10C1F000000000000000000000000000704D010081
:10C200006A6402000000000000000000000000005E
:10C21000065302001C070020E445020044C202004D
:10C22000000000000000000014C2020048E400000A
:10C23000C64A01004CC2020068660200366702006E
:10C24000B0670200E4A9020048C2020050C2020026
:10C25000C8EE010054C202001E11002098170020F1
:10C26000C4A902006AAB02003865020000000000A9
:10C2700000000000000000000000000000000000BE
:10C280006373B60082801C419105110523AEF5FE53
:10C29000C5BFB7270020372700209387078F1307D4
:10C2A000C7E66373F700828023A007009107D5BF1C
:10C2B0004111B7E700E022C480433707200006C6DB
:10C2C000798C23A0E7180F10000011C199E5B7E79A
:10C2D00000E023A08710014545A893073500C20759
:10C2E000C183F19BC207C183130740036366F70252
:10C2F00037270020032587A137270020832607A1A1
:10C300006391A60237270020032787AA69D3C207B3
:10C31000DD8D0545029765BF37270020032547A11E
:10C32000E1BF035765002DE7035745006362F70639
:10C33000B72600203306F7402148938606A263788B
:10C34000C8028328050003D86600138687001D8F66
:10C350002A9661172312E6002320160123130600F4
:10C3600010C12312F500130788FF2393E60023135F
:10C37000B50083D566002105B387F5402393F60009
:10C38000B7E700E023A08710B24022444101828039
:10C390000841BDB7B7E700E003A807003707200052
:10C3A00023A0E7183378E8000F10000001E523A070
:10C3B00007118280B727002003AE87A1B72700208E
:10C3C00003A307A18146F28763FC670A83A80700DD
:10C3D000636BF50A63E9A80A138787006362E50ABD
:10C3E00003D66700216705076319E600372600209A
:10C3F000034786970507230CE6963726002013058A
:10C4000006A283D547000357650023930700130650
:10C4100006A22E97420741832313E5006387C703D3
:10C4200037250020032545A16301F50203D56600E9
:10C4300009ED83D7460023A016012107BE95A1056B
:10C440002392B6002313E600B6879843630A670277
:10C45000B726002083A646A16304D702835667004F
:10C4600085E283D64700835547001843A106AE9660
:10C470002392D70098C383576600A1072313F600C1
:10C48000B7E700E02DB7BE86C6873DBFB7E700E03F
:10C490009843B706200023A0D718758F0F1000000F
:10C4A00001C599C1814711E6B7E700E023A0E71075
:10C4B0008280B386F50003C80600B306F500850741
:10C4C00023800601E317F6FEC5B737E700E01C43FB
:10C4D000B70620002320D718F58F0F10000019C1D0
:10C4E00091C111E637E700E02320F7108280910523
:10C4F00003A7C5FF11057D16232EE5FEDDB737E73F
:10C5000000E01C43B70620002320D718F58F0F103A
:10C51000000001C53307C50011E637E700E023201E
:10C52000F71082800505A30FB5FEE31DE5FEF5B704
:10C53000B7E700E09843B706200023A0D718758F0F
:10C540000F1000008147B306F5008386060099E6C8
:10C55000B7E600E023A0E6103E8582808507E5B7B8
:10C5600037E700E01C43B70620002320D718F58FDB
:10C570000F10000001C599C1014711EA37E700E03B
:10C580002320F710054582800507E309E6FE3308FE
:10C59000E500B386E5000348080083C60600E3050E
:10C5A000D8FE37E700E02320F7100145828037E707
:10C5B00000E01C43B70620002320D718F58F0F108A
:10C5C00000001307F6FFBA952A966317C50037E7F0
:10C5D00000E02320F7108280FD1503C71500050534
:10C5E000A30FE5FEDDB737E700E01C43B7062000E8
:10C5F0002320D718F58F0F10000001C53307C500A1
:10C6000019E637E700E02320F71001458280050591
:10C610008346F5FFE397B6FEE31BE5FE37E700E050
:10C620002320F71005458280797126D2B724002097
:10C6300022D403A444A706D64AD04ECE52CC56CA22
:10C640005AC85EC662C44DC8372A00203729002068
:10C65000B7290020814BB72A002037CBC901130A24
:10C660008AA7130909A2938949AC8357240099EF3B
:10C670005C44639A0B0023AAF4A6032CC400228511
:10C68000113B6284B9A823A6FB00C5BF83A7CAA635
:10C6900082971C443307F5406376F50003A74900F1
:10C6A0001D8F2A979306FB3763ECE60623280900C3
:10C6B000835524000345040097E000E0E780A0BF15
:10C6C0005C405844B1C70C4403A64900AE97BE86EF
:10C6D00063E4B70063E4C700B386C74014C4A28B09
:10C6E0003A8441F4B7270020938707A2984B8946E4
:10C6F00063FCE604791798CBB25022549254025945
:10C70000F249624AD24A424BB24B224C4561828086
:10C7100063950B0023AAE4A68DB723A6EB00B1BF57
:10C7200003274A0219CB63EDA7003385A74083276F
:10C7300009016374F5002328A900A28B404455B772
:10C7400003A74900BA97D5B723A8070075B7B7273D
:10C75000002003A7C7AB411122C406C63E8411C303
:10C760000297B727002083C7A7A693F7F70F99E38F
:10C77000232E04AAB24022444101828001114EC6F8
:10C78000B729002083A7C9A406CE22CC26CA4AC84E
:10C7900052C456C281C7829723A609A4B724002099
:10C7A0009387C4D683C75700372400209384C4D608
:10C7B000858B1304C4A481CF83C774001947631603
:10C7C000F70EA3820400EF00B0605C4482971C4423
:10C7D00091C382973724002037290020930704A2B1
:10C7E000032709A703C61700130A04A2834704A25C
:10C7F00093961700BA9683D60600F9C2834704A21F
:10C8000063E8C70C83A7C9A4230004A2639407129A
:10C81000B727002083A7C7A6638E0710B72700207D
:10C8200083A787AC2328FA00013583C7B40063933C
:10C83000071083C7940081CF83C7740093F7F70F65
:10C8400099E7A3840400974002E0E7804022B727DD
:10C85000002083A7C7A9F9CF83270A01E1CF83C7A7
:10C86000740015476368F70CB7270020938787DBB0
:10C8700083C7C700918BDDEFB727002083C7A7A62A
:10C8800093F7F70FC5EB83461A00032609A763CC7D
:10C89000D70A6244F240D2444249B249224A924AFB
:10C8A000056117E300E0670083FF83C774001D473D
:10C8B000E31FF7F0A3820400EF0090511C4839B742
:10C8C000850793F7F70F2300F4A2E3E1C7F23DB722
:10C8D00086073E978355070023100700034504A2EF
:10C8E000B727002083A787A413172500B72A0020A5
:10C8F000BA979C4323940AA6829783D78AA60347B4
:10C9000004A293C7F7FF7D8D93171700032709A78C
:10C910003E97835707005D8D2310A700834704A22D
:10C9200081C785072300F4A2034704A283471A00A6
:10C93000E37AF7ECF2406244D2444249B249224AD7
:10C94000924A0561828013971700329703570700B8
:10C9500075F385072DBF37C700408326C720B7076B
:10C96000FCFFFD17F58F2326F72001000100B727F4
:10C970000020938707A2C84F832787262326D72026
:10C980006A0593C7F7FF99835D8D8280B7270020E2
:10C9900003A387AD6303030002831305F00F8280B6
:10C9A0000327851163000712411122C406C683477D
:10C9B000C5008345E5042A8493F7C70F2306F500D5
:10C9C000834697000356C70013958601618563F17E
:10C9D000C508635A05060345870093F6F607A304C6
:10C9E000D700054693E627006314C50093E61700B9
:10C9F0002306D4005C4389075CC3A30AB400032563
:10CA000004112E864C4309055134832784110346B3
:10CA10005401D44303D7C700B296118FD4C32396D1
:10CA2000E7008947A30DF400B727002003476403FC
:10CA300083C7A7A86378F7048347C40093E7070177
:10CA40002306F40081A093E717002306F40075B7CE
:10CA50009376F60F635D050203458700854513E66F
:10CA600027006314B50013E617002306C400A30AC9
:10CA7000D400A30407008547A30DF4008327841185
:10CA80009C43DDF3B240224401454101828093E79B
:10CA900017002306F400A30AD400A304070003250B
:10CAA00004114C430905DD328327841103465401E8
:10CAB000D44303D7C700B296118FD4C32396E7009F
:10CAC0008D475DBF05458280B727002083A747D5E6
:10CAD000411122C406C6858B2A84DDEB416513050E
:10CAE00025F5970002E0E780A0FA5DC18347A50025
:10CAF0002315F50083270412B5E72320A41223226F
:10CB0000A41285472311F404232005008347640100
:10CB100054412316F5000347D4002304E5000547DC
:10CB2000A304E50037270020032707D91385170240
:10CB300015811C437D151375F50F9CC25C43DCC247
:10CB40001C479CC65C47DCC61C4B9CCA5C4BDCCAC1
:10CB50001C4F9CCE5C4FDCCE19CD9386060213078A
:10CB60000702C1BF8327441288C3835724042322AA
:10CB7000A412850741BFB7270020938707C303D7B7
:10CB8000870005072394E700B240224441018280D8
:10CB90008347C40023090400054593C747002306C3
:10CBA000F400DDB78347850193F7E70FDDEB83479B
:10CBB0009501C5EB034625018346C50009CA372701
:10CBC0000020834565030347B7A863E7E50013F733
:10CBD000060149CB014709C6C18A0357E51881C63A
:10CBE0008356251936973DCFB727002003D5C7AC0C
:10CBF0001307C71237460F00B335A70241111306BA
:10CC00000624814622C426C206C67D543305A702E7
:10CC100097C002E0E78080A7B727002083C7F7A866
:10CC2000B384A700B727002003A707CC83270709F1
:10CC300063F387003E84184375FBB727002083A762
:10CC4000C7A6829781476364A400B307A440B2409B
:10CC50002244B3B7970093C7170092443E85410121
:10CC6000828081473E858280B727002003A747D96D
:10CC70003C5BFDFF010001008280011122CC4AC80B
:10CC80004EC606CE26CA52C456C25AC00347B50085
:10CC900085472A842E8983290509631AF71E83573D
:10CCA0000508035BC503372A002093064AAC83DAE4
:10CCB0008600130A4AAC63F4671B83460501639040
:10CCC000E61A03278511631C07180327450A631812
:10CCD00007188346F5001D476393E6180355A5031F
:10CCE000330BFB409307204E33056503832444092F
:10CCF00037460F008146130606243305F502B72791
:10CD0000002083C7E7A8B3549502B3B5AA02BE9426
:10CD1000C204C180231394083385AA0297C002E09D
:10CD2000E780C096B307350133B5A7002E953E873F
:10CD300083264A0019E163E4D7003387D740B384E0
:10CD40005403B7460F009387F623938606242320C7
:10CD5000E900A697B3D7D702DA97636CF70E1D8F59
:10CD60002320E900B729002083A7C9A6832409004E
:10CD7000829763E1A4123385A4406350050C83A716
:10CD8000C9A6372B0020130B4BAC82970327090051
:10CD90006368E510198D8357E40303578B008E07F2
:10CDA000B387E7021307003293870719B3D7E70267
:10CDB00063EDA70E374A0F00930AFA23130A0A24D9
:10CDC0008357040485072310F4048347041499E36C
:10CDD0002285512A228597F001E0E78060F27DE10B
:10CDE000832604098327C40803274B00B6973E8592
:10CDF00063E4D70063E4E7003385E7408347F40149
:10CE0000835464082328A4088507A30FF4008357DC
:10CE10008B00B384F402D694B3D444036363950CBB
:10CE2000B304954083A7C9A623209900829763EE97
:10CE3000A40A3385A440E34505F8B727002083C73B
:10CE4000F7A863E2A708B727002023A487CC0145F1
:10CE50009DA883264A00B387F6403E9711B78354B6
:10CE6000640837470F009307F723B3845403BE9435
:10CE700093070724B3D7F40263E7F900B387F940B7
:10CE80002320F900C5B503274A00BA99C5BF23A0DE
:10CE90003501C9BDB727002083A787ACBE94E1BD8B
:10CEA00083274B00998F3E95FDB5A145228597F0CC
:10CEB00001E0E78000DEA305A402B727002083A7D6
:10CEC00087AA81EF7D55F2406244D2444249B2497B
:10CED000224A924A024B0561828089451545829714
:10CEE000D5B7B3049740AA9435BF83274B00BE94AF
:10CEF00089B72DC901116C0022CC06CE2A84B53B1E
:10CF000029CDFD576305F50237270020130787A7B2
:10CF10005453B2479DC62547637FF700D9173EC6D5
:10CF2000B2450345940297D000E0E780C04FF2403D
:10CF300062440561828037270020032787ACBA97B7
:10CF4000F1BF0347770163E4E700998FC9BFB726B4
:10CF5000002083A686ACB697CDBF97F001E0E780AE
:10CF6000A067F1B78280797126D206D622D44AD042
:10CF70004ECE52CC56CA5AC85EC6834755030344A8
:10CF80007513AA843E941374F40F9307400263F65A
:10CF900087001304B4FD1374F40F03AA841383AA47
:10CFA000C413A38B841222865285D68597B002E0E3
:10CFB000E780006B058915E503CBD412014981494F
:10CFC000337B6403930B50024A865285D68597B013
:10CFD00002E0E780E068058915C563916903137471
:10CFE000F90F238B8412B250225492540259F24901
:10CFF000624AD24A424BB24B456182808509E209BE
:10D0000093D989410509E31179FDE1BF832785099A
:10D0100003560504797193D60701BD8EC206C182FD
:10D02000358E1357764093575640898B058B5D8F0D
:10D0300093573640918B5D8F93571640A18B5D8F30
:10D0400093171600C18B5D8F9317360093F7070275
:10D050005D8F931756009355860093F707041E06BD
:10D060005D8F1376F60F518F93D7554013D6354009
:10D07000118A898BD18F13D67540D18F13D6154065
:10D08000218AD18F13961500418AD18F13963500CE
:10D0900013760602D18F13965500137606049E056B
:10D0A000D18F93F5F50FCD8FA20745465D8F3307DE
:10D0B000C70222D42A8426D252CC56CA032A841309
:10D0C000832AC4135AC806D636974207418393571A
:10D0D0007740135557400989858BC98F13553740C1
:10D0E0001189C98F135517402189C98F131517004E
:10D0F0004189C98F1315370013750502C98F1315A0
:10D10000570093558700137505041E07C98F1377C1
:10D11000F70FD98F13D5354013D755401189098B97
:10D12000498F13D57540498F13D515402189498FF3
:10D13000139515004189498F139535001375050224
:10D14000498F13955500137505049E05498F93F576
:10D15000F50F4D8F2207D98FB387C7024AD04ECE25
:10D160005EC662C4B697C207C18313D7774013D592
:10D1700057400989058B498F13D537401189498F4D
:10D1800013D517402189498F139517004189498F7D
:10D190001395370013750502498F1395570093D5E2
:10D1A0008700137505049E07498F93F7F70FD98FF2
:10D1B00013D5354013D755401189098B498F13D5A5
:10D1C0007540498F13D515402189498F1395150056
:10D1D0004189498F1395350013750502498F1395C1
:10D1E0005500137505049E05498F93F5F50F4D8F76
:10D1F0002207D98FB387C702130650025285D685FE
:10D20000B697BD8E93940601C18033F6C402137B9A
:10D21000F60F97B002E0E780A04405890DED834743
:10D22000D41201498149B3849702130C5002C18082
:10D230004A865285D68597B002E0E780604205892C
:10D24000937BF90F11C563863403850993F9F90FB0
:10D250000509E31F89FD230B6413B2502254925435
:10D260000259F249624AD24A424BB24B224C4561C2
:10D2700082805E8BCDB70111B727002022CC03A49A
:10D2800007CF26CA4AC84EC606CEAA84130925006F
:10D29000854915C083C7140003473400858B630498
:10D2A000F700405CFDB71946930544004A85EFF04E
:10D2B0002FABE31835FF2285F2406244D244424945
:10D2C000B249056182804111B727002022C403A41E
:10D2D00007CF26C24AC006C693042500054901E8C7
:10D2E0002285B24022449244024941018280A685AF
:10D2F0001305A402972002E0E78020A8E30225FF9F
:10D30000405CF1BF4111B727002022C403A407CF1E
:10D3100026C24AC006C693042500054901E82285B5
:10D32000B24022449244024941018280A6851305FD
:10D33000A401972002E0E78040A4E30225FF405CBF
:10D34000F1BF0111B727002022CC03A487CE26CA43
:10D3500006CE2AC42EC6854419E40145F240624433
:10D36000D244056182808347910003471400858B76
:10D370006304F7000044CDB719469305A1001305D7
:10D380002400EFF0EF9DE31795FE0545C1BFB726DA
:10D39000002003A786D601114AC81C5F4EC606CEE0
:10D3A000998322CC26CA858B3689B7290020ADCF38
:10D3B00093070006372400201CDF9307C4D683C7D9
:10D3C0006700130700089304C4D66319F70083A706
:10D3D00049D69C4393F707042383F4008347C4D6BC
:10D3E00093F7070489CFB727002083A7C7A68297A2
:10D3F000C8CC8347C4D693F7F70B2306F4D683C76C
:10D40000440093F707048DE38547A382F400B72710
:10D41000002083A747D93707020098C7130700FCED
:10D420002382E4009848F8D3032789D61C5F9183B0
:10D43000858B95C31C5F93E707011CDFB72700208E
:10D4400083A747D9054723A20706B727002093875C
:10D45000C7D62382E70083A749D6D8430583058B27
:10D4600019C7D843759BD8C3D843799BD8C3F2401A
:10D470006244D2444249B24905618280093F730047
:10D4800020309317D50063DF0700B727002083A75C
:10D4900047D97D57B8D7B7270020938707A2D84F21
:10D4A0000507D8CF9377850099CFB72700209387BA
:10D4B000C7D603C72700136717002381E7001307A8
:10D4C00000F82382E7009377150099CBB727002057
:10D4D0009387C7D603C7170013671700A380E70019
:10D4E000937765008DC713774500B727002059CF84
:10D4F00003C7C7D6136717002386E7D6B7270020D0
:10D5000003A787D65C57F19B93E717005CD7931767
:10D51000F50063D20702B7270020138707C38346AD
:10D520000707938707C3C18ABDCA8347070793E7E5
:10D5300007022308F7069317E50063D60702B7270B
:10D5400000209387C7D603C74700620761876355EA
:10D55000070005472382E700B727002083A747D9A4
:10D560003707020098C79317C50063D00702B72793
:10D570000020938707C303C71707058B29C303C779
:10D58000170713672700A388E70682809387C7D60B
:10D5900003C7370013671700A381E70085B703C7E8
:10D5A000070789463D8B6308D70003C707078D46E9
:10D5B0003D8BE312D7F811472388E706ADBF03C7B9
:10D5C0001707118B79D303C717071367870065BF48
:10D5D000B7270020B726002003A647D99387C6D6D1
:10D5E00003C7C6D6058B11C723820700A382070095
:10D5F000828003C71700058B65FB785275F303C75C
:10D600005700EDB737270020032887D683278803E4
:10D610009583858BC1E311C683270803BD8323004F
:10D62000F60085CA832787D6985B4607935767011C
:10D630006356070093E707C0C207C183039706003C
:10D64000C207C18709C7BA970947B3C7E702239042
:10D65000F6009DCD8345150085CDB7270020938723
:10D66000C7D683C7670013879500894593F70704DA
:10D6700085C33A95834705000547994593F6F70614
:10D680006398E600E207E187814563D30700B94567
:10D690002E8582808545EDBF411126C206C622C473
:10D6A0004AC0B724002035ED83A644D9AE87F8528E
:10D6B0007DFF372900201309C9D62301090037F45B
:10D6C00000E03E85832704D1B285ED9B2328F4D06A
:10D6D000832704D193E787022328F4D073005010E6
:10D6E000973002E0E780C025B727002083A787D6C0
:10D6F000B70680009843558F98C3D857719BD8D7E9
:10D7000083A744D9A3020900A3000900094798C3CD
:10D71000832704D193E787002328F4D073005010A7
:10D7200005A08D476314F504B727002083A787D68B
:10D73000B70680009843558F98C3D857719BD8D7A8
:10D7400083A644D9B72700209387C7D603C72700ED
:10D75000058B19E703C73700058B51CB23820700E0
:10D76000B240224492440249410182808547E31934
:10D77000F5FCB7F700E003A707D16D9B23A8E7D01E
:10D7800003A707D11367870223A8E7D073005010BF
:10D7900003A744D98177FD175447F58F5CC70F1055
:10D7A000000003A744D9B7070200130600F81CC7FE
:10D7B000B72700209387C7D62382C700B72700204A
:10D7C00083A787D69C439D83858B639FA700930780
:10D7D00060197CD354C737F700E0832707D193E75C
:10D7E00087002328F7D01DBF9307E01BDDB7F85251
:10D7F00031FFBDB7B727002083A747D98847D8474F
:10D80000798D09C988C7B727002003A30798630348
:10D8100003000283828037270020B726002013866A
:10D8200086D9130787DB8347D7008345B601484A6B
:10D83000AE97FD8BB355F500A300F600A306F700E5
:10D84000858995E903471701814613080002B3F75C
:10D85000E7020147B355E50085899378F70F89C939
:10D860006395D700A30016018280850693F6F60F14
:10D870000507E31107FF8280B72700209387C7D6EB
:10D8800083C7570093F7F70FD1EBB727002083A783
:10D89000C7A6411122C44AC006C626C282973729AC
:10D8A0000020930789DB8047130989DB6302A40604
:10D8B00063688504018DB7240020938784D983C7CA
:10D8C000A70113545500938484D96363F404A137EA
:10D8D00083C7A401032789009396570036971D8CB0
:10D8E0002324E900E375F4FE224403C51400B2408A
:10D8F0009244024981454101173302E06700C36F3A
:10D90000B727002083A787AC33848740229565B76B
:10D91000B240224492440249410182808280B7276A
:10D92000002083A7C7A6011122CC26CA52C406CE66
:10D930004AC84EC68297B7240020938784DB80476D
:10D94000014A6301A406938484DB63668506018D26
:10D9500037270020930787D983C7A70113545500A1
:10D96000137AF501130987D9636BF402B7290020F4
:10D97000938949AC4D358346A90103A8840083A54A
:10D980004900139756004297158C3A866364070145
:10D990006364B7003306B74090C4E37DD4FC16043B
:10D9A000336A4401F24062445285D2444249B2494A
:10D9B000224A05618280B727002083A787AC338481
:10D9C0008740229571B7B727002003A747D98967F9
:10D9D000938707F47CD3B727002083A787DE83A62D
:10D9E0000709139656006358060083A60709139685
:10D9F0006600634406007453FDF28280EFE03FD579
:10DA00007300000000000000970200009382222DA6
:10DA10000383020023800200630F0300F325103408
:10DA20002EC0970500009385A5FD73901534EFF087
:10DA30007FDC7300203086DCEFF0DFDBE650828095
:04DA400000000000E2
:10DA4400B72700203727002083A787A1032707A132
:10DA540001456313F700828083D6670081E683D68D
:10DA6400470036959C43F5B7B727002083A587A7C1
:10DA740037270020938787A713860522232CC7A066
:10DA840003D74700938785FFB72600204111BA9733
:10DA9400056523A8F6A006C61D05935637006374D2
:10DAA400E500930600203307D60037250020232AFB
:10DAB400E5A023A0E522E1162312D60023130600D5
:10DAC4001CC3998FE1172312F700231307008D3F1E
:10DAD400B240B72700202393A7A241018280B72731
:10DAE4000020B726002083A787A103A606A12A87C2
:10DAF400B305B5406314F6003A8529A893868700D8
:10DB04009C43E369D7FEE377F7FE2E85E3E4D5FE75
:10DB1400E3F2F5FE828023AC05FE1C4191E701008F
:10DB240001000CC18280BA8703A787FF6DFF23AC75
:10DB3400B7FE8280184183A785FF6319B7001CC113
:10DB4400FD5723AC05FE238FF5FE8280232CF6FEC1
:10DB5400C5BF411122C437E400E026C204403707A0
:10DB6400200006C6F98C2320E4180F10000009E9F0
:10DB7400232094101545B2402244924441018280EE
:10DB84000347E5FF9307F00F6306F7002320941083
:10DB94001145D5B79720FF1FE780C05801452320C2
:10DBA4009410D1BF411126C2B7E400E04AC003A9D2
:10DBB4000400B707200006C622C43379F90023A065
:10DBC400F4180F10000009E923A02411B2402244E4
:10DBD40092440249410182809565938505D0C98D9F
:10DBE4002A842105C2054205C18141819720FF1F76
:10DBF400E780004501CDFD57232005002312850051
:10DC04002303F50023A024112105C9B723A024115F
:10DC140001456DBF0111B7E700E04AC803A9070039
:10DC24004EC63707200006CE22CC26CAAA893379ED
:10DC3400E90023A0E7180F10000037250020032473
:10DC4400C5A18144014619E499E8A1654E85EF0018
:10DC5400B00631A88347E4FF6397370395C8A685C8
:10DC64001305C5A1C13D75D0A1654E85C92EF240ED
:10DC74006244B7E700E023A0271126854249D24435
:10DC8400B2490561828091E02286032484FF65BF46
:10DC9400A284E5BF41114AC037E900E022C403244D
:10DCA40009003707200006C626C2798C2320E9180C
:10DCB4000F10000089E523208910154515A0B7270A
:10DCC400002083C717A2AA842E8563F5F400894730
:10DCD40063EE9700BD3DB7E700E023A087100D4534
:10DCE400B2402244924402494101828083A785FFC5
:10DCF40099E703C7E5FF9307F00F6308F700913D29
:10DD0400B7E700E023A087104DBF37250020238FFD
:10DD140095FE1305C5A10135A16526850D2601458E
:10DD24002320891075BFB727002023AE07A0828067
:10DD3400B727002083A747A799E33E85828003D7AE
:10DD440027006316B70003C70700E308A7FEDC47F4
:10DD5400E5B7B9CD011106CE22CC26CA8147C1460A
:10DD640033D7F540058B21C312053E953147330562
:10DD7400E50237270020832487AB05443314F400DD
:10DD84002EC642044180AA949C40C8408297B24562
:10DD940023A0040023A20400A18DF2406244D244D3
:10DDA4002E85056182808507E39CD7FA0144EDB78F
:10DDB4002E858280BDCD797122D406D626D24AD052
:10DDC4004ECE01444147B3D78540858BB1CF120570
:10DDD400314722953305E502B727002003A987AB15
:10DDE4008544B3948400C204C180BE892A99032760
:10DDF400090011C7032549002EC60297B2453147D1
:10DE04003304E40283A789AB3E941C4489E72320AE
:10DE1400090023220900B2502254A58D02599254BC
:10DE2400F2492E85456182800504E31EE4F88144AD
:10DE3400DDB72E8582804111B7E700E026C2844316
:10DE44003707200006C622C4F98C23A0E7180F1058
:10DE54000000B727002083A787A9372400201304D4
:10DE6400048C91C782971C403E9508C031A0B72707
:10DE7400002083A7C7A6FDF70840B7470300938790
:10DE8400D73F3305F502B7A72600938737ECB24096
:10DE94003E9508C02244B7E700E023A097109244BF
:10DEA400410182800111B7E700E022CC80434AC8D7
:10DEB4003707200006CE26CA2A892E86798C23A00D
:10DEC400E7180F100000131506019305F0044181B3
:10DED40032C69720FF1FE780A016AA8419C53246D0
:10DEE400CA859720FF1FE7806033B7E700E023A0CF
:10DEF4008710F240624426854249D24405618280FB
:10DF04007971B7E700E022D480433708200006D6B1
:10DF140026D24AD04ECE52CC56CA5AC85EC662C425
:10DF24003374040123A007190F10000005E123A096
:10DF340087100945B250225492540259F249624A58
:10DF4400D24A424BB24B224C45618280B727002013
:10DF540083A7C7A6BA8A368AB28B2E8BAA898297E0
:10DF6400B727002003A787AB3E898144B146C14748
:10DF7400338CD40233068701104241E6C165938590
:10DF840005F041459720FF1FE780800B19EDB72767
:10DF9400002083A787AA81C7814511458297B7E7E7
:10DFA40000E023A087102D4571B7B727002003A7F1
:10DFB40047A721E723AAA7A623000500832789AB47
:10DFC40005473317970023260500232475012311E1
:10DFD400E50023225501E29723A0370123A267011C
:10DFE40023A4570163040A0023009A00B7E700E062
:10DFF40023A0871001453DBF3E875C47F5FF48C716
:10E0040065BF8504E396F4F6B7E700E023A0871024
:10E0140021450DB7B727002083A707AC411122C4BF
:10E0240006C637240020130404A289C782975C48DB
:10E034003E9548C84848B240224441018280B7E72F
:10E0440000E09843B706200023A0D718758F0F105F
:10E054000000B726002083C616A26372D5023726B5
:10E06400002093161500032506A736958356050050
:10E07400D58D2310B50023A0E7100145828023A08D
:10E08400E7100D458280B7E700E09843B70620000B
:10E0940023A0D718758F0F100000B726002083C661
:10E0A40016A26374D50237260020931615000325A3
:10E0B40006A793C5F5FF369583560500F58D231005
:10E0C400B50023A0E7100145828023A0E7100D4589
:10E0D4008280011137E700E026CA0443B706200016
:10E0E40006CE22CC4AC84EC652C4F58C2320D7187B
:10E0F4000F100000130705FF1377F70FFD4763E2C6
:10E10400E70AB146B306D502B727002003A787ABB9
:10E1140036971C43D9C71359450005443D89331527
:10E12400A400131405014180AE894A85A2850931F2
:10E134002A8A39C9A2854A85B937B727002083A717
:10E14400C7A637290020130949AC82978357890051
:10E154002A848146B385370313060064B3B73703B3
:10E1640013850532B335B500BE95EFE0A12AB30798
:10E1740085003E878326490063E4A70063E4D70053
:10E184003387D7402324EA00B7E700E023A09710A1
:10E194000145F2406244D2444249B249224A0561EF
:10E1A4008280B7E700E023A097100945DDB701118D
:10E1B400B7E700E026CA84433707200006CE22CC06
:10E1C4004AC84EC6F98C23A0E7180F100000BD47BB
:10E1D40063E8A70431473307E502B727002083A784
:10E1E40087ABBA979C438DCF05443314A4004204F3
:10E1F40041802E890145A285253EAA8911C5A285A3
:10E204000145513523A42901B7E700E023A0971065
:10E214000145F2406244D2444249B24905618280D8
:10E22400B7E700E023A097100945E5B779714AD014
:10E2340037E900E026D283240900B707200006D678
:10E2440022D44ECE52CC56CA5AC85EC6FD8C232068
:10E25400F9180F100000B727002083C717A26378AE
:10E26400F500B727002083ABC7A663970B00B7E779
:10E2740000E023A0971099A0B7290020938949AC06
:10E28400AE8A03AB490083D58900B74736FE93872E
:10E2940007C83E9BB387C5022A84328A8146B3B538
:10E2A400C50213850732B337F50013060064BE9523
:10E2B400EFE041166370AB02232099100145B25080
:10E2C400225492540259F249624AD24A424BB24B06
:10E2D40045618280829B83D589002A891306006464
:10E2E400B38745038146B3B5450313850732B33776
:10E2F400F500BE95EFE00112B30725013E8903A79F
:10E30400490063E4A70063E4E7003389E740D68566
:10E314002285393C09C923242501B7E700E023A05D
:10E324009710054569BF936504F0C205C181414555
:10E334009720FF1FE780C0D011E9B727002083A7EB
:10E3440087AA95D7A2851145829715B7372700204C
:10E35400832747A795E3232AA7A6854723260500F5
:10E36400232425012311550123008500A300F50072
:10E37400232205005DB7BA87D84775FFC8C7F1BF28
:10E384007971B7E700E026D284433707200006D628
:10E3940022D44AD04ECE52CC56CA5AC85EC662C4A3
:10E3A40066C26AC0F98C23A0E7180F1000002DC1C3
:10E3B4004144B689B28A2E8A2A89B14C372B00206F
:10E3C400054D130C0003B30B940303278BAB5E972B
:10E3D4001C43A5E39375F400B315BD0013554440E5
:10E3E400C2055686C1811375F50F893539C1832756
:10E3F4008BABDE9723A0270123A247016384090086
:10E4040023808900B7E700E023A09710014521A0ED
:10E4140023A097100945B250225492540259F2494C
:10E42400624AD24A424BB24B224C924C024D456155
:10E4340082800504E31984F9B7E700E023A097106C
:10E444002145D1BF0111B7E700E026CA844322CC9D
:10E454004AC84EC63707200006CE2A84AE893289C0
:10E46400F98C23A0E7180F100000C9332285CE854C
:10E47400C1302A8405C5B727002083D5C7AC13064D
:10E4840000648146B3872503B3B52503138507329A
:10E49400B337F500BE95EFD0F17748C013351400BB
:10E4A400F2406244B7E700E023A097104249D24407
:10E4B400B2490E05056182800111B7E700E04AC840
:10E4C40003A9070022CC4EC63707200006CE26CA71
:10E4D400AA892E843379E90023A0E7180F100000DD
:10E4E400EFF01F85AA8419C123110500A2854E856A
:10E4F400593EB727002083C707A263993701B7277E
:10E50400002003D787A6598C239487A6B7E700E099
:10E5140023A02711014591E01945F2406244D244F9
:10E524004249B2490561828001114AC837E900E0D5
:10E5340022CC03240900B707200006CE26CA4EC603
:10E544007D8C2320F9180F1000009307F00263E676
:10E55400A704B147B304F502B729002083A789AB08
:10E56400A6979C439DCB9377F5008545B395F5001D
:10E57400C205C1811181893783A789AB0145A6975B
:10E5840023A0070023A2070023208910F24062443D
:10E59400D2444249B24905618280B7E700E023A032
:10E5A40087100945E5B74111B7E700E026C2844367
:10E5B40006C622C437072000F98C23A0E7180F10E1
:10E5C4000000EFF0EFF619E90145B2402244B7E745
:10E5D40000E023A09710924441018280B7270020D5
:10E5E40083A7C7A600458297B7270020938747AC27
:10E5F4006368A402D843B74636FE938606C833053B
:10E60400A4403697E372E5FC13070064B335E502D2
:10E6140003D6870081463305E502EFD0B15F75B7B5
:10E62400D8433A94C1BF411122C426C237240020E2
:10E63400B7240020130744AC938404A2944858439D
:10E64400B727002006C683A7C7A6130444AC639269
:10E65400E60882975440B74736FE938707C8B697B3
:10E664003387A7003A856364F7006364D7003305F2
:10E67400D740B72400209387C4D6DC539384C4D6F0
:10E6840099CBB727002083A687DE3707CDFF7D17F8
:10E694009C46F98F9CC611E14840B727002083A708
:10E6A400C7A9829719E5DC5085C3EF604168EF5034
:10E6B400D166DC5091CBB727002003A787DEB706CD
:10E6C40033001C47D58F1CC7B240224492444101F9
:10E6D4008280829794485840B387A6003E8563E4BD
:10E6E400D700E3E8E7F83385E74061B74111B7277E
:10E6F400002006C623A0A7AC0295B240B72700208D
:10E7040023ACA7A2014541018280994763E9B70080
:10E71400B72700208A059387C7A4BE9588C1828045
:10E72400B727002023AEA7AA11C5B72700200547A5
:10E734002385E7A68280B727002023AA07A6B72748
:10E74400002023A007ACB727002023A607A637255F
:10E754000020B72700204111238507A67146B7275B
:10E76400002081451305C5A406C623AE07AA22C40A
:10E7740026C2372400209720FF1FE78040B11305ED
:10E7840004A21306800281459720FF1FE78020B072
:10E79400EFF08FADB7270020938787A703C5C70382
:10E7A40083C7D703130404A285453E958D473305DB
:10E7B400F5029947B724002039051375F50F230195
:10E7C400A4003305F502130505249720FF1FE780F5
:10E7D400208723ACA4AA49C1034624009947814554
:10E7E4003306F602130606249720FF1FE78020AAAB
:10E7F40083A784AB03472400B7240020938707240E
:10E804000A0723A4F4A4BA97372700202328F7A6DD
:10E81400EFF06FD1A5218347140083A684A437E6C3
:10E824000000139727003697130686DB10C313875F
:10E8340017001377F70F0A0737E600003697130619
:10E8440066D510C313873700890793F7F70F8A0734
:10E85400A300E400B69790C3B2402244924441011D
:10E86400828037270020130707A2834717008346B7
:10E87400270063F0D702B726002083A686A4138658
:10E884001700A300C70013972700369708C33E85D7
:10E8940082809307F00FE5BF1C41638C071041771A
:10E8A4007D8FB706002089476316D71003574500AC
:10E8B40063020710411126C21946AA849305F00F7A
:10E8C400610506C622C49720FF1FE780C0AA05473A
:10E8D4008D47630AE50C9C4491C7D858994761C792
:10E8E400985C71C337240020130600048145130586
:10E8F40084A79720FF1FE780809913060004A6854C
:10E90400130584A79720FF1FE7804091930784A7EE
:10E9140003D7C70009E7130700102396E70003C7CE
:10E92400E70001E705472387E70003D7070101E76D
:10E934006D472398E70003C7F70001E71547A3874E
:10E94400E70003C7270101E705472389E70003C759
:10E95400370109E703C7F700A389E70003C7570195
:10E9640001CB937637000983238ED702A38EE70267
:10E9740003C7470101E75547238AE70003C764013A
:10E9840009E71307C003238BE7009C5791C78297BD
:10E99400B72700202394A7A2B72700207D57A3867A
:10E9A400E7E4513B8147B240224492443E85410111
:10E9B400828089473E85828001114AC83729002018
:10E9C400832749AC06CE22CC26CA52C456C24EC6B0
:10E9D4008297130A0064B3354503130949AC835A7B
:10E9E40089008146568633054503EFD0B122B72707
:10E9F4000020138707A2004FAA84014563069402EE
:10EA0400938907A233858440636E940003254900EB
:10EA140056868146B335AA023305AA02EFD0911F68
:10EA2400018D269523AC9900F2406244D2444249B8
:10EA3400B249224A924A05618280011122CC2E8475
:10EA4400B7D502000A8541469385858606CEEFD068
:10EA5400F155180806043A94B7270020035504FF1B
:10EA640083D7E7ACF2406244AA9737450F001305F9
:10EA740005243355F50205618280B727002083D72A
:10EA8400E7AC51471D45637CF70279471945637824
:10EA9400F7021307200315456373F7021307B00445
:10EAA4001145637EF700130740060D456379F700AF
:10EAB4001307600909456374F70013B5B70F828023
:10EAC400011122CC06CE2A842EC6EFF0CFB6B24571
:10EAD400F240818D33A5A502229562441375F50F8A
:10EAE40005618280011122CC06CE2A842EC6EFF065
:10EAF4008FB4B245F240818D33A5A50222956244BC
:10EB04004205418105618280011122CC06CE2A840E
:10EB14002EC6EFF04FB2B245F240818D33B5A50257
:10EB24002295624405618280B7270020138787A756
:10EB340018572DC3411122C426C24AC006C61389E0
:10EB440087A70297B7270020138707A203578700D8
:10EB54002A84938407A20DCBBA876373A700AA877C
:10EB6400C207C183BA866373E400A286C206C18267
:10EB7400958F5147635AF7008327C90291C382973F
:10EB8400EF60010423948400B24022449244024979
:10EB94004101828082800111B727002022CC3724D2
:10EBA400002023AC07AC930784A7DC5706CE26CA03
:10EBB400AA85130484A781C72AC68297B245C9C10E
:10EBC4009C410545ADCBDC41BDC783D78500A5C7B6
:10EBD40083D7A500ADC3B7240020138544AC5146A8
:10EBE400938444AC9710FF1FE7804063238604009E
:10EBF400B727002083A647AC372700202326D7A6B3
:10EC0400034774011DE3938747AC03D5870093073B
:10EC1400805737460F003305F50213060624814654
:10EC24008145EFD0217FA30BA40037F50000130525
:10EC3400C59B6D3C0145F2406244D244056182802B
:10EC4400B7270020938707A23707002023AE0700C9
:10EC54001307676EB727002023A2E7AC378732007B
:10EC6400938747ACFD56130727A1D4C398C72386BF
:10EC74000700B7C7004023A4D7269DBF011122CCAB
:10EC840037240020930784A7884706CE26CA4AC89B
:10EC940001E90545F2406244D2444249056182805B
:10ECA400130484A75C58F5D7185C65D770008545B4
:10ECB40082971844B247E30EF7FC0355C40093054A
:10ECC400E004B72400209710FF1FE7806037138704
:10ECD40004A208D3938404A24DDD0356C400930513
:10ECE400F00F01499710FF1FE780605A8347E40043
:10ECF4009050634DF90032859710FF1FE7808042E2
:10ED0400014523A0040223A2040269B78355C40069
:10ED14000844185CB3872503898105093E9508C218
:10ED24000297E9B701114EC6B7290020938789A736
:10ED34009C4726CA4AC852C406CE22CC56C25AC0E0
:10ED44002A8AAE843289638D071E938989A703A713
:10ED54004903630407121307F01F6362A7123724E1
:10ED64000020130704A2832A0702130404A2639A4F
:10ED74000A0803D5C9009565938515E09710FF1F10
:10ED8400E780002C08D02A866DC983D5C90083A7E3
:10ED9400490303A589008981829783A78900832A6F
:10EDA40004025CD089476316FA08C1476397F40CE0
:10EDB40083D5C9009147938505FCB3C5F5028A053F
:10EDC400D69503C725009307A0056314F70A83D7D4
:10EDD40005006390470B4A85268691059710FF1F0F
:10EDE400E780C0431C505685639357130145F24096
:10EDF4006244D2444249B249224A924A024B0561D2
:10EE040082805850E380E7FA03D5C900956593855D
:10EE140025E09710FF1FE780A022AA8A39CD83D569
:10EE2400C9002A8683A7490303A58900898182979B
:10EE340095BF8D47631BFA00C1476390F40483D5E3
:10EE4400C900938545FDF199A5BF91476318FA0060
:10EE54006395440383D5C900A115F5B79307001042
:10EE6400631DFA00A14763EA970083D5C900C11561
:10EE7400D9BF1C5056856390570D29458DBF9D6A97
:10EE8400637C5509930A05E01947B3CAEA0203D71C
:10EE9400C900372B0020B38AEA02BE9A93070BA25B
:10EEA400DC53130B0BA26395570103240B021DE0E3
:10EEB40003D5C9009305E0049710FF1FE7804018AD
:10EEC4002A8445DD83D5C90083A749032A8689811D
:10EED4005685829791451307A0058981939725004C
:10EEE400A29783C627006393E60483D60700639C36
:10EEF400460385058A052686A2954A859710FF1F35
:10EF0400E780C03183270B02E38287EE22859710C6
:10EF1400FF1FE7802021D9BD21677917E36FA7F48C
:10EF2400B30A5541ADB783C5370045BF83270B02EC
:10EF3400E38587F422859710FF1FE780A01E35BF65
:10EF4400B727002083A507A48DD991479306A00570
:10EF54008983139727002E9703462700E31FD6F0D3
:10EF640003560700631C460185078A072686BE955B
:10EF74004A859710FF1FE780602A8DBD83473700BD
:10EF8400C1BFB7270020938787A7984729C3985FF5
:10EF94001DCF8546631DD502411122C437240020AC
:10EFA400130404A2105006C619CE83D5C7004850D6
:10EFB4008981029708509710FF1FE780A01623202D
:10EFC400040223220402B24022444101828082804E
:10EFD400011122CC37240020930784A756C283AAA8
:10EFE400870026CA4AC84EC606CE52C42A89AE84B1
:10EFF400B289130484A7638C0A1C1C5C99EB294511
:10F00400F2406244D2444249B249224A924A0561DA
:10F0140082805C58EDD79307F01F63E8A70C372A6A
:10F02400002093070AA29C53130A0AA2B9C70844F2
:10F0340083274A02639FA70489476317F906C147D8
:10F04400E39FF4FA0355C4009147130505FC3345C7
:10F05400F5029317250003250A022686CE853E95E0
:10F064009307A0052301F50023102501110597102E
:10F07400FF1FE780A01A014561B70355C40093053B
:10F08400E0049710FF1FE780A0FB2320AA0245F1AC
:10F09400BDB78355C4005C5803260A028981829750
:10F0A4001C442322FA0249BF8D47631CF900C1475F
:10F0B400E397F4F40355C400130545FD9377C5FFA6
:10F0C40059BF91476318F900E39B24F30355C40027
:10F0D4002115EDB793070010E313F9F2A147E3E01C
:10F0E40097F20355C4004115D1BF9D676378F506B7
:10F0F400930705E01947B3C7E7020357C400372A4B
:10F104000020B387E702BE9A93070AA29C53130A0E
:10F114000AA2A1CF83274A026395570703250A024F
:10F1240091461308A0059305F00F93D72600139773
:10F1340027002A970346270063160607835807000B
:10F1440003463700639C2805B306D64063C696047D
:10F1540085078A072686CE853E9511BF21677917D4
:10F16400E36FA7E8B307F54049BF0355C40093050F
:10F17400E0049710FF1FE780A0EC2320AA0259F9AE
:10F18400BDBD8355C4005C5803260A028981568597
:10F19400829723225A0359B72310B7009316060106
:10F1A400C18261B70356C400B38596009105130666
:10F1B40006FCE3F6C5E413863400719A1106B29690
:10F1C4002301070123102701A301D70051B7372AD0
:10F1D400002093070AA29C53130A0AA2A9C3032579
:10F1E4000A0291461308A0059305F00F93D7260051
:10F1F400139727002A9703462700631406058358AC
:10F2040007000346370063982801B306D640E3D1CC
:10F2140096F42310B70093160601C182C1BF0345BB
:10F22400E4008357C4009305E0043305F502420566
:10F2340041819710FF1FE780A0E02320AA0245F137
:10F244007DBB0356C4008345E400B385C502338601
:10F2540096001106E3E5C5DAB9BF0145828083C78C
:10F2640005002300F50083D72500A300F50083D70C
:10F274002500A1832301F50083C74500A301F50000
:10F2840011458280B727002023AA078EB7270020C4
:10F2940023A8078E828029C1411126C206C622C432
:10F2A400AA8401458DC52E84B7D502002285414626
:10F2B400938585879710FF1FE78040F683C7040076
:10F2C40005452306F40083C71400A306F400B240E6
:10F2D400224492444101828001458280011122CC62
:10F2E40026CA06CE0947AA8432846381E5044146CE
:10F2F4008147639BC500638FE6006397B6000DA842
:10F3040041478147638EE600F2406244D2443E8521
:10F31400056182808A852285BD3F41468A8519A878
:10F324008A85953F41468A85228531A0E39AB6FCB9
:10F334002E86A28526859710FF1FE78060FBAA878B
:10F34400E1B7B727002023A8A78E8280B727002023
:10F3540023AAA78E8280011122CC0354650006CE15
:10F3640026CA4AC84EC641C083298500AE842A886D
:10F3740003C909008147131789016187635507028F
:10F38400B147054563FA8704511442040355280024
:10F39400418033878900A2864E868545EFA0B01848
:10F3A400B337A00085077D1413556900420405890D
:10F3B4001379F90341802380F400A380A4002381FE
:10F3C400240123928400014719C01387190098C4AB
:10F3D40009476383E7000145F2406244D24442494D
:10F3E400B249056182800545C5BFC167F917630A43
:10F3F400F502D94763F7B702011122CC2EC606CE17
:10F404002A84EF703055B2456368B50022856244A2
:10F41400F24005616F90E078F24062440545056171
:10F42400828005458280C167F9176314F5006F7007
:10F434007052411106C6EF90806511E15D45B240FE
:10F444004101828091476394F502834705002300BC
:10F45400F6008347250003471500A207D98F23111F
:10F46400F6008347350001452302F60082801145EA
:10F4740082804111814522C426C206C6AA8405257C
:10F484002A8409E9B727002083A7078F81C7F94594
:10F49400268582972285B24022449244410182808B
:10F4A40039714ED656D25AD006DE22DC26DA4AD834
:10F4B40052D4AA8A2E8BB28941EF36C6AD37914514
:10F4C400EF70105BAA844D492DC9B246054A2380CA
:10F4D40034010544630A0B00B68513851400029BAE
:10F4E4000505131405014180E20993D9894163D3C9
:10F4F4000902C1455685EF90C067654905E9338621
:10F504008400A2852685EFA000472A8905E13104FD
:10F514004204418091472C085685231CF10026CED5
:10F52400231D8100EF8010702A8901C963070A0036
:10F5340026859710FF1FE780E0BEF25062544A858B
:10F54400D2544259B259225A925A025B21618280A2
:10F55400BA84014AADBF011122CC26CA4AC84EC69C
:10F5640006CE2A893284B689253FAA840DE1B727BD
:10F57400002083A7478F81CF05476317E40003C4A6
:10F58400090005041374F40FA2854A858297F2409A
:10F59400624426854249D244B24905618280AE86DE
:10F5A400B7F5000001470546938525266DB783D737
:10F5B40005002300F50083D70500A183A300F5000F
:10F5C4000945828083D705002300F50083D7050011
:10F5D400A183A300F50083D725002301F50083D779
:10F5E4002500A183A301F5001145828083D705007E
:10F5F4002300F50083D70500A183A300F50083D77A
:10F6040025002301F50083D72500A183A301F5007C
:10F6140083C755002302F50083C76500A302F500E4
:10F6240003D58500190542054181828083D70500F1
:10F634002300F50083D70500A183A300F500094545
:10F64400828083D705002300F50083D70500A183BA
:10F65400A300F50083D725002301F50083D72500F7
:10F66400A183A301F5001145828003D54500060559
:10F6740042054181828083D705002300F50083D7AA
:10F684000500A183A300F50003D525000905420563
:10F694004181828083D705002300F50083D70500CC
:10F6A400A183A300F50083D725002301F50083D7A8
:10F6B4002500A183A301F50003D5450011054205EA
:10F6C4004181828083C705002300F50005458280BF
:10F6D40083D70500411122C406C62300F50083D751
:10F6E40005002E841105A183A30EF5FE83D7250002
:10F6F4009505230FF5FE83D7D5FFA183A30FF5FE50
:10F7040003C6F5FF9710FF1FE78040B1034544008F
:10F71400B24022441105410182808947639CF5006F
:10F7240083471500034705000145A207D98F23101D
:10F73400F60082801145828003D70500D94763FE15
:10F74400E702011122CC06CE2EC62A84EF70902047
:10F75400B24683D70600636DF50022856244F24009
:10F76400B7F50000014709469385255B05610DBB8C
:10F77400F2406244094505618280094582809147CF
:10F784009DC583460500FD15C2058547C181639269
:10F79400F60213D725008D89914791E9914701CB52
:10F7A40005052301D6002310E60048C281473E85A3
:10F7B400828009479147E39CE6FEC94733D7F502A7
:10F7C400B3F5F502D1BFAE86B7F500000147114687
:10F7D4009385855CF1B193F7350091EB898191476D
:10F7E40089C52310B60048C281473E85828091476F
:10F7F400EDBF03C745008947631AF702011122CC04
:10F804002A84C84506CEAE86014719C52EC69D4535
:10F81400EFE0EFACB2462A8722856244F240B7F5A6
:10F82400000019469385055F05619DB909458280ED
:10F8340099E1114582808347050005472311F600AD
:10F84400E379F7FEFD1593F5F50F33D7F502B3878A
:10F85400E702E390F5FE050548C22310E6000145E2
:10F86400828083C745000947AE866385E700414728
:10F874006399E700B7F50000014721469385456D7C
:10F8840005B1094582802310B60091E1014548C2C3
:10F8940001458280AE86B7F500000147294693856D
:10F8A4000563FDBE2310B60091E1014548C2014540
:10F8B4008280AE86B7F500000147314693856564C2
:10F8C400C5B62310B60091E1014548C201458280C6
:10F8D40003D74500854763FDE702011122CC2A8442
:10F8E400884106CE0DC12EC68545EFE04F9F2A877D
:10F8F40022856244B246F240B7F50000394693854A
:10F90400E566056171BEF240624409450561828085
:10F914000945828091479DC5034705008D4691475F
:10F9240063F2E602FD15C205C181B3C6E5023308E0
:10F93400D7026399050105052310D6002311E600BB
:10F9440048C281473E85828083C745000947AE8609
:10F954006385E70041476399E700B7F50000014775
:10F9640041469385456D2DBE09458280B335B0006F
:10F97400139525008280011122CC26CA06CE03C726
:10F9840085008547AA842E8449466310F702613CAA
:10F994008357240049151306200963C8A700F240C1
:10F9A4006244D24409450561828003479400854737
:10F9B4006314F70013660604484011C58D4532C62A
:10F9C400EFE0EF913246A2866244F2402A87268510
:10F9D400D244B7F500009385A5670561D1B48D477E
:10F9E40063FFB7028347150003470500F115A2071B
:10F9F400D98F2310F6008347350003472500C2053D
:10FA0400A207C181D98F2311F6002312B60089C53C
:10FA1400110508C60145828023240600E5BF11456F
:10FA24008280011122CC2A84884506CEAE8611C577
:10FA34002EC69545EFE0AF8AB2462A8722856244F6
:10FA4400F240B7F50000594693858569056189BC84
:10FA5400B335B000139525008280AE86B7F500005B
:10FA6400014761469385856C25BC8547114563F440
:10FA7400D7028347160083450600A207CD8F2310C3
:10FA8400F7009387E6FF2311F70089476386F600A2
:10FA9400090650C30145828023220700E5BF0147C0
:10FAA400814679468145EDBA83D705002300F500E8
:10FAB40083D70500A183A300F5000945828083C78D
:10FAC400250005472300F50003D505006397E700EB
:10FAD4000A050505420541818280C9473305F502BF
:10FAE400CDBF03D505000A0542054181828083D735
:10FAF40025002300F50003D5050083D72500330531
:10FB0400F502050542054181828003D50500828006
:10FB140003D50500828003D50500828083D72500A4
:10FB24002300F50003D5050083D725003305F5022E
:10FB3400050542054181828083D705002300F50035
:10FB440083D70500A183A300F50083D725002301F3
:10FB5400F50083D72500A183A301F50003D5450053
:10FB6400110542054181828083D705002300F500F9
:10FB740083D70500A183A300F50003D5250009055B
:10FB840042054181828089471145639BF600834782
:10FB94001600834606000145A207D58F2310F700FF
:10FBA400828003D70500D947AE8663F9E700B7051D
:10FBB400010001470D469385C5AA71BA09458280A3
:10FBC40011456393A6028347160083460600014548
:10FBD400A207D58F2310F7008347360083462600FB
:10FBE400A207D58F2311F700828083C7250005471C
:10FBF400FD1793F7F70F6361F70483D705008DCFE3
:10FC0400011122CC2A84C84106CE15C12EC68945CD
:10FC1400EFD0FFEC2A8722856244B246F240B70552
:10FC240001001546938525AC05616FF0DF92F24023
:10FC340062440945056182800945828095471145E2
:10FC440063F9D706411122C426C24AC006C68347B7
:10FC54001600BA8403470600A2073284D98F239082
:10FC6400F400834736000347260093054400A207A7
:10FC7400D98F2391F40089472382F4000946138520
:10FC8400540036899700FF1FE78040599307A9FF66
:10FC94002394F4009947631BF90023A60400B2409F
:10FCA4002244924402490145410182801904C0C49E
:10FCB400FDB7828083D705008DCF011122CC2A8421
:10FCC400C84106CE15C12EC68545EFD05FE12A870F
:10FCD40022856244B246F240B70501001D46938571
:10FCE40065AE05616FF03F87F240624409450561E6
:10FCF40082800945828099476395F60489474111BA
:10FD040006C62302F7008347160083460600B28521
:10FD1400A207D58F2310F7008347360083462600B9
:10FD240003464700A207D58F130557002311F70098
:10FD340091059700FF1FE780604EB24001454101E5
:10FD44008280D14711456394F600C1474DBF82803C
:10FD540083D705008DCF011122CC2A84C84106CE59
:10FD640015C12EC68945EFD09FD72A8722856244C4
:10FD7400B246F240B70501002546938525AF0561DB
:10FD84006FF06FFDF24062440945056182800945C8
:10FD9400828089471145639BF6008347160083469A
:10FDA40006000145A207D58F2310F70082800111B8
:10FDB40022CC2A84C84106CEAE86014719C52EC678
:10FDC4008545EFD0DFD1B2462A8722856244F240CE
:10FDD400B70501002D469385E5B005616FF0AFF7D7
:10FDE40011456393A6028347160083460600014526
:10FDF400A207D58F2310F7008347360083462600D9
:10FE0400A207D58F2311F7008280011122CC2A8406
:10FE1400C84106CEAE8611C52EC68545EFD03FCC6F
:10FE2400B2462A8722856244F240B705010035466E
:10FE3400938545B105616FF00FF293F716001145F4
:10FE440089EB89476387F60085822312D70010C3A4
:10FE540001458280011122CC2A84C84106CE15C1F5
:10FE64002EC68545EFD0BFC72A8722856244B24695
:10FE7400F240B70501003D469385A5B105616FF0D9
:10FE84008FEDF240624409450561828083D7050005
:10FE94008DCF011122CC2A84C84106CE15C12EC6AD
:10FEA4008945EFD0DFC32A8722856244B246F240F7
:10FEB400B70501004546938505B205616FF0AFE9CA
:10FEC400F240624409450561828009458280854784
:10FED40063FCD7022304A700A304B70083471600DA
:10FEE40083450600A207CD8F2310F7009387E6FF12
:10FEF4002311F70089476386F600090650C30145BC
:10FF0400828023220700E5BF114582800147814694
:10FF14004D4681456FF02FE48D47114563FBD702B1
:10FF24008347160083450600A207CD8F2310F700F0
:10FF34008347360083452600A207CD8F2311F7009F
:10FF44009387C6FF2312F7006386A600110610C725
:10FF54000145828023240700E5BF011122CC2A84B5
:10FF6400884506CEAE8611C52EC69545EFD03FB75F
:10FF7400B2462A8722856244F240B70501005D46F5
:10FF84009385C5B305616FF00FDD85471145639710
:10FF9400F6008347060001452300F70082800147ED
:10FFA4008146654681456FF00FDB011122CC2A841E
:10FFB400C84106CEAE86014719C52EC68D45EFD081
:10FFC4001FB2B2462A8722856244F240B705010077
:10FFD4006D469385C5B605616FF08FCC011122CCB7
:10FFE4002A84C84106CEAE86014719C52EC68D4562
:0CFFF400EFD0FFAEB2462A87228562449F
:020000021000EC
:10000000F240B705010075469385C5B605616FF0EE
:100010006FC9011106CE2EC6EF80D02301C9B245AB
:10002000F2400355250005616FC0303AF240494562
:1000300005618280B7270020A3800792B7270020A0
:1000400023800792B727002023A40790B72700201A
:1000500023A60790B727002023A80790B7270020E2
:1000600023AA0790B727002023A20790B7270020D4
:1000700023A00790B7270020239E07AE1306403821
:100080009387C7AF2391C70271761307400B1306FE
:1000900006B82391E7002392C70211671D46930615
:1000A00000059305000A1305007D2392E7002393C2
:1000B000C70241470546130810F82395E700239629
:1000C000E7002399E700239AE700239BE700239C9E
:1000D000E7002394E7022393B7002394B700239704
:1000E000D7002398D700239DA700239E0700239FB6
:1000F0000700239007022395C7022396070323973F
:1001000007029308F007239807022392E70423933A
:10011000E704239FE7042390E7062391E706239251
:10012000E706239917031307C01C239AC702239BD2
:10013000C702239C0702239D0702239E0702239FD9
:100140000702239007042391C704239407042395EF
:1001500007042396C7042397D7042398D704239929
:10016000A704239A0704239B0704239C0704239DC9
:10017000D704239ED7042393A70623940706239529
:100180000706239607062397B7062398B7062399F1
:100190000706239AE7067D57239B07062390070946
:1001A0002391E7088280011126CAAA84214522CC26
:1001B00006CE2E8432C636C43AC2EFD0FF9E1DC989
:1001C000A24612473246930700FD2300F5009947E7
:1001D000A30095002301F5002303D500A303E50048
:1001E0002312C500AA8522856244F240D2440561EB
:1001F0006FD09FAAF2406244D24405618280B72743
:10020000002023A8A7908280B727002023AAA790C8
:100210008280011122CC4AC806CE26CA2A8901440E
:10022000B30489006368B400F2406244D244424996
:10023000056182802EC6EFD05FC093170501C18390
:10024000A183B2452380F4009307140093F7F70FBE
:10025000850463F9B700CA9709042380A7001374C3
:10026000F40F7DBF3E847DBF411122C4372400209E
:100270001304C4AD03556400C16706C6FD17630FC0
:10028000F500B727002003C607C2B72500209385D5
:100290008591EF80E05AFD572313F400B2402244C9
:1002A0004101828009C925151375F50F1335850E97
:1002B0001345150082800145828023900500C9C640
:1002C000797122D426D24ECE52CC5AC806D64AD004
:1002D00056CA5EC63684328AAE892A8B814463F35D
:1002E0004407B307940083C7070013891400420929
:1002F000939A070193DA0A011359090163840A04E6
:10030000CA976341FA04B307240183CB07005E85D3
:10031000513F0DC99387FAFF2390F90063906B0357
:10032000130519002295B250225492540259F249F1
:10033000624AD24A424BB24B45618280D694C20493
:10034000C18071BF0145C5B701458280011122CC32
:100350003724002026CA4AC84EC69307C4AD06CE2D
:100360002E89D0CB8CCBC8C7AA8441469305F00F09
:100370004A859700FF1FE780400085491304C4ADFC
:10038000631935030848C145693541469305F00FA7
:1003900026859700FF1FE78040FE0549631525036A
:1003A00048446244F240D2444249B249C1450561E1
:1003B0008DB5414681454A859700FF1FE780E0FBE8
:1003C000E31535FDC1B74146814526859700FF1FDE
:1003D000E780A0FAE30625FDF2406244D244424998
:1003E000B24905618280411122C43724002026C20F
:1003F0004AC0AE842A891306000281451305C4ADA4
:1004000006C69700FF1FE780C0E89307C4ADA3812D
:100410002701B7270020238297C2EFC0407D854780
:1004200019C181474945230EF4ACB240224492449D
:10043000024941018280814781CD19C98547631BEB
:10044000F50083C7550093E707FCA382F5008547B5
:100450003E85828089476317F50083C7550093F76F
:10046000F703E5B70D478547E314E5FE03C75500DD
:100470001377F70313670704A382E500D1BF814711
:100480008DC105C103C755009306000C854713773E
:10049000070C6308D700930600048D476303D70059
:1004A00089473E858280411122C4005D06C626C26E
:1004B0001DC8AA84085009C59700FF1FE780C0C661
:1004C000485009C59700FF1FE78000C6085409C5BA
:1004D0009700FF1FE78040C522859700FF1FE78038
:1004E000A0C423AC0402B240224492444101828061
:1004F00019E9B727002083C7E7AD91C7372500204A
:100500001305858F828037250020130545AF828033
:10051000B727002003C5E7AD8280B727002003A5D9
:1005200087AE8280B727002003A5C7AE8280B72799
:10053000002083A707AF88438280B72700209387D6
:10054000C7ADD44B9842050798C203C5370093073F
:10055000F00F6305F50091656FD0BFAE8280011189
:1005600022CC06CE2E8432C6EF80605F9147B24522
:100570006310F502B727002083A7479195C303A313
:100580000700630F030022856244F2400561028385
:10059000B727002083A7C79081C703A34700D5B71B
:1005A000F2406244054505618280011122CC2A8413
:1005B0000355450006CE26CA4AC84EC6EF804038CD
:1005C0003DC92A89834405008349C500E93D4A8520
:1005D000EF80101803554400EF80A0533729002006
:1005E0001309099283470900B9CB639A9704B72787
:1005F000002083C517922685293C19E123000900B4
:1006000003554400EF80A0559147631FF500B727BD
:1006100000209387C7AD8356440003D767006395D6
:10062000E6007D572393E700F2406244D2444249FA
:10063000B2490561828081499304F00F45B7930761
:10064000F00FE38FF4FA8346640003564400034539
:1006500024004E87A685813E65B779715EC6AA8B58
:100660002E8552CC56CA5AC806D622D426D24AD093
:100670004ECEAE8A328B368AEF80802C7DC1045DEF
:100680002A89E5C09C50614599C3130540039C54D9
:1006900081C751054205418163050A007105420584
:1006A0004181DC5081C75D0542054181EFD0CFCF4C
:1006B0002A8445C9614681459700FF1FE78060BDD8
:1006C000B727002083C9C7B2639409008349090092
:1006D000930700FD2300F400A947A3007401230140
:1006E000F400230364018C50231254011305840188
:1006F00091C908C47146930A44039700FF1FE7801D
:1007000020B256858C5491C948C45146930A45017C
:100710009700FF1FE780C0B05685630C0A0008C829
:100720007146D285930AC5019700FF1FE78040AF4D
:100730005685CC5099C548C85D469700FF1FE78095
:1007400020AEA2854E85EFD02FD52254B2509254C0
:10075000F249624AD24A424BB24B4A85025945613C
:1007600099B3B250225492540259F249624AD24A81
:10077000424BB24B4561828001114EC6AA892E853B
:100780004AC806CE22CC26CA2E89EF80601B21C91A
:10079000B727002083C4C7B299E0834405001945F8
:1007A000EFD08FC02A8405CD814519469700FF1FE1
:1007B000E78020AE930700FD2300F400B947A300B3
:1007C00034012301F40023122401A2856244F24083
:1007D0004249B2492685D24405616FD0EFCBF24041
:1007E0006244D2444249B2490561828039715ECE89
:1007F000AA8B2E8526DA4ED652D456D25AD006DE91
:1008000022DC4AD8AE84328BB68A3A8ABE8942C686
:10081000EF80001321CD2A894145EFD0EFB82A841B
:1008200031C5414681459700FF1FE78080A6B72765
:10083000002003C5C7B219E103450900930700FD75
:100840002300F400BD472301F400B247A300740164
:100850002312940023046401A304540123054401DA
:10086000A30534015CC4A285EFD00FC3F2506254DB
:10087000D2544259B259225A925A025BF24B216128
:100880008280797126D2AA8439454AD04ECE06D6C6
:1008900022D42EC6B2893689EFD00FB121C1B2451C
:1008A0009307000D2310F500B1472A842312B500E9
:1008B0002301F500CE85190519469700FF1FE78033
:1008C000209623062401A2852254B2500259F249EF
:1008D00013F5F40F925445616FD00FBCB2502254FF
:1008E00092540259F24945618280411126C2B724CF
:1008F00000209384C4AD03C7340006C622C44AC096
:100900009307F00F630CF7042A893945EFD0CFA97C
:100910002A8429C5930700FDB72500202300F50090
:10092000A300250123010500938545AF0D05194658
:100930009700FF1FE780C08E83D78400A28503C580
:1009400034002315F40083C714002306F400224466
:10095000B2409244024941016FD00FB4B2402244E8
:10096000924402494101828001115AC02A8B3145CB
:1009700026CA4EC652C456C206CE22CC4AC8AE843F
:10098000B28A368ABA89EFD02FA23DCD2A84268535
:10099000EF70107B11C50347C500A1476314F7042E
:1009A000B727002003C9F7AD930700FD2300F4002B
:1009B0009D47A30064012301F40023129400231334
:1009C00054012314440123153401A2856244F240EA
:1009D000D244B249224A924A024B4A8542490561B1
:1009E0006FD08FABB727002003C957C2E31E0BFAA5
:1009F000B727002083A7079C9C47DDD7CE86528669
:100A0000D685268582974DB7F2406244D24442494A
:100A1000B249224A924A024B05618280011122CCDE
:100A20002A84214506CE2EC6EFD00F9821C1B245AB
:100A3000930700FD2300F500C5472301F50083C798
:100A40003500A301F50083D745002312F50083C7C5
:100A500065002303F50083C77500AA85A303F5008D
:100A600022856244F24005616FD00FA3F2406244D8
:100A700005618280397162CC2A8C594526DA4AD8C0
:100A80004ED652D456D25AD05ECE06DE22DCAE848A
:100A900032C636C4BA8B3E8BC28A468A8359010459
:100AA00003494104EFD04F9025C93246930700FD1A
:100AB000A2462300F5009547A301C500A3008501C8
:100AC0002301F5002A8419461105A9C2B68597F0BD
:100AD000FE1FE780E07423066401230A2401231526
:100AE0007401231754012318440123193401A285EA
:100AF0006254F2504259B259225A925A025BF24B56
:100B0000624C2685D25421616FD00F99814597F0B0
:100B1000FE1FE7800078C1B7F2506254D2544259A8
:100B2000B259225A925A025BF24B624C2161828086
:100B3000411122C4372400201304C4AD834724008C
:100B400006C626C28DCBB7240020AA851946138578
:100B5000848F97F0FE1FE780A06C034524009385E7
:100B6000848FEFF05F8D2244B2401385848F9244CE
:100B700041016FC08008B2402244924401454101C6
:100B80008280411126C2B72400209387C4AD06C6D7
:100B900022C44AC003C737009307F00F9384C4AD43
:100BA0006304F7042A892945EFD00F802A840DCDEC
:100BB000930700FD2300F500A147A30025012301B1
:100BC000F50083C72400B72500209385858FA301F6
:100BD000F5001946110597F0FE1FE780606403C514
:100BE0003400A285EFD04F8B03C724008D476311DB
:100BF000F702B727002083A7079199CB03A38700AB
:100C0000630803002244B240924402494101028336
:100C1000B24022449244024941018280797122D437
:100C200006D626D24AD04ECE52CC56CA09445DCD05
:100C30002A8903550500AE895144EF707050AA848B
:100C400055C537270020930707C283C7470085464D
:100C5000BA8AFD1793F7F70F494463F9F60803477B
:100C6000C500A1476314F700639209089C5C4544E2
:100C7000B5EF9165938545711305C00297F0FE1F8E
:100C8000E780403C88DC2A8A4D442DC11306C0020F
:100C9000814597F0FE1FE780C05F835709009306E8
:100CA0004A0036852311FA0071469305490036C67D
:100CB00097F0FE1FE780C05689472300FA0003C55E
:100CC000C400B2460356090083C50AC26115133534
:100CD0001500EF8070792A8463860900CE85268509
:100CE000EF80A05601C42685EFF0EFFB2285B250BD
:100CF000225492540259F249624AD24A4561828092
:100D0000B727002083C747C20547FD1793F7F70FA2
:100D10006378F708894751C6011122CC26CA4AC810
:100D20004EC652C406CEAA89368AB2842E89EF7086
:100D300030412A84D14729C9485509C597F0FE1F7B
:100D4000E780803EF1452685EFD00F9648D4CD4709
:100D500005CD8346C40021478147639FE600630DAC
:100D60000A000347A5010356050193062501AA853C
:100D70004E85EF802055AA8703474400630F090082
:100D8000136767002302E400F2406244D244424900
:100D9000B249224A3E850561828013674700DDB76C
:100DA000C9473E8582809307000463EBA700B727FD
:100DB00000209387C7AF06053E9503550500828046
:100DC00041657D158280011122CC2A842E8526CA98
:100DD00006CEAE84EF70D0361DCDB7470F00938797
:100DE000F723094563E4870281450A85414697F068
:100DF000FE1FE780004AA685231081000A854180F6
:100E000023018100A3010100EF809045F24062447C
:100E1000D244056182804945D5BFB7270020238190
:100E2000A7C282806F80705E797152CC2A8A328527
:100E300022D426D24AD04ECE56CA5AC85EC606D64C
:100E400062C4AE8BB28A368BBA843E89C28946842C
:100E5000EF70102F15C92A8C63140A0213774B0008
:100E60008347450015CF93E727012302FC008DEC53
:100E7000631C0902639A090205E8ED9B2302FC004A
:100E8000832B8C03639F0B06B25022549254025959
:100E9000F249624AD24A424BB24B224C45618280AF
:100EA000F59B93E70701D1B793E747002302FC00C6
:100EB00001CC1C484146A2852324FC0213058C0169
:100EC00097F0FE1FE780C03563910B02D5D803254C
:100ED000CC0209C597F0FE1FE7800025F145268565
:100EE000EFC09FFC2326AC0261BFE30B09F803258A
:100EF000CC0209C597F0FE1FE7800023F1454A8523
:100F0000C5B79DC483A70B0299EB91659385357195
:100F1000714597F0FE1FE780E01223A0AB0203A506
:100F20000B0219C57146A68597F0FE1FE780402F7A
:100F30006388090283A74B0299EB9165938525711C
:100F40005D4597F0FE1FE780E00F23A2AB0203A5EB
:100F50004B0219C55D46CE8597F0FE1FE780402CF9
:100F60001DC483A78B0299EB91659385157151453B
:100F700097F0FE1FE780000D23A4AB0203A58B02B0
:100F800019C55146A28597F0FE1FE78060292254BB
:100F9000B2509254F249B24B224CCA865A86025938
:100FA000424BD6855285D24A624A45616FF0EFEADC
:100FB000011126CA52C406CE22CC4AC84EC62A8A7D
:100FC000AE84EF70F01725C5AA893945EFC0DFBDA3
:100FD0002A8431CDB727002003C9C7B263140900A2
:100FE00003C909009307000D2310F400AD47230146
:100FF000F4009385690013053400194697F0FE1F2D
:10100000E780002293F71400858085882306F4008A
:10101000A306940023154401A2856244F240D24401
:10102000B249224A4A85424905616FC0FFC6F24073
:101030006244D2444249B249224A05618280011188
:101040004EC652C456C206CE22CC26CA4AC8AA8A66
:101050002E8AB289EF70D00E2DCD2A891305C002D9
:10106000EFC09FB42A8435C5B727002083C4C7B218
:1010700099E0834409009307000D2310F400E94729
:101080002301F4009305690013053400194697F015
:10109000FE1FE780E018D285231554011305C40014
:1010A000414697F0FE1FE780A017CE851305C401C7
:1010B000414697F0FE1FE780A016A2856244F240E9
:1010C0004249B249224A924A2685D24405616FC0FC
:1010D000BFBCF2406244D2444249B249224A924AD9
:1010E00005618280411122C437240020130404903A
:1010F000084006C619C597F0FE1FE780E0022320CE
:101100000400B240224441018280011106CE22CC6B
:1011100026CA4AC82EC6EF70B00239CDB245B727ED
:10112000002003C9C7B20CD5AA846314090003497F
:1011300005004145EFC05FA72A841DCD9307000D30
:101140002310F500A5472301F50083C754009385BC
:1011500064001105A30FF5FE194697F0FE1FE78006
:10116000200C9C54A285F2405CC46244D2444A855F
:10117000424905616FC05FB2F2406244D2444249C5
:10118000056182801D71A2CC86CE2A842EC6EF70A6
:10119000207B05CD8346C5001147AA874945639248
:1011A000E6029C5FB24599C383C56701B7B60100EB
:1011B0002308B100938606C2100889452285EF7086
:1011C000907FF6406644256182805145DDBFB72798
:1011D000002083C747C20547FD1793F7F70F637ACF
:1011E000F704894721CA411122C426C24AC006C653
:1011F000B2842E89EF70C0742A84D14705C5630874
:1012000009008347450093E727002302F500414684
:10121000A6851305840197F0FE1FE78060009C48B7
:101220001CD48147B2402244924402493E85410188
:101230008280C9473E858280797122D406D62A846D
:101240002EC6EF70E06F01CDB2452285230EB100AE
:101250006C08EF70107CB250225445618280514579
:10126000DDBF6F709004C1671387E7FF6395E502E8
:10127000B727002083A7C79091EB49458280494555
:10128000B2402244924402494101828003A30700F4
:10129000E30503FE0283411122C426C24AC006C6EA
:1012A000FD172A892E84B284639AF502B72700209D
:1012B00083A7C79091CF9C4381CF829711E9B7272D
:1012C000002023802793B7270020A38097924DBF4B
:1012D000A6854A85EFE0FFD345F5D5B72E85EF709B
:1012E000206651DD834705000D45E39B27F92285E4
:1012F0002244B2400249A685924441016FB0F00CED
:101300009307000463E2A7064111C16722C406C621
:1013100026C2FD172A8409456382F502C547AE84BB
:101320006313F4022E85EFB0D0113725002013058A
:10133000C5AF06042A94231094000145B24022440C
:101340009244410182809307A0036316F4002E8526
:10135000EFB07008D9BF9307B003E318F4FC13F59E
:10136000F50FEFB09007D1B709458280011106CE85
:101370002AC6EFE03FCCEF10C01CEFA01129B72721
:1013800000209387C7AD130700F02391E700238265
:101390000700B72700203245138707C2FD562301F7
:1013A000D700F2402380A7C2954505616F50F066D3
:1013B000597193970501A6D286D6A2D4CAD0CECEB3
:1013C000D2CCD6CADAC8DEC6E2C4E6C2EAC06EDE55
:1013D000C187AE8463D3075237240020034504C27B
:1013E00037290020372A0020EFC01F83AA8C22CC87
:1013F000B72A0020B72B00201304C9AD372C0020DA
:1014000063930C022165258DB650265496540659D7
:10141000F649664AD64A464BB64B264C964C064D84
:10142000F25D6561828083C70C001307200A639C0C
:10143000E7008349340003D52C00C1656686FD159D
:10144000EFF0EF919DA26247130707C2834927007F
:10145000130710096398E71683C71C001547639F9D
:10146000E7006685EFF06F946685EFC0CFEEE24748
:1014700003C507C2EFC04FFAAA8C59B73947639B1F
:10148000E71603D54C008567A5076316F50483A509
:101490008C0003CB0500631D0B00850591C9372522
:1014A00000201946130545AF97F0FE1FE78040D78F
:1014B0000347C9AD85476317F71063080B00230E78
:1014C00009AC5A85EFF06FC245B78947230EF9ACD6
:1014D000EFB0607251BF896713872700631CE50472
:1014E00003AB8C0063000B0E83470B0089EF83472F
:1014F0002B0003471B00A207D98F2314F400834756
:101500003B00A300F4000347C9AD8947631CF70AF9
:1015100083470B0091C7230E09AC03450B005DB751
:1015200083451400035584008D47230EF9ACEF501A
:10153000D051E5B795076319F50083A78C0003C563
:101540000700EFF00FE40DB7F9771387A7FF2A978D
:1015500042074183914663F1E6049387A7FCAA976B
:10156000C207C18371476371F70289671387B700A8
:101570006310E50483A78A90E38807EE9C43E68521
:10158000E38407EE829715A0370700181307F7705A
:10159000B357F700858BA9CB83270A91E38607EC25
:1015A0009C43E38307EC66858297E31F05EA19A84D
:1015B0001387C7006311E50283A78C0083C7070068
:1015C000E38407EA9307F00FE380F9EAE6854E85A6
:1015D000EFC08FEC69BDB9076318F5008327CC9085
:1015E000E38407E8DC4361BF896793871704E3035B
:1015F000F5F8C9BF3D476399E70403D54C008967F7
:101600001387D700E30CE5FC13879701E308E5FC9B
:10161000CD07E319F5FA03576400C167FD17631D91
:10162000F7008327CC90E38107E4DC43E38E07E2F5
:101630000965E6854D05B9B7B727002083A747910F
:10164000E38407E29C43DDB71307E003E39CE7F67E
:1016500083C72C0005476398E70E83C76C003727C4
:101660000020930D0790E1E783A70D00D5CF03CBB2
:101670000700A14903C57C00138D8C00EA85EFE0CB
:101680001FE083C74C01A383AC0083D80C0103D8AF
:10169000EC0003D74C002A8603C53C003EC283D72A
:1016A0002C01EA86DA853EC0CE87EFF0AFBC83C757
:1016B0003C0095E7DD4783D80C0103D8EC0083C6D6
:1016C0007C0083D54C003EC283D72C016A873EC084
:1016D000CE8705465A85EF70805FA381AC0083A753
:1016E0000D0081C71145EFF0FF9F138B0B9203454F
:1016F0000B00E30B05D6B727002083C51792EFE058
:101700005F91E30305D683C63C0093071003638A09
:10171000F60003D64C0083450B004E873685EFE07C
:101720009FA823800B9289B3034B340099B783277A
:101730000A91034B3400914995DFDC4385DF8145F5
:101740000145829705BF29476398E70A83C76C0064
:1017500037270020930D0790A5EF83A70D00B5C78D
:1017600003CB0700A14903C57C0093868C009377C7
:101770002500BDCB13761500138E4C0183C70C02D8
:1017800083D8CC0103D8AC0103D74C0003C53C007F
:101790003EC283D7EC01DA8572CE3EC0CE87EFF031
:1017A0006FAD83C73C00724E9DFBDD4783D8CC01F3
:1017B00003D8AC0183C67C0083D54C003EC283D7DE
:1017C000EC0172873EC0CE8729B7034B340059BF66
:1017D00083270A91034B34009149D1D7DC43C1D709
:1017E00081450145829741B7B68536CEEFE03FC9C6
:1017F000F2462A86368E59B70947639CE70083A7CD
:101800008A90E38307C6DC43E38007C66685829738
:10181000A1B92D476398E70083A78A90E38607C4A0
:101820009C47DDB70D476397E70066868D4503D576
:101830004C0039B119476395E7069305610213051A
:101840001031EFA021652C1013052031EFA0816429
:1018500003D66C008357810203D54C0063E8C700B0
:1018600083D68C000357610263F7E60093050002FC
:10187000EFB0203CD5BE6374E6002393EC0063F424
:10188000D7002394FC0003D7CC0083D6AC0003D64A
:101890008C0083D56C0001488147EFB04039E9B630
:1018A0001D47E381E7D231476395E7006686B1457E
:1018B000BDBF35476398E70083A78A90E38607BAE0
:1018C000DC4799B74947639DE70083270A91E38B7B
:1018D00007CEDC43E38807CE814505458297DDB11D
:1018E0004D47E391E7CE83270A91E38D07CCDC4394
:1018F000E38A07CCE6850945D5B793F7150089CF6C
:10190000B727002083A7879089C7DC4399C3014587
:10191000829713C51400CDBC93F7250091CFB7274C
:10192000002083A7079191C7DC4381C78145054506
:10193000829713C52400C9BC93F745000145E38590
:1019400007ACB727002083A7479037240020130453
:10195000C4AD91CF85472302F400B727002083A7A9
:10196000079191C7DC4381C781450545829748446B
:101970002C10EF70507B2810EFF08F9BB7270020C2
:1019800083D7E7B181CF130600643386C702B72738
:10199000002003C507C29145EFC09F8913C54400CD
:1019A000A5B4411122C4372400200325449006C663
:1019B00019C597E0FE1FE780207723220490B240EC
:1019C0002244410182805971A2D437240020832708
:1019D000449086D6A6D2CAD0CECED2CCD6CADAC849
:1019E0000545638D070C9305F1041305F041EF8065
:1019F000512B9305F1041305F041EF80912AB7278D
:101A000000209387C7AD83C727000347F104B3378E
:101A1000F00011C38907032744903EDE03453700D9
:101A200093054700EFE03FA1032744902ADC0D45D2
:101A3000834527002EDAEFF00FB72AD81145EFF0D3
:101A40008FB6032444902AD665450347A400034B70
:101A5000B4003AD4EFF02FB5AA846945EFF0AFB4E3
:101A60002A897145EFF02FB4AA896D45EFF0AFB325
:101A70002A8A7545EFF02FB3AA8A7945EFF0AFB205
:101A8000E2046258F2572257B2564256D2551375A5
:101A9000F50F93FAFA0F137AFA0F93F9F90F1379F6
:101AA000F90FE1842ACC56CA52C84EC64AC426C28F
:101AB0005AC0930844000545EFB06019B65026544B
:101AC00096540659F649664AD64A464B6561828065
:101AD000011122CC06CE26CA8D472E846315F50649
:101AE00003C73500B7240020E94703D54500938498
:101AF000C4AD6316F70083D764006382A706EF6066
:101B0000306409C5835764002317F5000357A40008
:101B10008356840003566400835544000345340013
:101B2000EFE09FE40357440083D764006309F700A4
:101B30008547F2406244D2443E8505618280FD576C
:101B40002393F400F5B78967CD07631DF50083C7BC
:101B5000250031476385E7004547E39BE7FCEFE05D
:101B6000AFF0F9B7B1476319F500B727002003C5F7
:101B700057C2EFE0BFEA6DBF41677D178147E31AA7
:101B8000E5FA83C655004947E395E6FA83C5450063
:101B900003552400300023140100EF60B04649BF14
:101BA000411122C4372400208347249226C206C64E
:101BB0004AC01307E00FAE846386E7041307F00FF3
:101BC000130424926387E7021145EFB0FFFD15C1AE
:101BD000930700FD2300F50089472301F5008547A1
:101BE000A3009500A301F500AA8503450400EFC0FA
:101BF000AF8AF9572300F400B240224492440249CC
:101C0000410182802A891145EFB01FFA75D59307EB
:101C100000FD2300F50089472301F500A30095008E
:101C2000A30125012244B7270020B2409244024973
:101C3000AA8503C5379241016FC00F8679714AD0DA
:101C4000372900208327499022D406D626D24ECEAB
:101C500052CC56CA4544D5EFB7240020938704C21E
:101C600083C747004944958BCDC7B72700202E8AEC
:101C70009165A381A792AA8993857571314597E0F3
:101C8000FE1FE780203C2322A9904D4459C1230028
:101C90003501A30005002946D285090597E0FE1FFE
:101CA000E780005883274990914603C7270063EDDA
:101CB000E60835EB4D472381E70003C7270013678C
:101CC00007012381E700930571001305F041EF80C0
:101CD000417D83477100F1EBB727002003C7E7ADD3
:101CE0008D476314F70CEFE05F832C00EF70B04377
:101CF0002800EFE0FFE34545EFF0EF8A014411C90A
:101D0000130600643306C50203C504C29145EFC043
:101D10002FD22285B250225492540259F249624A7B
:101D2000D24A4561828085466314D700754761B702
:101D300089466314D7004947BDBF8D466314D70059
:101D4000414795BF554785BF9546CA8A630ED70060
:101D500099466316D70009472381E70031A01D4645
:101D60006314C702238107006545EFF0CF83930713
:101D7000F007E30AF5F403A74A908347270093E7A7
:101D800007042301F70081B721466314C700054704
:101D9000E1B725466315C7002381D700F1B7A946EF
:101DA0000544E318D7F6114745BF31392A8435D1A8
:101DB000CD3E85B7011126CAB724002083A74490E1
:101DC00022CC06CE4AC84944B1C783C707000D4498
:101DD0006392A70437290020034509C28945EFC053
:101DE000EFED034509C2B7270020914523920792E2
:101DF000EFC0CFEC83A7449001478146A3808700C2
:101E00001306F100854785450145A307F100EFA0C2
:101E100070672A842285F2406244D24442490561B7
:101E20008280011106CE22CC26CA4AC88547631E8D
:101E3000F506372400201304449283570400A9CBED
:101E400037270020034707AE21E71307B003636C71
:101E5000F702B724002003C504C28945EFC00FE68E
:101E6000035604009307006403C504C23306F60258
:101E70008945EFC0EFBB23100400F2406244D24416
:101E8000424905618280938747FC2310F400F5B72F
:101E9000B727002083A74790EDD36244F240D24495
:101EA000424903C50700056131B7B724002083A765
:101EB0004490E1D737270020130907C28347490020
:101EC000918BC5DF89476313F5062D452EC6EFB00C
:101ED000BFCD2A845DD1B245930700FD2300F500F4
:101EE000E547A30005002301F50083C7350015056C
:101EF0001946230FF5FE83C745009505A30FF5FE90
:101F000097E0FE1FE780C031034559009307F00FAB
:101F10006316F50083A7449003C50700A2856244B9
:101F2000F240D244424905616FB01FD7034507C252
:101F30008945EFC0AFD86244F240D2444249B72746
:101F400000202392079205616FF0BFA5494582806A
:101F5000B727002083C747C2958B638F071293076B
:101F6000C01C63FCC70009458280F2406244D24431
:101F70004249B249094505618280B727002083A7FD
:101F80004790638B0710B72700209387279203C8D9
:101F900007001307E00F6311E810011122CC4AC8B3
:101FA00006CE26CA4EC62380A7001305860042052A
:101FB000368932844181ADC991659385657197E019
:101FC000FE1FE7802008AA894DD1B724002003A571
:101FD000C4929384C49209C597E0FE1FE780C014A1
:101FE0001385890023A0A9002286814523A03401FE
:101FF00097E0FE1FE780E0299C402286CA8588433F
:1020000097E0FE1FE780C0219C40A286F240239209
:1020100087006244D2444249B249984305468D45FF
:10202000054505616FA0904591659385557197E0D1
:10203000FE1FE7802001AA890DD9B724002003A53F
:1020400044939384449309C597E0FE1FE780C00D35
:102050001385890023A0A9002286814523A034018D
:1020600097E0FE1FE780E0229C402286CA858843D5
:1020700097E0FE1FE780C01A9C40A286F2402392A0
:1020800087006244D2444249B249984305468D458F
:10209000054505616FA0D03E494582809307C01C6D
:1020A00063FCA700094582800945F2406244D2449E
:1020B0004249B2490561828045CD011122CC2A8472
:1020C00021054EC64205AE899165938565714181B2
:1020D0004AC806CE26CA97E0FE1FE780A0F62A89E6
:1020E00061D5B724002003A5C4929384C49209C586
:1020F00097E0FE1FE7804003130589002320A90015
:102100002286814523A0240197E0FE1FE780601806
:102110009C402286CE85884397E0FE1FE7804010D2
:102120009C4023928700B727002083A747908DCF3C
:10213000B727002083C747C2958B8DCBB7270020D8
:1021400083A7C79299CF984383D647006244F24051
:10215000D2444249B24905468D45054505616FA007
:10216000F03101478146DDB7014581B7494535BFAB
:10217000B727002083A7479095C7B727002083C7BC
:1021800047C2958B95C3B727002083A7C79281CB01
:10219000984383D6470005468D450545C9B7014795
:1021A0008146D5BF01458280494582809307C01C86
:1021B00063FCA700094582800945F2406244D2448D
:1021C0004249B2490561828045CD011122CC2A8461
:1021D00021054EC64205AE899165938555714181B1
:1021E0004AC806CE26CA97E0FE1FE780A0E52A89E6
:1021F00061D5B724002003A544939384449309C573
:1022000097E0FE1FE78040F2130589002320A90014
:102210002286814523A0240197E0FE1FE780600706
:102220009C402286CE85884397E0FE1FE78040FFD2
:102230009C4023928700B727002083A747908DCF2B
:10224000B727002083C747C2958B8DCBB7270020C7
:1022500083A7479399CF984383D647006244F240BF
:10226000D2444249B24905468D45054505616FA0F6
:10227000302101478146DDB7014581B7494535BF6A
:10228000B727002083A7479095C7B727002083C7AB
:1022900047C2958B95C3B727002083A7479381CB6F
:1022A000984383D6470005468D450545C9B7014784
:1022B0008146D5BF01458280494582809307C01C75
:1022C00063F4A70009458280797122D44ECE06D6E8
:1022D00026D24AD0AE892A842DC1210591654205B6
:1022E00093857571418197E0FE1FE780A0D52A890B
:1022F000094563060908B724002003A504939384C5
:10230000049309C597E0FE1FE78000E213058900EA
:102310002320A9002286814523A0240197E0FE1FE7
:10232000E78020F79C402286CE85884397E0FE1FF9
:10233000E78000EF9C4023928700B727002083A707
:10234000479001458DCFB727002083C747C2494535
:10235000958B95C76C001305D030EF90B133B24721
:10236000014593F7070F81CFB727002083A7079375
:102370008D450545944303D64700EFA0F010B250B9
:10238000225492540259F24945618280B7270020B5
:1023900083A7C79291CF03D647008C43411106C64D
:1023A00097E0FE1FE780C0E7B2400145410182800F
:1023B00009458280B727002083A7C7928DC7B7271A
:1023C000002003A74793894705C3035647000C43E2
:1023D000411106C697E0FE1FE78080E4B2408147C6
:1023E0003E854101828089473E858280797106D68B
:1023F00022D426D24AD04ECE52CC8D4763FCA700C1
:102400008944B2502254268502599254F249624AB4
:1024100045618280372900200347C9ADC144E312DA
:10242000F7FE9307F5FF9309C9AD93F7F70F8546BC
:10243000AE842A8403CA29001309C9AD63EAF606EB
:102440008DE199452800EFD0DFDCB729002003C5D6
:1024500009C2914523018900EFC04F8635E48144CC
:102460004DB719468145280097E0FE1FE78060E2DE
:1024700019462C00268597E0FE1FE780A0E749F16A
:1024800019469305F00F280097E0FE1FE78060E0F3
:1024900019462C00268597E0FE1FE780A0E52DF168
:1024A0001946A685280097E0FE1FE78060D771BF18
:1024B000E31DE5F803A5C9002C00EF70C046AA840F
:1024C00049D52381490135BF2800EFE06FE6AA8492
:1024D0000DED930571001305F041EF70917C83447D
:1024E0007100B5FC8D47E31CF4F64545EFE0BF8B6A
:1024F0003DD5B7771800938707A03306F50203C5CB
:1025000009C29145EFB05FF4EDBD23014901D5BD8E
:10251000B727002083C747C2918B8DC33725002082
:1025200041111305859206C6EFD01FCEB240B727E2
:1025300000207D572391E7AE4101828001456FD095
:10254000BFCCB72700207D57A381E792B727002093
:1025500079572381E792B7270020238007B8B72750
:10256000002023920792B727002023A60792B727BF
:10257000002023AA0792B727002023A80792372715
:102580000100B72700209387879C1307C77598C35E
:1025900037270100130727E2D8C3372701001307A5
:1025A000679C98C7B727010037270020938707AD9E
:1025B0002324F7928280411126C2B724002083A7EA
:1025C000449006C622C48DCF2A840D45EFB0CFDDDE
:1025D000AA8505C1930700FD2300F5008D47A300E0
:1025E00085002301F50083A7449003C50700EFB0E1
:1025F000AFEA19C42244B240924441016FF06FBA6D
:10260000B2402244924441018280797152CC372AEF
:10261000002083274A904AD006D622D426D24ECE16
:1026200056CA0149B1C703C91700B724002085471E
:10263000AA899384C4AD6307F90483C7440005499C
:1026400085EB0D45EFB04FD6AA8505C1930700FD78
:102650002300F5009147A30035012301F5008327EE
:102660004A9003C50700EFB02FE3EFF08FB30549A1
:10267000B25022544A8592540259F249624AD24ACF
:1026800045618280B727002083A7C792D28A85E35D
:102690000145EFE04FF12A8601CAB727002003C5A4
:1026A00007C28945EFB0DFB883A74A9081A8944359
:1026B00003D647009305E1000545EFD01FC069D957
:1026C00083470500858BE9D70545EFE0CFED9307FC
:1026D000B0032A8463F0A704B727002003C507C20C
:1026E0005D66130606708945EFB01FD6B727002038
:1026F000130444FC2392879283274A900947A380BE
:10270000E70083C7440081C72382040095B74E8544
:102710005D35B9BF130600643306C502B5BF41116C
:1027200022C42A840D4506C6EFB00FC805C593071D
:1027300000FD2300F500CD472301F500A30085002F
:102740002244B7270020B240AA8503C53792410131
:102750006FB08FD4B240224441018280835645003D
:102760000111896706CE22CC26CA138667002A8704
:102770006399C6001C47014583C50700EFF04FC2AF
:102780003DA8138687006397C6001C47054583C58F
:102790000700EDB7138697006395C602B7270020A0
:1027A00083A74790014595C7184703450700631164
:1027B000050E0547A380E7000545EFA04044054509
:1027C00009A81386A700639BC6001C4703C5070022
:1027D0002D3DF2406244D244056182801386670336
:1027E000E38AC6F813867703E381C6FA1386870364
:1027F0006392C60A1C45372400201307E00F83C4E8
:1028000007008347249213042492638EE702130780
:10281000F00F6386E7021145EFB00FB9AA8505C135
:10282000930700FD2300F5008947A30095002301CD
:10283000F500A301050003450400EFB0EFC5F9570B
:102840002300F400ADBFB727002003A747903E84C4
:10285000014541D38DEC85447D4523059100EFE092
:102860008FD42316A10013050002EFE0CFD38327F6
:102870004490A305A1001307B100A3809700740042
:102880001306A10085450545EFA0C03F0DBF268575
:102890001D3335B713869703E389C6F21386E70322
:1028A0006397C6001C45094583C50700C1BD9387D2
:1028B000F7030145E39FF6F01C4703C5070005E950
:1028C0006C001305D030EF90E15CB247414793F7BD
:1028D000070FE386E7EE9305B10013056031EF9033
:1028E000615B0345B1008545EFA0403AC9BD053D98
:1028F000F9B5B727002083C747C2411106C6958B9B
:1029000099CB372500201305859CEFD05F8F4D456F
:10291000B240410182800145EFD07F8E0145CDBF9D
:1029200003C70500937625009377D70F99C2936765
:102930002700131885011358884113F7F7076354CC
:10294000080013E70708937685009377770F99C2FD
:10295000936787001377050293F6F70D19C393E683
:1029600007022380D500634508009377A50281CB39
:102970008347060093E7C7002300F60082807DFDB1
:1029800083470600CD9BCDBF2D456319071403C8AF
:10299000050009476310E814C841034715000345C3
:1029A00005002207498F42070D654187930825A03E
:1029B000630B170B011122CC26CA4AC84EC606CE9D
:1029C000BE89B68432842E8963CEE800930705A0C1
:1029D000630DF702130515A06300A70623900400FA
:1029E0000545B5A0930745A06309F7086348F706B6
:1029F000130565AAE314A7FE85472390F600DC457E
:102A000083C707002300F60091A0C84597E0FE1F8A
:102A1000E780408B420541814E86637335012A86EB
:102A20002390C400420641828325C900228597D0A5
:102A3000FE1FE780E07E19A8DC4583D707002390BE
:102A400006012300F600A183A300F6000145F24031
:102A50006244D2444249B249056182809947239039
:102A6000F6001946D1B785472390F600DC450145AD
:102A700083C707002300F6008280DC45A9CB2147ED
:102A80002390E60003D707002300E60003D70700E2
:102A90002183A300E60003D727002301E60003D724
:102AA00027002183A301E60003D747002302E600A5
:102AB00003D747002183A302E60003D7670023035F
:102AC000E60083D76700A183A303F60041B72390F4
:102AD0000600ADBF2390060005458280828083C832
:102AE000050089476394F816DC41797122D406D633
:102AF00026D24AD04ECE52CC56CA03C8170083C73E
:102B000007002E8422083368F80042088D671358A6
:102B10000841138327A0630C68102A8A3A89B68477
:102B2000B285634C0301138707A0630BE802938708
:102B300017A06301F80A854711A8138737A063031C
:102B4000E80C138767AA8D47E317E8FEB2502254BA
:102B500092540259F249624AD24A3E8545618280C6
:102B6000484432C697D0FE1FE780C07542054181B8
:102B70009D47E36D25FDB72A0020938AAA9383C75A
:102B80000A00B3099900B24563D43701B5477DBF48
:102B900048442686C2094A9597D0FE1FE7804068C0
:102BA00003C60A00484493D9090105063306364195
:102BB00081454E9597D0FE1FE780A06DB727002076
:102BC00083A7C79399E3814751B79C438145E5DFCC
:102BD00052853DA0AD47E31B09F6E39916FB8347F9
:102BE0001600834606005844A207D58F2310F7002D
:102BF000B727002083A7C793F9D79C438545E1D722
:102C00008297D1B7AD47E31309F49947E390F6F8FB
:102C10004844194697D0FE1FE7808060B727002000
:102C200083A7C793CDD39C43D9DF8D4555B7AD4717
:102C300011FF8547E39CF6F403470600930700085D
:102C4000E3E6E6F0DC452380E700B5BF85473E8537
:102C50008280B727002023AE0792B7270020A38DDC
:102C60000792B7270020238D0792B7250020B707CA
:102C7000A0009385C58C938707059CC1B707E8031F
:102C8000DCC137D60200B71700209387477D1306B3
:102C900086EAD0C3B72E002037D602000947938EAC
:102CA0007E8C1306C6E7372E00202380EE00130E1D
:102CB0004E8CD0C723AED70137230020B728002081
:102CC000372800203725002037D60200B7DE020063
:102CD00085461306C6E82300EE009388888C23AE51
:102CE000C703130383931308688C1305558C938EC5
:102CF0004EE937DE02002380E8002380E7002388C6
:102D0000E7002380E7022388E7022380E70423000B
:102D1000E8002384D70023950700D0CB238CD7006D
:102D2000239D070023A2D7032384D70223950702FC
:102D300023A60702D0DB238CD702239D0702231092
:102D400003002300D500130E4EE823A2C7052388F5
:102D5000E70423AE17052380E7062388E7062380D0
:102D6000E708B7D8020037D70200130787E893882F
:102D700048EA23A2E7082384D7042395070423A65F
:102D80006704F0CB238CD704239D070423A21707E5
:102D90002384D70623950706ECD7F0DB238CD706D0
:102DA000239D070623AE07072384D708239507082A
:102DB00023A6A70837370100B72700209387478647
:102DC0001307879898C3373701001307E7ADD8C3B7
:102DD00023A407008280A54763ECA710B7D70200A1
:102DE000938787880A053E951C41011122CC26CA8B
:102DF00006CE4AC8B2842E8482879307800F63F977
:102E0000B7006145F2406244D24442490561828084
:102E1000371900209307497DC8571309497D09C90F
:102E200097D0FE1FE7804030B7270020238D079200
:102E300013061400916593850571328532C697D0CB
:102E4000FE1FE78020202326A90245DD324681456A
:102E500097D0FE1FE780E0430325C9022286A6859E
:102E600097D0FE1FE780C03BB7270020238D8792B5
:102E7000014549BF8947E396F5F803570600B72790
:102E80000020239CE792EDB7A147E39CF5F6372598
:102E900000202146A6851305C58C97D0FE1FE7802C
:102EA0002038F9B78547E39EF5F4B71500209385E0
:102EB000457DD04D9385850203C50400EFF05FA6E4
:102EC00045BF8547E39FF5F2B71500209385457D03
:102ED000D05D93858504CDB78547E394F5F203472C
:102EE0000600B7270020A382E78C59B7094519BF10
:102EF0000945828005476302E5044111AA8706C699
:102F00002E8581CF11476383E70425476388E70453
:102F10008947B2403E8541018280B727002083A5C2
:102F200007808947FDD5B727002003C6A79397D010
:102F3000FE1FE780E02E8147E9BFB727002083D737
:102F400087932390F50081473E858280B725002036
:102F500021469385C58CEF90B105F1BFB7270020BE
:102F600083C7578C2380F500F9B7B72700209387D4
:102F7000B79303C7070015E305472380E7000589DA
:102F800009CDB72600203715002093864686414696
:102F9000A5451305457D6F30406D014582800111C7
:102FA00006CE22CC0546638CC50211460944639EB9
:102FB000C5023EC63AC436C2EFD0EFC22A8492465A
:102FC0002247B2471DE13E86BA853685EFD00FB85D
:102FD000EFF03F92EFF0CFD3EF60107C39A0EFD04D
:102FE0008FC02A8419E1EFF0DF902285F24062441D
:102FF0000561828079714ECEAE896C0022D426D2D2
:103000004AD006D62A89B284EF00707A2A840DE16C
:10301000CE854A85EFC05F882A8419E93245B70614
:10302000010026879386A6882D468145EF10C012A1
:103030002285B250225492540259F249456182804D
:1030400079714ECEAE896C0022D426D24AD006D6F3
:103050002A89B284EF00B0752A840DE1CE854A85B5
:10306000EFC0BF912A8419E93245B70601002687CF
:10307000938606974D468145EF10000E2285B2508B
:10308000225492540259F24945618280397126DAFC
:10309000AE844C0022DC4AD84ED652D406DEAA8931
:1030A0003289368AEF00B0702A8431EDA685630339
:1030B000090283D704002C002314F10083D72400D5
:1030C0002315F100930720302316F10093078002A7
:1030D0002307F1004E85EFC00FF92A840DE559460C
:1030E000A6851305A1002304210197D0FE1FE780C8
:1030F00020131245B7060100528793864683254662
:103100002C00EF1060052285F2506254D2544259CF
:10311000B259225A21618280797126D2AE846C0024
:1031200022D44AD04ECE06D6AA893289EF00306822
:103130002A840DE1A6854E85EFC0EFF72A8419E9B0
:103140003245B70601004A879386868A3546A685AA
:10315000EF1080002285B250225492540259F24955
:1031600045618280BD47638CF50663E9B702A547D8
:103170006387F50663EDB7009947638CF5049D47B7
:10318000638FF5049547638CF50401458280B5474C
:103190006387F50463E1B704AD47F5B7DD47638E98
:1031A000F50263EAB700C947638BF502D947638626
:1031B000F502C547C9BFF5476383F50263E4B7006D
:1031C000ED47D1B793072005638BF5009307200DDA
:1031D0005DBF484582800841828008458280484121
:1031E00082809307F00F630EF506011126CAAA84A8
:1031F0001305000222CC4AC84EC652C456C206CE9F
:103200003A89B689B28A2E8AEFA01F9A2A844D4540
:1032100015C8930700FB2300F400A30054012311F9
:103220004401230234011305840061466305090249
:10323000CA8597D0FE1FE780A0FEA2852685EFA055
:10324000BFA50145F2406244D2444249B249224AF4
:10325000924A05618280814597D0FE1FE780600316
:10326000E9BF09458280011122CC06CE2A842306BB
:10327000B100A306C100EF50A06C15C18346C50084
:10328000B72700202147938707C2639EE60003C546
:10329000670078009306E0070146A2859937F2405F
:1032A00062440561828078009306E0070146A285AA
:1032B00003C55700E5B7930700643306F6026FB005
:1032C0006F8C05C90347050085469307270093F7D0
:1032D000F70F63F0F602411122C42A843A8506C62C
:1032E000EFB0CFA4FD572300F400B24022444101C7
:1032F00082808280035705009307000B6313F70257
:10330000834745004947639CE7000347150185470C
:103310006399E7000355250085456F3090646D473C
:10332000C5BF828001112314B1006C0022CC26CAD3
:103330004AC806CE2A89B6842315C100EF0030475B
:103340002A840DE12C004A85EFC02FC82A8419E990
:103350003245B7F6000026879386267815462C005E
:10336000EF00905F2285F2406244D24442490561F9
:1033700082807971930720302314B1002315C10096
:103380002316F1002C0093078002014606D623077E
:10339000F100EFF0BFCFB25045618280C177797103
:1033A00085073EC4894726D22316F100AE849307D1
:1033B00080024C0022D44AD006D62A892307F10085
:1033C000EF00F03E2A840DE12C004A85EFC00FD8B3
:1033D0002A8419E91245B70601002687938686914B
:1033E00045462C00EF0050572285B250225492548B
:1033F000025945618280B28605466FF03FC97971F6
:1034000026D2AE846C0022D44AD04ECE06D6AA89EB
:103410003289EF00D0392A840DE1A6854E85EFC0B0
:10342000EFB12A8419E93245B7F600004A8793863E
:10343000E6710D46A685EF0030522285B250225427
:1034400092540259F2494561828079719307202094
:103450002314B1002315C1002316F1002C0093079B
:103460008002014606D62307F100EFF03FC2B250BA
:1034700045618280011122CC06CE2A842EC632C438
:1034800036C2EF50E04B0DCD0345C500B7270020F5
:10349000A146938707C212472246B245631CD50056
:1034A00003C56700B2862E86A2856244F24005619C
:1034B0006FF03FD3B28603C557002E86A285F5B7BD
:1034C000F24062440545056182806FF0BFB26FF043
:1034D0007FB26FF07FC46FF03FC479714ECEAE897A
:1034E0006C0022D426D24AD006D62A89B284EF00B4
:1034F000102C2A840DE1CE854A85EFC0AFBD2A8409
:1035000019E93245B706010026879386668C3D4649
:103510008145EF0070442285B250225492540259E2
:10352000F24945618280B28601466FF03FB60111D3
:1035300022CC2E846C0026CA06CEAA84EF00302747
:10354000DD47630AF500930710102314F400A285E9
:103550002685EFC08FC2F2406244D244056182806A
:103560002394050083D7850099E36FF07FAD09456B
:103570008280FDB7B727002003C76797854763F9A7
:10358000E702011122CC2E846C0026CA06CEAA8442
:10359000EF00F02109E9930700102314F400A2853D
:1035A0002685EFC08FBDF2406244D244056182801F
:1035B00059458280B727002023A0A7948280B7278F
:1035C000002023A2A7948280011122CC26CA06CE15
:1035D0002A84AE84EF50C036A6852285EFB03FE145
:1035E0000DE9228523169100EF5080351DC18346D9
:1035F000C500B72700202147938707C26390E602E2
:1036000003C5670078009306F0070146A285EFF036
:103610005FBDF2406244D2440561828003C5570019
:10362000D5B7011126CA06CEB68422CCDD4663E2A8
:10363000B608D94663FED50AA5466381D50A63EE6E
:10364000B6049546638CD50899466387D50A054428
:1036500041687D18631606093AC6EFB01FDD3306D0
:103660008540324742064182420441803305C4000E
:103670004205BA85418132C6EF30D03FAA8749C1A1
:1036800081C432462390C400B30580406244F240B6
:10369000D2443E8505616FA0CFC4C5466380D50482
:1036A000C9460D44E395D5FAC167FD17E31EF6FA46
:1036B00065B7F5466380D50463E4B600ED46D5B73B
:1036C000930620056388D5029306200DE391D5F873
:1036D000C167FD170D446319F600BDBF09448DBFD6
:1036E0009306200DE392D5F8310642064182ADBF24
:1036F00015445DBF0D444DBFC167FD171D447DB727
:10370000F2406244D24405618280011122CC26CA73
:1037100006CE03C645002E84130700028146994554
:10372000AA8401372AC629CD8357040003464400E2
:10373000930554002310F100835724002311F10056
:1037400089472312F100930780022303F10097D0E9
:10375000FE1FE780E0AC834744008A85268523145A
:10376000F100EFC04F892A8411C5324597D0FE1F62
:10377000E780809B2285F2406244D24405618280CA
:103780004D44CDBF5D7186C6A2C4A6C2CAC04EDE7E
:1037900089476306F600C14709446319F6040144EA
:1037A000B1C52E894C0832C6B689AA84EF00300014
:1037B0002A84324605EDC1778507CA851305D101F4
:1037C0003ECC230EC10097D0FE1FE78060A52C08D9
:1037D0002685253F2A8419E95245B7F600004E8711
:1037E0009386A67D1D462C08EF0010172285B64053
:1037F000264496440649F25961618280797122D447
:1038000036844AD04ECE52CCB2892E8A3A8981462D
:10381000130710022286D94526D206D6AA8411356E
:103820002AC629C12286CA85231481002312410198
:103830002313310197D0FE1FE780809E4C00268520
:10384000EFC06F9E2A8411C5324597D0FE1FE780D6
:10385000A08D2285B250225492540259F249624AF4
:10386000456182804D44F5B7011122CC26CA06CEAF
:103870004AC8DD472A84AE84638DF502814703552B
:1038800004006C002306F100EFC06F9D0545638DB9
:10389000A40803458400B165938505B8EFA0BF83F4
:1038A000E5472301F400B7070100938747A55CC0F3
:1038B0009DA8034755013149B286330627031849AD
:1038C0009C4232971043E31BF6FA83D74600035617
:1038D0004700E315F6FA8C46084797D0FE1FE780AD
:1038E00060A149DD8347540103474401850793F7ED
:1038F000F70FA30AF40063FFE702B3872703184812
:1039000003550400BA97984783D6470003D627008B
:1039100083D50700E5353DF103458400B165938506
:1039200005B8EFA04FFB5945F2406244D2444249EA
:10393000056182808347640199B7011122CC26CAB0
:1039400006CEDD472A84AE84639BF5060355050049
:10395000EFB0BFAD0356C4018356240103574401A1
:103960006D162A9642064182B307D640C207231E2F
:10397000C400C18363F0E7089305C5FF3308F7402F
:10398000635BB802BA96918EC206184C8355040147
:1039900003550400C1823E97953515E10345840027
:1039A000B165938505B8EFA00FF35945F240624425
:1039B000D244056182806D1593160501F9B78147E0
:1039C000035504006C002306F100EFC04F89054544
:1039D000E38EA4FC03458400B165938505B8EFA090
:1039E0008FEFE5472301F400B7070100938747A550
:1039F0005CC065BF8547E9B7397126DAAE842C0013
:103A000022DC4AD84ED606DE2A89B2894D232A8482
:103A100021ED4A85EFB07FA183D644006D1563C5C3
:103A2000A60093160501C182984403D6240083D5CD
:103A300004004A85EFF09FDC2A841DE53146A68507
:103A400008082306010097C0FE1FE780607D83D72A
:103A500024002245B70601004E879386269E5D46C8
:103A60006C00231EF100CD2D2285F2506254D254F9
:103A70004259B2592161828041B7BDBF797126D2C6
:103A800006D622D44AD04ECE52CC56CA5AC8894401
:103A9000C5C159CE2E842A89BA8A368B328AEFB0B4
:103AA000DF98930544008147711503D705006352E1
:103AB000A70A850793F7F70FB105E318FAFE8A8581
:103AC0004A85F521AA842DE531453305AA02916581
:103AD00093851570CD4497C0FE1FE780A056AA8934
:103AE00021C931463306CA02A28597C0FE1FE7806E
:103AF0002073184483564400035624008355040061
:103B00004A85EFF0BFCFAA841DED0245B70601003C
:103B1000854756879386269E5D464C002302F1001A
:103B20004EC423064101A3060100230761012D2590
:103B3000B2502254268502599254F249624AD24A1E
:103B4000424B456182804E8597C0FE1FE780C05D75
:103B5000C5B7ED44F1BF79714ECE37D60200AE89BC
:103B6000C16526D20147AA848946130606EBFD15D6
:103B7000054522D406D64AD0EF10301A054431CD7F
:103B80002A891307300281461146F5452685EFF054
:103B90005FA92AC6554431C18357A900CE86014684
:103BA0002314F10091472315F10085472300F50008
:103BB000B2472C002685A38007003247FD5723011A
:103BC000F7003247A301F700EF10F00A2A8411C56D
:103BD000324597C0FE1FE78020552285B2502254FF
:103BE00092540259F24945618280411106C6EFF0B4
:103BF0006FD719C5B240410117C3FE1F6700C352FA
:103C0000B24041018280011106CE2AC6EFB0CFE753
:103C10003245B727002023A00794B727002023A20E
:103C200007949145B7270020A380A7C2EF30E05E3C
:103C3000F24005616F20F0387971939705014AD001
:103C400006D622D426D2C187014963DE070AB727E8
:103C5000002003C517C22E89EF901FFC2A844DC196
:103C6000034705009307000A6319F70885474C08C6
:103C7000A305F100EFB06FEEAA840DED834761015B
:103C800071476379F708138717FE1377F70F9306C9
:103C9000000263F8E608858BD5CBB727002083A701
:103CA0000794994481CB035524001306B1004C08B6
:103CB0008297AA848347B10099C7084409C597C071
:103CC000FE1FE780604695E05247B70700019387E3
:103CD00007F07D8FB707120093870710630FF70077
:103CE00003476101ED47631AF7000355240085453A
:103CF000EF302047CD476388F4002285EF90BFE581
:103D0000A1673349F900B25022544A8592540259AE
:103D1000456182803707301405073357F700058B5C
:103D20003DDB372700200327479449D7034751013C
:103D300051F32306F10099472308F10003552400AD
:103D40006C0023170100EFB0DF85ADB7B727002067
:103D500083A747949DC3035524001306B1004C0864
:103D6000829729D9AA8483475101A9F78347610122
:103D7000230891002306F100D1B79944EDB73971BA
:103D800022DC26DA06DE4AD84ED652D456D25AD093
:103D9000A5472A84B2846399F510834745020357E7
:103DA0000600835A260085072302F5029307F7FFD2
:103DB000B387FA025442C207C183B69703C91700FA
:103DC00083C707008346C50022093369F900854788
:103DD0006390F60233075703231006008149014A16
:103DE000130B3501931A070193DA0A0163E15907AE
:103DF000C167FD176302F90C83570401637EF90A5A
:103E0000050942098346C4001359090123172401F7
:103E10000547035504009305E400639FE60023155E
:103E2000F100930720302316F1009307800223143A
:103E300021012307F1002C00EFB0FFA2034584000D
:103E4000B165938505B8EFA00FA95945BDA083D6EC
:103E50002400DC4083452401ED1613865900C20678
:103E6000C1823E965A85EFB0AFC705C9630C3A01CF
:103E7000C84003D62400B3053501529597C0FE1FF4
:103E8000E780003A83D724003E9A83D70400420A91
:103E9000135A0A0185072390F40083D72400BE99A2
:103EA000C20993D9090199B703474600A94763108E
:103EB000F7028347450281CF0145F2506254D25444
:103EC0004259B259225A925A025B2161828083463A
:103ED00024011309340137D502004A8689451305A8
:103EE00085EAEFB0EFBF19C10545C1BF8346240184
:103EF00037D502004A8689451305C5EAEFB04FBEA3
:103F000065F58346240137D502004A8689451305A5
:103F100005EAEFB0EFBC69F98346240137D502000A
:103F20004A8689451305C5E8EFB08FBB55FD03C729
:103F30004400BD47E3EAE7FAA56793874712B3D782
:103F4000E700858BD5D38347440285072302F4021B
:103F500003D9240071BDB727002003C687C2B72745
:103F6000002003A7879481476315F60081463685B4
:103F70008280BA8613078702835587FDE389A5FEF1
:103F8000850793F7F70FCDB7011106CE2EC6E1379F
:103F900001CD8347A500B245138717006396E5005E
:103FA00093F707F82305F500F240056182800111BF
:103FB00006CE2EC64D3705C5B24591C188C183478F
:103FC00085001307E00F5D456388E7001307F00FD6
:103FD00001456383E7005945F24005618280094548
:103FE000E5BF411122C42A84210506C626C24AC063
:103FF000EFF02FAD83472400A51793F7D70F91EB70
:104000000347C40085476310F7061C4881443149C3
:10401000A9E3FD5723010400A304F40023020402D2
:104020001305C4002244B2409244024961468145CE
:10403000410117C3FE1F6700C325B38724033E95C4
:10404000084509C597C0FE1FE780000E850493F45C
:10405000F40F834744010848E3E1F4FE97C0FE1FD4
:10406000E780800C7DB7084C75F965B7411122C413
:10407000416406C626C29307E4FF630CF500AA84D8
:1040800091EDD13D19E51305F4FFF13519C1231068
:104090009500B24022449244410182808547639456
:1040A000F504EFF05FEB2A846DD5FD572310F50082
:1040B000834784001307F00F6384E7021307E00FC0
:1040C000638BE70083462400034594000147514673
:1040D000A685EFF00F9122852937FD572304F400C0
:1040E000230504007DB78947E395F5FA8545EF4040
:1040F000902845F12685EFF01FE62A8455F951BF37
:1041000039C9034785009307F00F6306F7040111CF
:1041100022CC06CE2A84834625008355050003451C
:10412000950001475D46EFF0CF8B03472400E14740
:104130006319F700035504006C0023060100EFB07B
:104140001F92F9572304F4002285EFF09FE9F24013
:1041500062440561828082809307F00F6306F70650
:10416000011122CC26CA2A844EC6AE84B689AA85FD
:1041700093068500374501004AC852C43A89328AFD
:1041800013050510794606CEEFF0EF92A304240143
:10419000230144012322340185C01305C400624475
:1041A000F2404249B249224AA685D244614605619D
:1041B00017C3FE1F6700C306F2406244D24442495F
:1041C000B249224A056182808280B7270020238677
:1041D000A79482809547639CF506834745028546F0
:1041E00085072302F502835706005842034626003E
:1041F000FD17C207C1836318D6048A07BA9703C79D
:10420000170083C707002207D98F0357E50063F91A
:10421000E704411106C622C485072316F5002A8447
:104220009305C50003550500EFB02FDA0345840060
:10423000B165938505B8EF901FEAB2402244D94793
:104240003E8541018280C946B387D70245BF834678
:104250004600294785476396E6000347450211C398
:1042600081473E8582809D476392F50683474502DC
:104270008356E50085072302F5028357060058425E
:10428000FD178A073E978347170003470700A207D9
:10429000D98F014763F6D704411106C622C48507AA
:1042A0002A842316F5009305C50003550500EFF099
:1042B000CFC503458400B165938505B8EF90BFE194
:1042C000B240224459473A854101828083464600E4
:1042D000A94705476396F6000347450213371700C1
:1042E0003A858280411122C406C626C2B5472A8477
:1042F000639BF50483474502B28485072302F502D8
:1043000003550500EFB06F9283D704001307F5FF44
:10431000014563C5E7020357E40003550400930514
:10432000C400BA972317F400EFB0EFD80345840018
:10433000B165938505B8EF901FDA5945B240224424
:10434000924441018280034746009D470545E3179B
:10435000F7FE0345440213351500CDB7C547639EEC
:10436000F5068357060003572600FD17B387E702BB
:104370000347450205072302E5025842C207C183ED
:104380003E978347370003472700A207D98F41672D
:104390007D176395E70081473E858280138717006C
:1043A0002316E5000357E500E3F7E7FE411122C4B9
:1043B0009305C5002A840355050006C6EFB00FD942
:1043C00003458400B165938505B8EF90DFD0B24016
:1043D0002244D9473E8541018280834646002947D1
:1043E0008547E39BE6FA0347450255F775B7011188
:1043F00022CC26CA4AC852C406CE4EC683C7250060
:1044000015472A8AAE8432843689639DE70436864E
:10441000A2852685EFF01FDCAA8955E98547631838
:10442000F40A03474900A9476301F70203C5940052
:104430004A8785460146D285EFE0BFDA19E5854512
:104440004A85EFE03FD21334150083C6240003C52C
:10445000940001476946D285EFE0BFD82685EFF08A
:104460005FB851A01D476398E7003686A285268570
:10447000EFF07FDF55B725476398E7003686A285C2
:104480002685EFF0DF8F49BF35476398E700368612
:10449000A2852685EFF01FE541B745476398E70001
:1044A0003686A2852685EFF07FEBBDB75D47639F1B
:1044B000E70003C7C50085473686A2852685631DAC
:1044C000F702EFF06FBA8547631BF5048549A547EE
:1044D0006317F402835709009DE30544E38709F657
:1044E000D947E39DF9F62285F2406244D24442491D
:1044F000B249224A05618280EFF02FC4E9B703C5B3
:1045000094004A87A2860146D285EFE09FCD71F5DF
:10451000A2854A85EFE01FC513341500C1B70544D5
:10452000D9B7397122DC06DE26DA4AD84ED652D403
:1045300056D283D705001944B1E783C925002A89DB
:10454000328A938759FE93F7D70FAE84DDE7B727FA
:10455000002083C6C7941307F00F938AC7941944A9
:104560006382E602F5476394F904EFF0DF9EAA89BF
:1045700021C10346A5000DCE93178601E18763DDB7
:10458000070001442285F2506254D2544259B25974
:10459000225A925A21618280F5454A85EFE0BFCCCC
:1045A00083C7A90093E707F82385F900D9BF81499C
:1045B00083D64400904483C5140003C5040038002A
:1045C000EFB0EFCA2A845DFD83C6240003C50A004C
:1045D00038000146CA85EFE0DFC02A8445F5B247BE
:1045E00099C323000A0083C724007547E39BE7F8BB
:1045F000E38909F82385F90071B7EFF0DF95AA8AFE
:1046000049D185476391F90A83D544008844300035
:10461000EFA09FE32A843DF503C72A00C54763F254
:10462000E70ADD476301F70CB727002003C59A00AE
:1046300083C717C2639CA70A014403C72A008D479A
:10464000631FF7048357810003D7CA0063F4E700B0
:104650002396FA0083D5CA004A85EFE0FFF6B72714
:10466000002083D787A86D47637BF70283D5CA00F4
:104670005D476376B7021387350091056349F700FC
:104680001307B00FBE856374F7009305B00F116672
:10469000C20513060629C1814A85EF8080535685DD
:1046A000EFF03F94C5B5834725001144E39C37EDF7
:1046B0005C41E38907EC83D544008844300082974D
:1046C00091BFB72702009387072AB3D7E700858BEE
:1046D000A1DF03C624003400D6854A85EFF03FD120
:1046E0002300AA0045B583A70A01DDB783C62400CD
:1046F00038000146CA85EFE0DFAE2A841DFD83C580
:1047000024002800EFE01FA605D923000A0035B7D2
:10471000011122CC3724002006CE26CA4AC84EC634
:1047200052C4930904C203C58900930780029165AE
:104730003305F50293856570372900209304899429
:1047400097C0FE1FE780009003C689009307800290
:1047500081453306F60288C097C0FE1FE78060B32C
:104760009C404D45A1C3930404C21309899401449C
:10477000130A8002FD5983C78400636DF402374534
:10478000010013052552EFE0FFE237450100130554
:1047900085F8EFA05FBB374501001305C506EF4064
:1047A000A0340145F2406244D2444249B249224A0F
:1047B00005618280B30744030325090061468145F2
:1047C00005041374F40F3E952310350123010500F1
:1047D000231435012305050023020502310597C086
:1047E000FE1FE78000AB41BF01458280B727002054
:1047F00083C697C2814763E5D70001473A85828027
:104800002E87910503D6C5FFE30AA6FE8507E5B707
:104810000DCD834725000547890793F7F70F63768A
:10482000F702411122C406C62A84835505000345B8
:1048300035000147F9465D46EFE0BF9AF95723116D
:10484000F400B2402244410182808280B7270020D8
:1048500003C797C2FD56814763E3E70082802310B8
:10486000D5002301050085071105FDB701458280AC
:10487000372600201306368E930700022300F60029
:1048800037270020FD572301F78E37270020A30A82
:10489000F78C37270020230AF78C8545B72700209F
:1048A0002390B78EB727002023970794B7270020BF
:1048B00023AC0794B727002023A40796B72700202E
:1048C00023AE0794B7260020B7D702009386868DC3
:1048D0009387C7E9DCC2B727002023880794B7274E
:1048E00000209387078709472380E6002380E7009D
:1048F0002388E7002380E7022388E70237D70200F6
:10490000130707E9D4C7D8DBB7D602000D47238CBD
:10491000E7029386C6E837270020D4CB03274795C4
:1049200037D50200B7D60200130585EA938606EB59
:10493000C8C32384B70023950700238CB700239DA9
:104940000700D0CFD4D3238407022395070223A6E0
:104950000702239D0702D8DFB72700203757010041
:104960009387078B130787A223A00700D8C323A42C
:1049700007008280411106C6EFF05FE711C50345CD
:104980002500B240410182800145E5BF411122C4AA
:1049900026C24AC006C6AA842E893284EFF01FE5DB
:1049A00011E94165CA857D15EFF05FE4C54711C582
:1049B00023109500230185008147B2402244924490
:1049C00002493E854101828029E789483547639342
:1049D0001605011106CE22CC26CA0347160003464F
:1049E000060093C7F7FF2207598EF18F32C68DE775
:1049F000C4452A84A685EFF0FFF732460147630FCE
:104A0000A60022856244F240A685D24405616FF07B
:104A1000FFF72D473A85828013070008F240624471
:104A2000D2443A850561828083C8050009486395B0
:104A3000080303A845008347180003480800A2079D
:104A4000B3E70701C2070D68C18713082890639573
:104A5000070189476FF05FF705458280011122CC7D
:104A6000372400201304548D0347040006CE26CAC1
:104A70004AC84EC69307F00F6300F704AA89294578
:104A8000B2842E89EF904F9205C99307100B231023
:104A9000F5002302050023113501231325012314FA
:104AA0009500AA85034504006244F240D24442497D
:104AB000B24905616F904F9EF2406244D244424930
:104AC000B249056182804111B727002026C2AE8419
:104AD00083A5479522C406C62A84EFF0BFE9098959
:104AE00009C922852244B240A685924441016FF053
:104AF0008F86B24022449244054541018280411193
:104B000022C426C24AC006C6AA841304450013095B
:104B1000850B835704009DC3084409C597B0FE1F49
:104B2000E780806022853146814597B0FE1FE7808F
:104B300040763104231A04FEE31D24FDB2402244D2
:104B4000FD572390F4000249924441018280B72727
:104B5000002003C697C2B727002003A70796814706
:104B60006315F600814636858280BA861307870B67
:104B7000835587F4E389A5FE850793F7F70FCDB733
:104B8000B727002083A7879689CB03D747006314F4
:104B9000A700884782809C43C5BF014582804111A0
:104BA00006C6F93F09C50845B2404101828001456A
:104BB000E5BF011126CA9384450022CC4EC606CE1D
:104BC0004AC852C456C25AC0268781490144814608
:104BD00081473D450356070055CED9E203544700AF
:104BE00083572700B286A297C207C1838509310780
:104BF000E392A9FE25C82E8991659385457022858B
:104C000097B0FE1FE78000442A8B29CD814A014AD4
:104C10008C4485C503D6440033054B0197B0FE1F75
:104C2000E780006083D7440088443E9A420A135AC2
:104C30000A0197B0FE1FE780204F63890A003146C2
:104C40008145268597B0FE1FE780A064850AB104E0
:104C5000E3E03AFD2326690123148900054521A0DC
:104C6000630DD6000145F2406244D2444249B24944
:104C7000224A924A024B0561828003562700E313C1
:104C8000F6FE035647003294B2974204C2074180B1
:104C9000C183A9BF0545E37835FDA9BFB72700202B
:104CA00083A7C79599E30145828098470357A700DA
:104CB0006315A7001385470082809C43E5B7411127
:104CC00006C6E93F11C503550500B2404101828087
:104CD0000145E5BF411106C6D13711C50345250081
:104CE000B240410182804145E5BF411122C42A847E
:104CF0002E8506C6C537AA8505462285EF30704742
:104D000095476305F500BD476313F5002145B240A3
:104D10002244410182804111B727002022C406C6E7
:104D200003A4C79581469387C79529C018440356A5
:104D3000A70018406317A60285CA98C22E8581C9AC
:104D400021469305440097B0FE1FE780604D228501
:104D500097B0FE1FE780403D0145B240224441012B
:104D60008280A2863A84D1B798C3C9BF0545F5B7FA
:104D70003727002083278796014613078796A9C700
:104D800003D847009443631CA802011106CE22CC2D
:104D900026CA0DCA14C2AA843E852E8497B0FE1F6F
:104DA000E78080382C002685EFF0FFF601E519C07A
:104DB000B2471CC0F2406244D244056182803E8604
:104DC000B68775BF14C3C1BF05458280411122C497
:104DD0002A84090506C6EFE0CFCEFD57A301F400F3
:104DE000B240224441018280B727002003C797C206
:104DF000B727002083A747962A86050781463E8568
:104E000083D707006388C700850693076500E3E83A
:104E1000E6FE01458280411122C4416406C626C2D5
:104E20009307E4FF630EF500AA8485E1EFF0DFFB52
:104E300001E91305F4FFEFF03FFB19C123109500C2
:104E4000B240224492444101828085476394F50434
:104E5000EFF09FF92A846DD5FD572310F5008347A5
:104E600024001307F00F6384E7021307E00F638A3F
:104E7000E700034534000147F9465146A685EFE0B7
:104E80004FB62285EFF09FF4FD572301F400230273
:104E900004007DB78947E395F5FA8545EF30B04DBD
:104EA00045F12685EFF05FF42A8455F951BF1D7155
:104EB000A6CACEC686CEA2CCCAC8D2C4D6C2DAC0D2
:104EC0005EDEAE8483C52500F947AA896397F504A1
:104ED000EFF09FF12A8411ED01442285F6406644EB
:104EE000D6444649B649264A964A064BF25B2561A6
:104EF0008280834725000547890793F7F70FE37DF5
:104F0000F7FC034535000147F9460146CE85EFE041
:104F10004FAD2285EFF09FEBC1B703AB0400B7079D
:104F20000001938707F037071200B377FB001307E0
:104F30000710B28A0149638AE7022EC6EFF0DFEA62
:104F40002A89B2451DC10346450005C29317860153
:104F5000E187E3C307F84E85EFE0EFB083474900F0
:104F600093E707F82302F90085BF372A002003479B
:104F70002A8E9307F00F130A2A8E1944E30FF7F4D1
:104F8000E147E3ECB7F493D71500FD17139737000B
:104F9000B7D702009387078BBA9703A80700E30EE1
:104FA00008F283AB4700E38A0BF2420B135B0B0161
:104FB00063050B00C947E392F5F283D644009044A1
:104FC00083C5140003C50400380802982A84E31638
:104FD00005F02C084E85829B2A8421C983C71400C2
:104FE000E39D07EE83C72400230AA1003947230865
:104FF000F1006399E7026247834717000347070000
:10500000A207D98F0C084E852319F100EFA06FD9A4
:10501000E30405EC14080546D9454E85EFE08FC53D
:105020002A8465BD83578101F1BF83C6240091475F
:10503000E384F6EA03450A0038080146CE85EFE02E
:105040004F9A2A84E31B05E883C524002808EFE073
:105050006F9119C123800A009840B7070001938718
:1050600007F07D8FB707120093870710E306F7E676
:10507000E30409E683C724002302F900B9BD011146
:1050800006CE2EC6EFF05FD601CD83474500B24570
:10509000138717006396E50093F707F82302F500DE
:1050A000F24005618280B727002003A7C79519E366
:1050B000014615A81C4703D8A700636B0501835858
:1050C0004700B38608016355D500814663941601F5
:1050D0001843F1BF3E86C10703D3A7FF6317A300A0
:1050E00099C123900501328582808506C206C1825E
:1050F000F1BF397152D42E8A4ED69305E101AA89A7
:10510000528522DC4AD856D206DE26DA328936C6E5
:105110003AC4BE8AEFF03FF9054435C5AA84035569
:10512000E1013944EFF0DFA539CD03284500630CD8
:1051300008042247B246D6874A86A6854E8502983D
:105140002A8431E19307E00F638FFA0203C704005A
:105150008947631AF702D8408347170003470700BF
:10516000A207D98FC2070D67C18713072790639CD9
:10517000E7008347190003460900D285A2075D8E28
:105180004E85EFF0BF8D2285F2506254D2544259C1
:10519000B259225A925A21618280797122D40354E1
:1051A00025004ECEAA89228556CA06D626D24AD0D6
:1051B00052CC5AC85EC662C4AE8AEFF05F9901E96C
:1051C0002285EFA01FDE594429E90144B9A003C795
:1051D00089008547AA840144631AF702AA851385CA
:1051E0008900EFF01F9D29CD03D7640083D684008A
:1051F000D04483D5440003D52900E147EFF07FEF89
:10520000D9472A846318F50223A604002685EFF007
:105210001F8F49C0D947E30AF4FA2285B2502254BD
:1052200092540259F249624AD24A424BB24B224C42
:105230004561828061DD83D744002390FA00F9B78D
:1052400013894400014AB94B594C3D4B8355090021
:10525000D5DDE14763067A010357C90011C3D94779
:1052600003572900835649000326890003D52900E6
:10527000EFF03FE82A846319850123240900050A19
:105280003109E3156AFD59B77DD983570900239089
:10529000FA00F5B703D529002DB701112317C10076
:1052A0009307E00F1306E1000147894606CEEFF0B1
:1052B0005FE4F24005618280797122D42A8403552B
:1052C000850026D2AE849305210106D64AD0EFF0A0
:1052D0009FDD6308050E834785002AC693F7070202
:1052E0008DCF03552101EFF09F8BAA87B24501EDC9
:1052F0008357840039452390F400B25022549254CD
:10530000025945618280035524004946829711C5A0
:10531000835784002390F400CDB7035924004A85B5
:10532000EFF0FF8211ED41657D15EFF05F8219E529
:105330008357840025452390F400C1B7231025012D
:10534000130745008147BD46035607002DE6314748
:10535000B387E702130984003146CA8591073E9559
:1053600097B0FE1FE780C0EB3146CA85480897B06A
:10537000FE1FE780E0EA0356C400035524004147BE
:105380008146DD45EFE0EFA92ACE19E58357840079
:1053900045452390F40095B70C480356C40097B0D8
:1053A000FE1FE780E0E7035524004C08EFA03FBB59
:1053B00029D5594599B785073107E397D7F825458A
:1053C00081BF0545B1B7797122D42A840355850080
:1053D00026D2AE849305E1014AD006D63289EFF099
:1053E0009FCC51C58347850093F70702A9E7034780
:1053F00014019307200519E3834744008356A40052
:10540000504483558400035524000147EFF07FCEBC
:10541000AA8721E98347140199E703552400EFA0E7
:105420003FAFD94711E18147B250225492540259FB
:105430003E85456182802AC60355E101EFF02FF6D3
:10544000AA8705C9B2450355240049468297AA8711
:1054500059DD035784002390E4000347140161F7EA
:10546000E1B75947E317E5FE230009006DBF854703
:10547000CDB7B947F9BF397122DC4AD84ED652D4DC
:1054800006DE26DAAA892E8A32C63689EFF0DF9543
:10549000094415C5834725001307E00FAA845D441E
:1054A000638FE7001307F00F5944639AE700324611
:1054B00005E2D2854E85EFA0BFB22A8415CD2285A4
:1054C000F2506254D2544259B259225A2161828018
:1054D00003550A009305E101231F0100EFF0BFBC53
:1054E0000355E101EFF00FFFAA8505464E85EF3029
:1054F00040482A845DDDE1B79307F00FE301F9FC32
:1055000037550100938624007946A6851305058149
:10551000EFD07FDAA38124015DB73971B72700206E
:1055200026DA83A4C79552D45AD05ECE62CC06DE6A
:1055300022DC4AD84ED656D266CA2A8BAE8B328C23
:10554000368A99E08149B9A0804483DC440001494E
:10555000835AA400631499018440E5B78357A400DB
:10556000A28963F867010509420913590901410439
:10557000D5B7E3EAFBFE630C0A008345040048400C
:10558000D28662863AC6EF90BFD5324769DD19C32D
:1055900023105701F25062544E85D2544259B259E9
:1055A000225A925A025BF24B624CD24C21618280A9
:1055B00003D7050083D62500854763E9E60439C78C
:1055C000411183C6450026C237D502009384550099
:1055D00022C426862E84130585EA894506C6EF90E7
:1055E0003FD0C14711CD8346440083552400035565
:1055F000040001472686EFF05FF2814711E1A947D9
:10560000B240224492443E85410182803E858280A0
:105610002E860355060083D52500854763E2A50243
:1056200005C18346460041110147150606C6EFF045
:10563000DFEE814711E1A947B2403E8541018280FA
:105640003E8582802E860355060083D5250085473A
:1056500063E2A50205C183464600411101471506D4
:1056600006C6EFF09FEB814711E1A947B2403E85A6
:10567000410182803E85828039714ED683D72500D4
:1056800083D9050006DE22DC26DA4AD852D456D267
:105690005AD05ECE62CC66CA6AC863E037198547C5
:1056A000638E0914416BAE8A2A8A2314010002C654
:1056B000014401497D1B894B054CC94C054D83D5DF
:1056C0002A000147814601464E8523130100EFF071
:1056D000DFE4AA846300051209EC13072002930695
:1056E00061005A8695455285EFD0BFF32A8463083E
:1056F00005120357810083C7040045C70347A10073
:10570000630CA70741476385E7022C005285EFA091
:105710000FCE09CD34001546D9455285EFD09FD51F
:1057200011C5324597B0FE1FE78000A08147F9A060
:1057300083D7A4004146130524002300F40083D737
:10574000A400A183A300F400CC4097B0FE1FE78023
:1057500020AD4904835781008507C207C183231404
:10576000F10063F9270983D7A400638567098509D8
:10577000C20993D90901A1B7E39977F983D7A400A6
:105780000946130524002300F40083D7A400A18355
:10579000A300F400CC4097B0FE1FE78060A811047E
:1057A00055BF22C60359610003C7A4001305240096
:1057B0006382770333599903230571012300E400C1
:1057C00083D7A4004146A183A300F400CC40137901
:1057D000F90FA5BF230581012300E40083D7A400AE
:1057E000135929001379F90FA183A300F400094686
:1057F000CC4055B78357810089FBA947F2506254CA
:10580000D2544259B259225A925A025BF24B624C1C
:10581000D24C424D3E85216182808547C5B7C54740
:10582000F1BFB727002003C76797854763F3E706F3
:10583000011122CC26CA4AC806CE2A843289AE84F7
:10584000EFF08FDA01C9034725009307E00F5D45AC
:105850006308F700631C0900A6852285EFA02FF5D9
:10586000F2406244D24442490561828003D504007B
:105870009305E10023170100EFF0FF820355E100DB
:10588000EFF04FC5AA8505462285EF30800E69D519
:10589000C1BF5945828013F7050201C7B2856FF079
:1058A000CFC4411126C24AC006C622C413F98500DE
:1058B000AA8463170900139785016187635D070256
:1058C00032853684EFF00FC1AA85054663130900BF
:1058D00001462685EF30E00901E90145B240224446
:1058E000924402494101828083479400E5DB83476B
:1058F0008400E5F7E5B793F72500E5F30D45F9BF1B
:105900007971AE8622D42A8403D506009305E1017D
:1059100006D636C6EFF02FF909CD83458500B2468D
:105920000356E1012285EFF01FF7B2502254456182
:1059300082800545DDBF13F7050201C7B2856FF010
:10594000CFBA411122C426C206C693F485002A8428
:1059500091E4139785016187635007023285EFF068
:105960006FB7AA85054691E0014622852244B240E0
:10597000924441016F20F07F93F72500014591E3A8
:105980000D45B24022449244410182807971AE8635
:1059900022D42A8403D506009305E10136C606D633
:1059A000EFF06FF0B24601CD834585000356E1016B
:1059B0002285EFF05FF8B2502254456182800545A0
:1059C000DDBF797126D2AA840355A500C16722D410
:1059D0004AD04ECE06D623170100FD173284B68971
:1059E0000149630DF500050583C60400D04042055A
:1059F0001307E1004181EFF05FB22A8983C60400FA
:105A0000D04037D502008945130585EAEF905F8DB8
:105A10001DC503D4A4002285EFF06FAA09C57D142B
:105A20002A94420441806384090023908900B25083
:105A300022544A8592540259F2494561828083C6B4
:105A40000400D04037D5020089451305C5EAEF9020
:105A50003F8961F183C60400D04037D502008945F3
:105A60001305C5E8EF90DF8719C9E30609FA8357E4
:105A7000E100E39287FA0354A9007D145DB703D4D3
:105A8000A40055B7397122DC26DA4AD84ED652D452
:105A900056D25AD062CC06DE5ECEBE8983C7850060
:105AA0002A8AAE84C18B328C36843A89C28A468B6C
:105AB0009DE783CB04008947638BFB046285EFF08D
:105AC0002F8C1DC183280500638008025A88D68761
:105AD0004E87CA862286A6855285829839A032854D
:105AE000EFF0EF8BAA8711ED3945F2506254D25492
:105AF0004259B259225A925A025BF24B624C2161CE
:105B000082802946A6855285829745D5F9BFD8401F
:105B10008347170003470700A207D98FC2070D6705
:105B2000C187930607906384D72263CEF606930657
:105B30002780638ED70C63C1F60213070780E3CF7B
:105B4000E7F62D45E39309FADC4403C60700CC438E
:105B50002310C900228569A213073780E390E7F676
:105B60002D45E39409F885472310F900DC4481456D
:105B700083C707002300F40003D5A40005054205F0
:105B80004181EFF04FD28357090063170512910747
:105B90002310F900114681451305140097A0FE1F3C
:105BA000E780206F29A2930627906383D71863CEDE
:105BB000D71293063790638CD71813074790E39F4B
:105BC000E7EE2D45E39309F2DC441D472310E9007D
:105BD00003C707002300E40003C71700A300E40085
:105BE00003D727002301E40003D727002183A30163
:105BF000E40003C747002302E40003D76700A302C1
:105C0000E40083D76700A1832303F4004DA02D4552
:105C1000E39D09ECDC446C0083C9170003C707004F
:105C2000A209B3E9E90011472310E90083C707007F
:105C30004E852300F400DC4483C71700A300F40062
:105C4000EFF06FC6AA8435C50356C100C16593063F
:105C5000E100FD158329C500EFF0BFD619ED83C61D
:105C60000400D04037D5020089451305C5EAEF90FE
:105C70002FE701E5FD572317F10003C70900894706
:105C80006310F70283A5490009461305440097A055
:105C9000FE1FE780E0588357090089072310F900A9
:105CA0008357E1002301F400A183A301F40001451F
:105CB0002DBD23173101EDB7034705008907BA97BA
:105CC0002310F9008357A500A300F4008357A50013
:105CD000A1832301F400034605004C411305340061
:105CE00097A0FE1FE780C053D9B7C84497A0FE1FF6
:105CF000E780405D93170501C1832A871D45E3E6D0
:105D000037DF6399F90023100900CC4403560900DA
:105D1000CE9589B54207B3863A01418363C7E60051
:105D2000B38737412310F900CDB723105901F1BFD4
:105D30002D45E39C09DACC445285EFE0BFC3231024
:105D400079012300A4002181A300A4008DB72D4573
:105D5000E39D09D8DC442310790183C707002300A1
:105D6000F400DC4483C71700A300F40089B71D7159
:105D7000CAC82A8903552500A2CCCEC6D2C4D6C231
:105D8000DAC05EDE62DC66DA6ED686CEA6CA6AD875
:105D9000AE8AEF908FE9130CF5FF93170C01B72B28
:105DA0000020C1832A8A814913848B9D3EC6372BEC
:105DB0000020B72C0020C16D8357C90063F6F9009D
:105DC0008357040063CC87010355290093858B9D7D
:105DD000EFA08F882A8D15CD594D25A883278900DE
:105DE000139719009305E101BA9783C4170083C77D
:105DF0000700A204DD8C2685EFF0EFAAAA8515E93D
:105E000023909A004840054D09C597A0FE1FE780E2
:105E1000A031F64066446A85D6444649B649264ACA
:105E2000964A064BF25B625CD25C425DB25D2561D4
:105E3000828032488348490083A68C950356E1014D
:105E40000355290081471307EB94EFF0BFC32A8D58
:105E500013888C9509C523909A00484075B75C401B
:105E600085E703552900514781461386FDFFBD454F
:105E7000EFD02FFBB727002048C01388879509E58E
:105E800023909A00454D71B7835704000357EB9454
:105E90009304EB943E976347470113C7F7FF52976C
:105EA0002390E400484003D60400832508003E9573
:105EB000850997A0FE1FE780A0368357040003D70B
:105EC0000400C20993D90901BA972310F400EDB573
:105ED000397122DC2A840355250006DE26DA4AD8E9
:105EE0004ED652D45AD05ECE62CC66CA2E8B56D2D3
:105EF0006AC8EF908FD32A8A8346C4008355A400D2
:105F00000355840078001306D400130CBAFF651AF9
:105F1000EFF0AFE0420A37290020AA898144135AE2
:105F20000A01B72B0020B72C00201309899D638636
:105F3000090463D48405938A8C958348440083A61E
:105F40000A000356C1000355240052888147138775
:105F5000EB94CE85138DEB94EFF0DFB215C5814A3B
:105F60000356C1008355A4004E859306E100EFF06F
:105F70005FA5AA89639D0A065DF9E5E08357840061
:105F800029452310FB0089A083570D000356040107
:105F9000E317F6FC83A50A00484897A0FE1FE78098
:105FA000603555DD83274900A1E303552400416690
:105FB000454781467D169D45EFD0AFE605E5835701
:105FC000840045452310FB00F2506254D2544259DC
:105FD000B259225A925A025BF24B624CD24C424D59
:105FE000216182802322A90083DAA90095BF83273B
:105FF0004900A69723805701938714001397070140
:1060000083274900418393DA8A00BA972380570196
:1060100013872400832649009387340042079104A4
:106020004183C207C204C183C180369711CD835614
:10603000E1002300D70003274900BA970357E10086
:1060400021832380E700E5B5FD562300D700032711
:106050004900BA972380D7000DB703552400B72510
:1060600000208980239C959C9385859DEF90DFC4BB
:1060700021DD594591BF411122C406C693F70501A0
:106080002A84328585C3EFE0FFC4AA8505462285B0
:10609000EF20300E95476305F500BD47631DF502FF
:1060A000214515A893F7450099CBEFE0BFC20546FF
:1060B000AA8522852244B24041016F20900B93F7BC
:1060C000050489C7EFE01FC10146DDB713F51500D0
:1060D000133515000605B2402244410182807971D2
:1060E0004AD04ECE52CC06D622D426D22A8AAE89A7
:1060F000014983D749006364F9000145A1A083A742
:106100000900131419009304140033879700034700
:106110000700A29703C5070022079305E100598DE8
:10612000EFE07FF805E983A7090005453E940347A2
:1061300004002380E70083A70900BE9403C704007E
:10614000A380E700B250225492540259F249624AA5
:1061500045618280834585000356E1005285EFF05A
:106160009FF105C183A709003E94034704002380E3
:10617000E70083A70900BE9403C70400A380E700DB
:10618000D1B70509420913590901A5B7011122CC5C
:106190002A8403D505009305E10006CEEFE0BFF0A9
:1061A00001CD834585000356E1002285EFF0BFEC69
:1061B000F2406244056182800545DDBF1D71CAC899
:1061C0002A890355250086CEA2CCA6CAD2C4D6C23F
:1061D000DAC05EDE62DC66DA2E8ACEC66AD86ED699
:1061E000EF90AFA42AC68346C9008355A900035582
:1061F000890078081306D900EFF02FB2B247B72410
:106200000020416B938AA7FFC20AAA8B014493DA4C
:106210000A01372C0020B72C00209384849D7D1B1D
:1062200063860B180356C10183C58B0003552900F3
:10623000EFF07FE4AA8D631605168348490083A614
:106240008C950356C10103552900568881471307D1
:10625000EC94DE85EFF01F83AA8D9309EC94138DE7
:106260008C956310051429C003D7090083D7240037
:1062700011076397E7003247A2976D1763CAE706D5
:10628000B72500209387859D03D727000355290054
:106290009385859D3354E40223908700EF905FBF80
:1062A000AA8D15C1D94D05A003552900494781463E
:1062B0005A86C545EFD0EFB6C8C015E583D7AB0009
:1062C000C54D2310FA00F64066446E85D644464913
:1062D000B649264A964A064BF25B625CD25C425D46
:1062E000B25D2561828083D7090091072391F40074
:1062F000DC4003D7AB009306E101A2972380E700BF
:106300009307140013970701DC4041835E85BA9719
:1063100003D7AB0021832380E7000356C1018355D7
:10632000A900EFF00FEAD440130724000356E1015F
:106330004207418336972300C700D84093073400B3
:10634000C207C183BA970357E101AA8B11042183C5
:106350002380E700C8404204418003D6090083251A
:106360000D00229563950B0297A0FE1FE78040EB7E
:1063700083D709003E9442044180E31304F083571D
:1063800089002310FA00E3900DF4A94D2DBF97A0CA
:10639000FE1FE780E0E883D709003E944204418075
:1063A00041B583D7AB002310FA00C1BF814DF1B7CF
:1063B0005D71A6C2CAC0AA84035985000355250091
:1063C000A2C44EDE52DC5AD85ED662D466D286C6ED
:1063D00056DA6AD06ECE2E8BEF902F85930BD5FFB9
:1063E0007115131A0501B72900200144135A0A0137
:1063F000372C0020B72C00209389899D6359741590
:1064000083C6C40083D5A4001307E1001386D4001B
:106410004A85EFF08F902A8D630B05120359A50072
:10642000834585000356E10003D52400EFF0BFC487
:106430006314051283C8440083A68C950356E100BB
:1064400003D52400528881471307EC94EA85EFF0C6
:106450006FE3930DEC9413888C95631F050E1DC894
:1064600083D70D0003D729008907630CF706B725EA
:1064700000201387859D8357270003D5240093852B
:10648000859D3354F40223108700EF90BF8C15C50F
:10649000594525A003D5240041664D4781467D1608
:1064A000A545EFD00F98B727002023A2A900138895
:1064B00087951DE123102B014545B640264496449F
:1064C0000649F259625AD25A425BB25B225C925C34
:1064D000025DF24D6161828083D70D0089072391AF
:1064E000F90083D70D00A29763D3770783A74900EC
:1064F0000357AD00930A2400A2972380E700050408
:106500009317040103A44900C183C20A3E94835730
:10651000AD008325080093DA0A01A1832300F4006B
:1065200003A5490003D60D00569597A0FE1FE780EE
:1065300020CF03D40D00C167FD175694420441805B
:10654000E30EF9EA050942091359090145BD294538
:1065500019FC23102B0195B76DDC11BF8357050083
:1065600081E789473E858280411126C2444122C489
:1065700006C64AC083C60400D0402A8437D502002C
:106580008945130585EAEF80BFD519C983472400E3
:106590002547E51793F7F70F6377F702E14729A837
:1065A00083C60400D04037D5020089451305C5EAEB
:1065B000EF801FD361FD8947B240224492440249D3
:1065C0003E8541018280372900208356098E854708
:1065D0001309098EF5D2035704003697C166E3CD3F
:1065E000E6FC916593852570314597A0FE1FE780F5
:1065F00060A5AA84CD4769D13146814597A0FE1F89
:10660000E78020C9835704008355090001460147EC
:10661000B386E500C206C182636BF702AE97C2077C
:10662000C18319C22310F90023A004002146A285CA
:106630001385440097A0FE1FE78080BEB727002087
:106640009387C795984311EF84C38147B5B75040EE
:106650001315470005072A962315D60005464DBF9A
:106660003E871C43F5FF04C381BF011106CE22CC37
:1066700026CA4AC809E98944F2406244268542494B
:10668000D244056182802AC62A84280036892314D0
:10669000B1002305C100EFF07FECAA8471FDE30D8A
:1066A00009FC8357A400E1DB916593855570314562
:1066B00097A0FE1FE780009915C58357A4002320EB
:1066C0000500232425012312F500B7270020938716
:1066D0008796984301E788C345B73E871C43F5FF7B
:1066E00008C359BFCD4449BFB727002093870795FA
:1066F00003C7070015E305472380E700058909CD97
:10670000B7260020372500209386068B4146914509
:10671000130505876FF07FF501458280B7270020BC
:10672000A38AA78C8280C167FD176315F5002E85AB
:106730006FE0CF91411106C6EFE04F8B11C5FD57B9
:106740002310F50023010500B240410182800111B0
:106750004AC806CE22CC26CA85472A896393F50407
:106760004A85EFE0CFBE39E9C16437D60200938590
:10677000F4FF1307E1008946130606E90545EFE03B
:10678000DFD92A84FD140DC44C444A85EFF0BFF9CB
:106790000356E10022858146A685EFF08FA22A8468
:1067A000DDB789476396F5008545EF20C03C4DD99C
:1067B000F2406244D244424905618280EFE02FB446
:1067C00065B7011126CAB7240020938404C222CCE5
:1067D00003C594003724002013040496B727002033
:1067E0003727002006CE4AC84EC62320040023A225
:1067F0000796232A079449C9138947969307200CC3
:106800003305F50291659385157093094795190530
:106810004205418197A0FE1FE780C08203C6940015
:106820009307200C81453306F60208C0190697A08D
:10683000FE1FE78000A61C4003C794008145938695
:10684000870B7D5563ECE5069306800BB306D702F4
:106850000146FD550507B6972320F900BE86239013
:10686000B600A381B6002381B60023820600050688
:106870009906E366E6FEF9562390D700994633075A
:10688000D702BA9723A0F900375501001305E5EAAE
:10689000EFC0FFD2375501001305E507EF805FAB6E
:1068A00037550100130565E1EF200024F2406244F2
:1068B000D2444249B2490145056182802394A6F43D
:1068C0001386C6F423100600232406003106E31BBA
:1068D000D6FE85059386860BB5B7411106C622C440
:1068E0002A84EFC00FB7EFD0BFF8B7270020238A64
:1068F000878CB727002003A54795EFD03FF5B72732
:1069000000202381878E2244B240376501001305A1
:10691000E57441016F20401D93970501C18763D342
:106920000734B727002003C5478D797122D45AC890
:1069300006D626D24AD04ECE52CC56CA2E8BEF70F7
:10694000AFAD2A8429C9034705009307000B6311E3
:10695000F704B7240020854793848495A304F100AD
:106960009C4023150100A9E7EF00007F9165938506
:1069700035709790FE1FE780E06C88C015E983476B
:10698000910099C78345440013058400EFD0EFA51B
:106990002285EF704F9CB250225421653345AB00E5
:1069A00092540259F249624AD24A424B456182806E
:1069B000372A00206146814513058A9D97A0FE1F56
:1069C000E780208D03494400894793048A9DD2893A
:1069D000930A8A9D6314F906EF0000782390A400BF
:1069E0000355240093058A9DEF90EF9B03572400E5
:1069F00083D704008356840011ED63E4F60023146A
:106A0000F400835584003A85EFC01FBC2285EFC097
:106A10007F8EB5B763E4F6002314F4008357840037
:106A2000D9459386899D0D463A852390FA00EFC09B
:106A30007FA48D4561DD1385899DD1A09947631A97
:106A4000F9029305A1002285EFF08FC8AA845DDDCD
:106A5000D9476396F40E0509035524001379F90FFD
:106A6000D9459386899D4A86EFC0DFA0CA8559DD46
:106A7000D9B7A1476318F9009305A1002285EFF06B
:106A80003F93E9B7A947631FF906035584006C00DB
:106A9000EFE06FE12A89630D051403552400416678
:106AA0009306E10055477D16AD45EFC09FB7C8C0BE
:106AB000AA8649C1834844000358E1000356C10037
:106AC00003552400814713078A9DCA85EFE09FFB89
:106AD000AA84631E050E0355240093058A9DEF903A
:106AE0004FAD0DD50355240093068A9D2D46D945FB
:106AF000EFC05F98E30C05F0AD4513058A9DEFD01C
:106B0000CF8E29B7B147631BF90E035584006C0083
:106B1000EFE06FD9AA8469CD03552400416693063E
:106B2000E10059477D16B545EFC0BFAF23A2AA00CB
:106B3000AA8629E983578400C5442315F100034739
:106B40001400D147E304F7EC8347440003552400C5
:106B50009385899D2380FA008357A10023829A00A0
:106B60002391FA00EF80FFA3E30205EA0355240016
:106B70009386899D0546D945EFC0DF8FE30805E878
:106B8000854555BD834844000358E1008357A40060
:106B90000356C10003552400A68513078A9DEFE024
:106BA0007FEEAA840DE50355240093058A9DEF909E
:106BB0000FA6E30D05E403552400D94593068A9DED
:106BC0003546EFC03F8BB545E30205E4ADB5D94787
:106BD0006393F400814403A54A009790FE1FE78069
:106BE000A054E38504E2835784002315F10081BF9C
:106BF0008357840085442315F10091B7B947631882
:106C0000F9009305A1002285EFF06F9681B5C14789
:106C10006318F9009305A1002285EFF02FDA3DB546
:106C2000C947631AF900130691009305A100228554
:106C3000EFE06FF921BDD947631DF9009305A1006D
:106C40002285EFE06FE7AA84E31405E0A3040100C6
:106C500075BBE147E31CF9DA9305A1002285EFE05B
:106C6000CFD3EDB301458280EDC2011152C42E8A0B
:106C7000854522CC4EC656C206CE26CA4AC8AA8A26
:106C8000B6893284EF10306FD1471DC5B727002079
:106C90003727002083C7479783465797814419E0D9
:106CA000B684BE86372700200327C79693974400F3
:106CB000BA9763EDD400D547F2406244D2444249CA
:106CC000B249224A924A3E85056182803E89C107C7
:106CD00003D727FF09C7850493F4F40FD9BF25C054
:106CE0009565938525C0130500029790FE1FE780E8
:106CF00060352326A90061D11306000281459384E3
:106D000004049790FE1FE780C058231199002300C8
:106D10000900231359011DC437270020834794001D
:106D2000032647B82304F900118C8327C900118476
:106D30001180238E870023A029018147B5BF232618
:106D40000900F1B723044901FDB785473E858280DC
:106D5000B727002083C54797B727002003A7C7960A
:106D600081476395F500814636858280035627006A
:106D7000BA8619C2E30AA6FE850793F7F70F410703
:106D8000CDB7B727002003C64797B727002003A732
:106D9000C79681476315F600814636858280835504
:106DA0002700BA8689C583454700E388A5FE850785
:106DB00093F7F70F4107F9BFB727002083C57797EF
:106DC000B727002003A747B881476395F5008146A0
:106DD0003685828003560700BA8619C2E30AA6FEEA
:106DE000850793F7F70F4107CDB7B727002003C8F2
:106DF0005797B727002083A7C79601476315E80078
:106E000081463685828003D62700BE8619CA03D6FE
:106E100067006318A600D04709C603562600E302A0
:106E2000B6FE05071377F70FC107C9BF411122C48A
:106E3000404526C206C6AA8415C0484409C5979095
:106E4000FE1FE780602E484809C59790FE1FE78027
:106E5000A02D22859790FE1FE780002D26854146B4
:106E600081459790FE1FE780C042B2402244FD5703
:106E7000A384F400924441018280011122CC2A842F
:106E80000355250006CE2EC6EF10F0183246228597
:106E90008145EF00B07222856244F24005616FF0D7
:106EA000FFF80DC503572500411122C406C62A84E8
:106EB00011CBDD45EF00707422852244B2404101C0
:106EC0006FF0DFF6B240224441018280828041119E
:106ED00026C2B1469304C5FFB386D402B72700206B
:106EE000138747B906C622C436978356A70063980E
:106EF000B60248430DC5138447B99307F00F6306E4
:106F0000F60083470500639CC7009790FE1FE7804B
:106F1000A021B147B387F402A29723A20700B24091
:106F20002244924441018280411122C42E8426C20F
:106F30004946AA848145228506C69790FE1FE780B0
:106F40004035A5C083C7C40113974700B727002069
:106F500083A747B8BA9703D707002310E40003D7E5
:106F6000270083D767002311E40037270020035749
:106F700027972312E40003D704002313E40003D768
:106F800024002314E40003D744002315E40003D7AE
:106F900064002316E40003D784002318F4002317A9
:106FA000E400B2402244924441018280B72700208D
:106FB00083C54797B727002003A847B8B727002005
:106FC00003A6C796014781476394E5003E8582800A
:106FD0008346060081CE544691CA83C6C6019206F6
:106FE000C2966315D500850793F7F70F050713774A
:106FF000F70F4106D1BF130600643386C50293061E
:107000009500AA8537750100130525EA6F708FB7C3
:10701000411122C406C62A8403459500EF700FD1A2
:10702000FD57A304F400B2402244410182800111C3
:1070300022CC4AC84EC652C456C25AC006CE26CA30
:107040002A89AE890144372A0020B72A00201D4B27
:1070500083475A976365F40463990902B7290020AE
:10706000372A0020930AF00F83C749976367F40615
:107070001144A1442285050442041306F00FCA8579
:107080004180EFF0DFE4E31794FEF2406244D24423
:107090004249B249224A924A024B0561828083A743
:1070A000CA9693144400BE9483C704009DC383D73B
:1070B0006400639027036396690103D52400EF10F1
:1070C000807526854E868145EF00504F2685EFF06E
:1070D000FFD505041374F40FA5BF8327CA96931434
:1070E0004400BE9483C704009DC383C7940063809B
:1070F000570383D76400639C27012685EFF05FF177
:107100002685D145EF00704F2685EFF03FD205046C
:107110001374F40F91BF41677917630BE5024111B6
:1071200022C406C685472A846399F5002285224435
:10713000B240814541016FF09FEF89476396F500AA
:107140008545EF1050237DD1B24022444101828019
:1071500082809D456FF0BFEDB727002003D52797AC
:107160008280B727002003C70797011106CE231797
:10717000A1002316B10085476318F700700093053E
:10718000E1000545EF50B025F24005618280A94736
:10719000631CF60483C7150003C70500A207D98F37
:1071A0002310F50083C7350003C72500A207D98F38
:1071B0002311F50083C7550003C74500A207D98FE7
:1071C0002312F50083C7750003C76500A207D98F96
:1071D0002313F50083C7950003C78500A207D98F45
:1071E0002314F50001458280054582809147631490
:1071F000F60283C7150003C70500A207D98F231025
:10720000F50083C7350003C72500A207D98F2311D6
:10721000F50001458280054582809387C5FF9396DE
:107220000701C1820D476360D7023147B387E70288
:1072300037270020130747B9BA972381A700239067
:10724000B700014582800945828093064020372798
:107250000020AA8763F4A60093074020F1172319A2
:10726000F796B7270020238BB796B7270020238CEB
:10727000B79682801905956542054111938535C001
:10728000418106C69790FE1FE780C0DB11C5B24062
:10729000E95541016F60FF84B24041018280B72708
:1072A0000020238B0796B727002079710547238894
:1072B0000796B72700202388E7B84ECEB7270020CF
:1072C000B729002022D426D24AD037240020B72460
:1072D0000020A38C079637290020B7270020938928
:1072E000799706D652CC2AC6230A0496A38A049616
:1072F000239907962326099623800900EF10405909
:107300003245B7270020130600032384A7B837258A
:107310000020130545B981459790FE1FE78060F76F
:10732000372A002003454ABC13044497938454979A
:107330001309C99615CD9565938545C0120597909B
:10734000FE1FE78020D0372700202322A7B80DC1D9
:1073500003464ABC93074ABC83C717002380C90071
:10736000814512062380F4009790FE1FE78060F2AB
:10737000B727002003C587C283C70400956593859E
:1073800055C03E951375F50F2300A4001205979084
:10739000FE1FE78020CB2320A90049C50346040037
:1073A000814512069790FE1FE780A0EE0327090093
:1073B00083460400814725077D56639EF604EF103F
:1073C0000072B1473305F5029565938565C04205A6
:1073D00041819790FE1FE780E0C6B727002023A6D3
:1073E000A7B82A8401CDEF10806F31463306C5025D
:1073F000814522859790FE1FE780A0E92254B25074
:1074000092540259F249624A377501001305651119
:1074100045616F10606D85072300C70093F7F70F74
:10742000410761BF230004002380040049BF4111CC
:107430009397050126C206C622C44AC0C187AE84FE
:1074400063D1070A37290020034589B8EF60CFFCD4
:107450002A8429CD03470500930700096315F70423
:1074600003471500CD47631CF706B72600200348E5
:10747000250003C576A837270020834767971306A2
:1074800064008145814613076797AA886318D8026C
:1074900099C12300F7008347070091C7034589B8C6
:1074A0008545EF601FBA2285EF60EFEA2165258DE3
:1074B000B240224492440249410182808345060041
:1074C000AE9793F5F70F93F7F80F63F4A50093F7D2
:1074D000F50F850693F6F60F0906854545BF012D84
:1074E000D9B793F715000145E1D7EF00107009CD2A
:1074F000B727002083C7679781CBB727002003C534
:1075000087B88545EF60FFB313C5140055B78546AE
:107510002A8763FBC60483C7150003C60500A207BC
:10752000D18F2310F500639CD70083C7350083C635
:107530002500A207D58F2311F500014582808946D9
:1075400001456394D70283C7350083C62500A2078F
:10755000D58F2311F70083C7550083C64500A207C6
:10756000D58F2312F70082800545828091476314EE
:10757000F60283C7150003C70500A207D98F2310A1
:10758000F50083C7350003C72500A207D98F231153
:10759000F500014582800545828091476314F6021B
:1075A00083C7150003C70500A207D98F2310F50074
:1075B00083C7350003C72500A207D98F2311F50023
:1075C0000145828005458280A1476314F60483C784
:1075D000150003C70500A207D98F2310F50083C744
:1075E000350003C72500A207D98F2311F50083C7F3
:1075F000550003C74500A207D98F2312F50083C7A2
:10760000750003C76500A207D98F2313F500014554
:107610008280054582808947631CF60083C7150078
:1076200003C70500A207D98F2310F500014582800A
:10763000054582808357260079714ECE06D622D426
:1076400026D24AD01307F007AE896372F7020947C2
:107650003AC42316F100300093F5F50FEF10801AAD
:10766000B250225492540259F24945618280035724
:107670004600D9462A89328463F8E60083576600BB
:1076800063F4F6006379F70023140100300093F5EA
:10769000F90F4A85E1B70355060002C4EFF0CFF1B8
:1076A000AA8459C1EFF09F9083C784006369F500F5
:1076B0001146A246CE854A85EF10400A55B73400E0
:1076C00026869305F00F4A85EFF00FDA75F1A24791
:1076D00003578400DC472390E700035724002391DD
:1076E000E700035744002392E70003576400239305
:1076F000E70003D744002394E700DC4485CB93F4F0
:10770000F90F2286A6854A858297C167FD172A86CA
:10771000E311F5FA22459947F9452300F5002302C4
:107720009500EFF05F8D2DBF094661B7014651B757
:10773000A947631CF60483C7150003C70500A20709
:10774000D98F2310F50083C7350003C72500A20792
:10775000D98F2311F50083C7550003C74500A20741
:10776000D98F2312F50083C7750003C76500A207F0
:10777000D98F2313F50083C7950003C78500A2079F
:10778000D98F2314F500014582800545828083C787
:1077900005002300F50083C71500A300F50083C78B
:1077A000350003C72500A207D98F2311F500828079
:1077B0002322050003C7450089476304F7000545F8
:1077C000828083D665000D47E37BD7FE9C4501117F
:1077D00006CE22CC26CA4AC84EC683C4170003C6AA
:1077E0000700A204D18C138644006311D60403C49D
:1077F000370083C72700AE8922045D8C9307C4FF3E
:10780000C207C1832A89636FF70003A5890023118A
:10781000990023108900F155EF60AFAC2322A90035
:10782000014531A02285EFF0AFD265F10545F24068
:107830006244D2444249B24905618280397122DCF6
:107840002E84834704004AD806DE26DA4ED619472E
:107850002A89B285639AE706034624002800EFF0E0
:10786000FFD0AA8415E903558100EFF06FCEAA89F5
:107870008345140015C9378701002E861307477307
:1078800034009D454A85EF00D0424E85094681452A
:1078900035234E85EFF08FD9F25062542685425938
:1078A000D254B2592161828089472310F100835755
:1078B00081000A862311F1008357A1002312F100F1
:1078C0004A85EF003074C9BF4947639DE7020356FC
:1078D00024002800EFF05FCFAA845DFD372500204B
:1078E000130545B98357C50099E3814475B703472C
:1078F0001400834604000345E5003C000146CA85A8
:10790000912659BF51476390E7020356240028008F
:10791000EFF0FF87AA8449F18345140030004A85BF
:10792000EFF05FD195BF59476393E70603562400F4
:107930002800EFF0BF8BAA8425F1835581004A858A
:10794000EFF0AFCA1DC958458356A1008357070001
:10795000B697C207C1832310F700C1DB5C47D1D7BC
:10796000B727002083C76797C9D3B727002003C56F
:1079700087B88545EF60EFEC05B789473EC0835770
:1079800081000A86834514002312F10015BF834548
:1079900014000A8623100100EF00D066B9B75D71AC
:1079A000A6C256DA86C6A2C4CAC04EDE52DCAA8A75
:1079B00003C51500AE8432C6EFF0AFBCB24501ED91
:1079C0008144B6402644268506499644F259625AB7
:1079D000D25A61618280230205002311050083C908
:1079E000040085472A84639AF90003C62400280806
:1079F000EFF0FFB1AA8405492DA09D476394F904D7
:107A0000034705008D47E31DF7FA03C62400280845
:107A10000549EFF09FB8AA8409E50546814522850E
:107A2000712E2285EFF0CFDE034584003C0801472C
:107A3000CE862686D6853924E30509F82285EFF01F
:107A4000EFBE41B7CD47639DF9000347050091475D
:107A5000E318F7F603C624002808EFF0DFBB59BF90
:107A6000D547E39FF9F4034A05008947E31AFAF47E
:107A700003C6240028080549EFF09FCBAA8455F1DE
:107A800083570102BDE3035781011306F0035C44F1
:107A9000930607FCC206C182636CD6000356A1019F
:107AA000D94663F7C6008356C101D94563EFD500B7
:107AB000035524002391E7000549EF00D0550356F4
:107AC0000102D2852285692CA9BF8355E10123914A
:107AD000E7002392C7002390B7002393D700854780
:107AE0002300F400014A0149D9BF014AC9BF797195
:107AF000AA8522D426D203542500AA84280806D6B3
:107B0000EFF01FCBF24599E535E985452285EFF089
:107B10004FE5C1A0835781011547639BE7060357D3
:107B2000A1018D4763FCE7046800EFF05FC60357CF
:107B3000E100DD4763FCE7008345D100B70717008C
:107B40008507100822853EC8EF00D04B8357E1001F
:107B50000357A10191076305F7002285EFF06FDF5E
:107B60008347C10072466C00858B1106228591CF38
:107B7000EFF0FFE201C52285EFF0AFDD884451D57B
:107B80009780FE1FE780405A49B7EFF03FCBDDB743
:107B900011476389E7001387A7FF420741838546A2
:107BA00063EEE6023147F117B387E702372700207B
:107BB000130747B9BA9703D7070069D303C527004E
:107BC0003008A2850D205DF9035781019147E31E1E
:107BD000F7F2B25022549254456182802C082285DB
:107BE000812E49FDFDB701114AC82A89314526CAAF
:107BF00006CE22CC2EC6B284EF501FFB31C1B24557
:107C00009307000A2310F5002311B5002A842146AA
:107C100011058DC0A6859780FE1FE7806060A28554
:107C20004A85EF606F870145F2406244D244424981
:107C30000561828081459780FE1FE7808065C5B71A
:107C40000545DDB7797126D2AA841305000206D650
:107C500022D42ECE32CC36CA3AC83EC6EF50DFF41C
:107C600031C96246F2454247D246B2472A841305DB
:107C700020FA2300A400A300C4002311B4002302AF
:107C8000E400A302D40013058400614691CFBE85B1
:107C90009780FE1FE780C058A2852254B2502685E7
:107CA000925445616F505FFF81459780FE1FE780CA
:107CB000405EDDB7B25022549254456182805845EF
:107CC000797122D406D62A84AE8649C38357270009
:107CD000231DF10093072006639FF504B7270020BA
:107CE00003D62797835767006373F600B28713F6AE
:107CF000F70F83552701834707018D8F93F7F70F00
:107D000081E5890793F7F70FB297FD17B3C7C7024D
:107D1000231EF1008357240083556400034584002B
:107D2000231CF10001473C080146EFF0BFF1B250BF
:107D30002254456182800347C701B727002083A7EB
:107D400047B81207BA9783D76700D9B72EC6194626
:107D5000814528089780FE1FE780A053B2465DBF8B
:107D6000797122D406D626D22A848DC18147014753
:107D7000930600062E868355640003458400EFF0C9
:107D80007FECB2502254925445618280B284280024
:107D900059469780FE1FE780C04F2314910089E861
:107DA0008357240048446C002315F100EFF0CF976F
:107DB0003C00014793060006014675BF797106D65F
:107DC000814799ED8357250058452316C100231498
:107DD000F1003C0011C7835727002315F1003C0038
:107DE0002E868355650003458500014793060006EE
:107DF000EFF05FE5B25045618280411122C406C6B2
:107E00008347050011472A846395E7022E86835530
:107E100065000345850081470147CD46EFF09FE2AD
:107E20004946835564002244B240154541016FF034
:107E30000F8A13F7B70F89466317D7000146EFF093
:107E40003FF25146F9BF0D476398E7002244B24024
:107E5000014641016FF09FF6B24022444101828009
:107E600003D70500B146B727002071173307D702A3
:107E7000938747B9BA97D84319EBD8412395A70000
:107E80000145D8C303D725002394E70082805945D4
:107E90008280797122D4404526D24AD006D6AA845F
:107EA0002E8925C0484419C59780FE1FE780C0274A
:107EB000232604008357040083D5640003C584008F
:107EC0002315F1008357240001479306400623162B
:107ED000F100835784004A862317F1001C483EC8EE
:107EE00083D724002314F1003C00EFF0BFD5A30E8C
:107EF000240123280400B2502254925402594561AF
:107F000082802800314681459780FE1FE7806038D7
:107F100083D7240083D5640003C584002314F100B3
:107F200001473C00930640064A86EFF0BFD1E1B717
:107F3000797152CC2A8A03D5050026D206D622D4DE
:107F40004AD04ECE56CAAE84EFE09FE019E1854795
:107F5000BDA84045AA8965DC83576500E39947FFC2
:107F600083578400638707128346C401B72A002021
:107F700003A74AB89206FD173697C2070357670052
:107F8000C1832314F4006316F70093053006EFF065
:107F90001FD35C48A5EFC84003491500834705007F
:107FA00022093369F90083D7240013072900631AD3
:107FB000F702F955EF50FFB2C8C02391240103C561
:107FC00089002686D285EFF01FC2814721E1B25099
:107FD000225492540259F249624AD24A3E8545617E
:107FE00082809565938515C04A859780FE1FE7803E
:107FF000600548C8C840231C2401F955EF507FAEE6
:1080000083D72400C8C0F9172391F400484859C504
:1080100003D624008356A401835784013308D60075
:1080200063C007090347C40183A74AB895451207EF
:10803000BA9783D7270063CF0705CC403695978042
:10804000FE1FE780E01D0357A40183D72400BA97E1
:10805000C20703578401C183231DF400E399E7EEAF
:1080600003D7290003C5890030002314E1005848D4
:10807000D2852315F1003AC6EFF0FFB611C5484886
:108080009780FE1FE780400A232A0400232C040067
:108090007DBD99454E85EFE05FDE55BDA545DDBF51
:1080A0009145CDBF03D725007DC3B727002083D6D8
:1080B0002797ED4763EEE60C011122CC2E8426CAE9
:1080C000AA844840914506CEEF50BFA183572400B3
:1080D000AA862300F50083572400A183A300F5009E
:1080E000835704002301F50083570400A183A301F3
:1080F000F50003562400C167F917110642064182B4
:108100006396F4042AC4314532C6EF50FFA9AA850C
:10811000CD471DC5930700F92300F5003246F957F6
:10812000A2462311F50089472302F500B727002056
:108130002313C50014C503C587B8EF50FFB58147A9
:10814000F2406244D2443E850561828081452685A5
:10815000EF401035AA8711E9B726002003C76697BC
:1081600065D37D17238BE696E1BF09476304E502DB
:108170001D476303E50249476302E5027D47E311BA
:10818000E5FCB726002003C766978147D1BFED47BE
:108190003E858280D1476DB791475DB789474DB71E
:1081A00001114AC831471309C5FF3307E902B72750
:1081B000002026CA938447B906CE22CCBA94D84070
:1081C00029CB138447B9B727002083C66797854713
:1081D00095CA2314A10083D7840003D5A4002C00E2
:1081E0003AC62315F100EFF0FFEB11C5C8409780A8
:1081F000FE1FE78060F3B147B307F902A29723A2FD
:1082000007008547F2406244D24442493E850561F9
:1082100082808147C5BF797126D244453727002027
:108220004AD083D764000359279752CC06D622D46C
:108230004ECE56CA2A8A63F327013E8903D724010A
:1082400042091359090183D7040141CB998F4A840C
:1082500063D5270113940701418089452285EFF0FA
:108260006F81AA89CD4A25C183D724002AC6231548
:1082700081002314F10083D7240185E383D704010F
:10828000930925002300F50083D70401A183A300EF
:10829000F5006376240503D4040183D72401CC447C
:1082A00022864E85BE959780FE1FE78060F70355B6
:1082B0006A002C00EFF01FDFAA8A15C54E85978053
:1082C000FE1FE78060E6B250225456859254025950
:1082D000F249624AD24A4561828089078DBF79148A
:1082E000420441805DBF03D7240183D704003A9440
:1082F000FD17C207420403D70401C18341802390C4
:10830000F400239984006377E400D5FFFD57A38E22
:10831000F40055BF81455285EFF0BFB76DB7797155
:108320004AD03729002052CC034A999722D456CA02
:108330005AC85EC662C406D626D24ECE5284B72A2A
:108340000020054B930BF00F372C002083A7CA9613
:1083500093144400BE9483C90400639D6907DC4400
:10836000B5CBD84725CB03D7070029CBB7270020AB
:1083700083C7679799CF2685EFF0FFE9AA8515E9AE
:10838000B727002083C7579705046351F402A30C55
:108390008996B25022544E8592540259F249624A4B
:1083A000D24A424BB24B224C45618280A30C0996C3
:1083B000CDB72685EFF0FFAD8149E1BF83C7D70177
:1083C000639A7701930520062685EFF05F8FDC44E2
:1083D000A38E070083475C9705041374F40F63634F
:1083E000F4000144E31444F7C1BF4111154506C62A
:1083F000EFF01FDB09C50545B240410182801945F8
:10840000EFF01FDA6DF91145EFF09FD96DF51D45BD
:10841000EFF01FD96DF1B727002083C75797E9DF29
:10842000B24041016FF0BFEF83D705000D47F11750
:10843000C207C1836365F706DC41B5C3411122C49D
:108440002E84854526C206C6AA84352739C92685C5
:108450008925C167F9176381F40219ED8357240058
:1084600081CF8356040019476393E6043727002021
:108470000357279763FDE702B727002083C7679755
:10848000A285268599C72244B240924441016FF0EB
:108490007FC12244B240924441016FF07F9C094564
:1084A00082805145B24022449244410182806D4510
:1084B000D5BF397126DA4ED6AA84AE895D45894585
:1084C0004AD806DE22DC328936C63AC4EFE09FDAAB
:1084D00035C522472A84014511C7B2461305440019
:1084E000B68502979357850023003401A300240129
:1084F000A301F4009547231CF100B727002083C790
:1085000067972301A4001105231DA10022CE2C088A
:10851000268595C3EFF01FB9AA8411C522859780DF
:10852000FE1FE78060C0F250625426854259D25443
:10853000B25921618280EFF0BF92F9BFCD44E5B717
:10854000797126D24AD052CC56CA06D6BA8A22D4DB
:108550004ECE19472E89B284368A639DE5060355AF
:1085600026000944EFE0CFFE2AC62DCD5C45835995
:10857000650083D727002390F400B247B726002078
:1085800015472380570103C606B92391E700130757
:1085900016001377F70F2388E6B82382C70001E798
:1085A00005472388E6B85147631AE9001547239128
:1085B000E400DC4703D784002394E7005287A686B3
:1085C000CA854E85EFF0FFEE2A84324515C4EFE0F0
:1085D000FF8509A842867400BE85AA89EFE0CFE82E
:1085E0002A8441DD2285B250225492540259F24924
:1085F000624AD24A45618280F945EFE0DF9FDDB7EC
:1086000083D705002300F50083D70500A183A300CD
:10861000F50083D725002301F50083D72500A1832A
:10862000A301F5001145828083D705002300F500E2
:1086300083D70500A183A300F50083D7250023017C
:10864000F50083D72500A183A301F50083D745005A
:108650002302F50083D74500A183A302F50083D749
:1086600065002303F50083D76500A183A303F5000C
:108670002145828083D705002300F50083D70500BC
:10868000A183A300F50083D725002301F50083D73C
:108690002500A183A301F50083D745002302F5003F
:1086A00083D74500A183A302F50083D76500230388
:1086B000F50083D76500A183A303F50083D7850068
:1086C0002304F50083D78500A183A304F500294581
:1086D000828003D705008546AA872300E50003D7DB
:1086E00005002183A300E50003D70500631DD70023
:1086F00003D725002301E50003D725002183A3012B
:10870000E5001145828009456315A70203D72500BE
:1087100019452381E70003D725002183A381E700C2
:1087200003D745002382E70003D745002183A382B6
:10873000E700828083D705002300F50083D705007A
:10874000A183A300F50083D725002301F50083D77B
:108750002500A183A301F50011458280797126D2FD
:108760004AD04ECEB2842A89AE8929468145480036
:1087700022D406D636849780FE1FE78080B1231668
:1087800091008DEC835724002312F100B7270020BD
:1087900083D727972314F1005C448DC383C6C70198
:1087A00037270020032747B8920683D787003697DC
:1087B000035727002315F1002313E1003787010039
:1087C0004A8513074767540013F6F90FD545EFF0B4
:1087D0005FCE2A8911C19DE085472300F400230262
:1087E0000400014681452285EFF08FD7B250225414
:1087F0004A8592540259F249456182802285EFE010
:10880000EFE2EDB737870100B2861307276D2E869A
:1088100085456FF01FCA01112317A100B78601001B
:108820004165700001489307F00F0D47938606607D
:1088300099457D1506CEEFF0BFD0F24005618280EC
:10884000B7860100B28701482E861147938686625B
:10885000C9456FF0FFCE011122CC3724002013044C
:10886000C4BC26CA4AC84EC606CE2A89AE8993041D
:1088700004031C4081C7CE854A8582971104E31A00
:1088800094FEF2406244D2444249B249056182807A
:1088900041113727002022C406C626C2130787A726
:1088A0008347C7030345D70337240020130404C2BA
:1088B000A304F400AA9793F7F70F2304F400A5CFBD
:1088C0001305C0033385A702A5658505B7240020DD
:1088D0009770FE1FE7800077034684009307C0036C
:1088E00081453306F60223A4A4BC9780FE1FE780CF
:1088F000409A83A784BC83468400014789077D563C
:108900006341D7022244B240924437250020130627
:10891000000381451305C5BC41011783FE1F670095
:1089200043972390C7002381070023A5070205076B
:108930009387C703F1B7B240224492444101828039
:10894000B727002003C687C2B727002003A787BC2C
:1089500081476315F600814636858280BA86130703
:10896000C703835567FCE389A5FE850793F7F70FD7
:10897000CDB7011122CC2EC632C406CE2A84EFF028
:108980003FFC2246B24511E9C167F9176303F400C1
:108990005145F24062440561828054558347450049
:1089A00095C213F7270141456314A700154575F2D9
:1089B000C18B3D45F9DF83C7A6010145E3FBB7FC49
:1089C0003145C1BFC18B0145E9F71545D9B779716B
:1089D00026D24AD0B7240020416922D44ECE52CCB0
:1089E00056CA5AC806D6AA890144938404C2372AB3
:1089F0000020930AC0037D19054B83C7840063647C
:108A0000F400014535A8B307540303278ABCBA977D
:108A100003D727006316270105041374F40FF1BF71
:108A200003C55700300093856700EF1031491946A0
:108A3000CE8528009780FE1FE780C08BE31E65FD72
:108A4000B250225492540259F249624AD24A424BDD
:108A500045618280B727002083C587C2C166B727DA
:108A6000002003A787BCFD1681476395F5000146EA
:108A700032858280035827003A866306D80003486F
:108A80000700E307A8FE850793F7F70F1307C7034F
:108A9000E9BF411106C6EFF0BFEA11C50355450114
:108AA000B240410182800145E5BFB727002083C65F
:108AB00087C2B727002003A787BC0145814711075C
:108AC0006393F60082800346070001C6050513750F
:108AD000F50F850793F7F70F1307C703D5B7B72728
:108AE000002003C587C28280372700209306C7BCB9
:108AF00081471307C7BC31468C4291E58A07BA9774
:108B000088C30145828085079106E397C7FE4D45DE
:108B10008280411106C622C4EFF09FE21DCD2A8457
:108B2000035525008545EFF01FD3485409C59770BC
:108B3000FE1FE780605F22851306C00381459770A2
:108B4000FE1FE7800075FD572311F4002302040087
:108B50000145B2402244410182800945DDBF4111F7
:108B600006C6EFF0FFDD11C50345C500B240410167
:108B700082800145E5BFC167F9176304F502411121
:108B800022C406C62E84EFF0BFDBAA87014591C739
:108B900003C54700698C33358000B240224441014F
:108BA000828005458280011106CE2EC6EFF05FD986
:108BB000854711C903574501B24585476305B7008D
:108BC000231AB5008147F2403E850561828031CD90
:108BD00001114AC84EC637290020C16922CC26CAD5
:108BE00052C456C206CE0144AA84130909C2372AC8
:108BF0000020930AC003FD1983478900634BF400EA
:108C0000F2406244D2444249B249224A924A056142
:108C100082803305540383278ABC3E958357250001
:108C20006383370182940504C1BF8280B727002087
:108C300003C687C2B727002083A787BCC16601454A
:108C400089070147FD1691456313E600828003D82A
:108C500007006309D80003C8A7006315B80005051D
:108C60001375F50F05071377F70F9387C703E9BF50
:108C7000B727002003C687C2B727002083A687BC7A
:108C80000147814791066310E602858393C7F7FF8A
:108C9000C207C18305456364E50285473395A70094
:108CA00042054181828083C5060081C583D5C60205
:108CB000CD8F05071377F70F9386C603E9B793F6B1
:108CC0001700E1FE050585831375F50FE9B7797186
:108CD00056CAAA8A2E8526D24AD04ECE52CC5AC81F
:108CE0005EC662C406D622D4AE84328B368CBA8B72
:108CF0003E8AC2894689EFF0BFC449E141657D15CE
:108D0000EFF01FC42A84554531CC1946DE85130582
:108D10006400A30284019770FE1FE78060508357B0
:108D2000010323119400230264012319F4008357E3
:108D300041032300540123260402231AF4002306CE
:108D400044012317340123182401EFF07FF2231884
:108D5000A402232A04022685232C04028145EFF075
:108D60009FAF0145B250225492540259F249624ACF
:108D7000D24A424BB24B224C456182804545DDB719
:108D8000B727002083C687C2B727002003A787BC68
:108D900081476395F60041657D1582803A86130709
:108DA000C703835547FF6395A500035526008280BE
:108DB000850793F7F70FF1BFB727002003C887C2D5
:108DC000B727002083A687BC416601477D169548DA
:108DD00011436314E8000145828083D7260036855D
:108DE0006380C704CC5A8DCD83C7350083C5250069
:108DF00089CD938597FD93F5F50FE37FB3FC9387BA
:108E0000D7FA93F7D70F89EF82809385F7FD93F513
:108E1000F50FE3F3B8FC9387D7FA93F7D70FCDDFBD
:108E200005071377F70F9386C60365B7B7270020AA
:108E300083C587C24166B727002003A787BC7D167C
:108E4000814725486394F5000145828083562700B9
:108E50003A85638CC600545B89CA83C63600938604
:108E6000E6FD93F6F60FE372D8FE850793F7F70F4A
:108E70001307C703C1BF011122CC2A84494506CE7E
:108E8000EF707FF215C12AC62285EFF07FAB09CDC6
:108E90006244B7270020324683550503F24003C5DC
:108EA00037C205616F50CFB8F240624405618280DD
:108EB00039714ED652D4AE892A8A93053005414580
:108EC00026DA4AD856D206DE22DC32C63689BA8A7B
:108ED0009770FE1FE7800017CD4431C92A8489446A
:108EE0006382090432468145231AC10041469770C6
:108EF000FE1FE780003A5686CE8522859770FE1FBA
:108F0000E78000322146630E0902CA85280897705F
:108F1000FE1FE780E030A28650082C085285EF3013
:108F2000904FAA8422859770FE1FE780E01FF250C1
:108F3000625426854259D254B259225A925A21611A
:108F40008280814528089770FE1FE7808034E1B752
:108F5000411122C4405926C206C6AA8429CC08540D
:108F600009C59770FE1FE780201C285809C5977017
:108F7000FE1FE780601B685809C59770FE1FE780D9
:108F8000A01A285C09C59770FE1FE780E019685C8D
:108F900009C59770FE1FE78020190325040809C53D
:108FA0009770FE1FE780401822859770FE1FE780AC
:108FB000A01723AA04022244B727002083D5040364
:108FC000B240924403C537C241016F502FCF4111C7
:108FD00026C206C622C4AE84EFF09F9621C54C5926
:108FE0002A84A9C183A8C50703A88507FC59B859D5
:108FF00083C6650003D6050083C525002685EF706E
:10900000BFE22285EFF0DFF4EFF05FE201CD224412
:10901000B7270020B240924403C537C285454101BD
:109020006F502F82B240224492444101828001114C
:1090300022CC06CE2A842EC6EFF09F905C5991CFA9
:1090400083D70700B245639A870085476397F50089
:109050006244F24005616FF0BFEFF2406244056187
:109060008280411106C622C426C2EFF0FFD421C57A
:109070004059AA8429C0834724008DCBB7270020FC
:1090800083A707C089C7DC4399C32285829703471A
:1090900034009307F0026310F702224403D5240042
:1090A000B2409244814541016FF07FF2B727002022
:1090B00083A7C7BFC1BFB24022449244410182800E
:1090C000411126C24AC006C622C4AA842E89EFF0E6
:1090D0003F8731C140595DCC83570400639C970A98
:1090E0008347340013071002639CE708834724007A
:1090F000D9C37C540327040883D7470105E713F736
:1091000017000DC3185403574700058B01CF930771
:109110002002A301F400B2402244924402490545D2
:109120004101828013F7270009CB185403574700E9
:10913000098B01C793074002E9BF918B89CB1C546F
:1091400083D74700918B81C793076002D9B7B727B0
:10915000002083A707C0E1D3DC43D5DF22858297B7
:10916000034734009307F0028145E316F7FA26859A
:10917000EFF0FFE54DB7B727002083A7C7BFE1BFDA
:109180001307A0026398E700630409001309200392
:10919000CA85F1BF631C09002685EFF06FFA19C577
:1091A0008347450093E707012302F500A6854A851A
:1091B000EF708FDC8DB7797126D29947231DB100EE
:1091C000AA842E858D4522D406D632C636C4231CE9
:1091D000F100EFE02F8A2ACE4D441DC13246A2464F
:1091E000AA85328582962A8419E52C082685EFF017
:1091F000AFA32A8411C572459770FE1FE780C0F2A5
:109200002685EFF05FC72285B25022549254456103
:1092100082804111B7B6010022C42E862E84938627
:1092200066C0894506C626C24AC02A89EFF0BFF843
:1092300083450400AA844A85EFF07FD9B2402244D6
:1092400026850249924441018280B727002083A7E6
:10925000C7BF95CB9C4385CB1D71A2CC86CE9841D0
:1092600010082A843AC8D84185453ACA829701C96C
:109270002306A100035524006C00EFF09FF9F6408F
:109280006644256182808280AE8715C5785505C702
:10929000834607002380D50083461700A380D500AE
:1092A000834627012381D50083468701584BA3813C
:1092B000D500D8C18280414681453E851773FE1F87
:1092C000670023FDB727002083A707C091C703A32A
:1092D000870063030300028309458280372700204B
:1092E000032707DF1DC75843AA8705450DC703A5F8
:1092F0000708411106C6930605021306050C9305DF
:109300000506130505040297B2401375F50F4101D8
:1093100082800545828082804DC9357122CD2A84A4
:109320000355050026CB4AC94EC756C306CF52C5C2
:109330005AC1DEDEB68AB2892E89EFF06FE0AA84C8
:1093400039C50C182285EFF03FF483472400138AB7
:109350006400A9CBEF70CF9B2A8B014583CB5400CF
:10936000EF700F99AA840C100818EF10806B085446
:109370002C10EF10A06BD288268A56C05E88D28748
:109380005A8714103010CE854A85EF20D026FA4037
:109390006A44DA444A49BA492A4A9A4A0A4BF65B6D
:1093A0000D618280EF70CF96AA8B014503CB5400EC
:1093B000EF700F942ACE08540C10EF1080662C101A
:1093C0000818EF10A066F2484DBF8280C14709CD52
:1093D0001455C14791CA785501CB83C73600BD46A5
:1093E00063F4F600834787013E85828089476309DD
:1093F000051063870510411106C622C426C28347A3
:1094000015002E842380F50083472500A380F500F6
:10941000834735002381F50083474500A381F5008C
:1094200083475500858B9396870083D7450093F734
:10943000F7EFD58F2392F5008346550093F7F7DFBA
:10944000A20693F60620DD8E2392D5000347550031
:1094500093F6F6BF220713770740558F2392E50056
:1094600083475500FD769386F67F8D87858B758FB4
:10947000AE07D98F2392F50083466500F99B858A54
:10948000DD8E2392D500034765009377270013F7FD
:10949000D6FF5D8F2392E5008347650093F6470072
:1094A0009377B7FFD58F2392F50003476500DD9BC7
:1094B0004D45218BD98F2392F500EF70DF8EAA8462
:1094C0005145EF705F8E0347340093F4F40FC947A2
:1094D000636297021375F50F636EE500834604001F
:1094E0001147E1476368D70083461400054763636B
:1094F000D7008147B240224492443E854101828098
:109500003E85828015C1AA8709458DC141112E85EE
:1095100041469385170006C69770FE1FE78040D02E
:10952000B24001454101828009458280828089479D
:109530001DC595C5411106C603471500AE871946DE
:109540002380E50093052500138517009770FE1F03
:10955000E78000CDB24081473E85410182803E8553
:10956000828015C1AA8709458DC141112E854146CA
:109570009385170006C69770FE1FE78060CAB24049
:1095800001454101828009458280828089471DC949
:1095900095C9411106C60347250083461500AE87CD
:1095A0002207558F2390E50021469305350013854A
:1095B00027009770FE1FE780A0C6B24081473E8516
:1095C000410182803E85828015C1AA8709458DC1EF
:1095D00041112E8541469385170006C69770FE1FE0
:1095E000E78000C4B2400145410182800945828084
:1095F0008280894719C991C903471500BD46E147D3
:1096000063E5E6002380E50081473E85828015C141
:10961000AA8709458DC141112E85414693851700C2
:1096200006C69770FE1FE780A0BFB240014541010A
:10963000828009458280828015C1AA8709458DC133
:1096400041112E8541469385170006C69770FE1F6F
:10965000E78000BDB240014541018280094582801A
:1096600082801DC1AA87094595C141112E85130627
:1096700000049385170006C69770FE1FE78040BA66
:10968000B24001454101828009458280828015C136
:10969000AA8709458DC141112E8541469385170042
:1096A00006C69770FE1FE780A0B7B2400145410192
:1096B00082800945828082801D71A2CC2A8408455F
:1096C00086CEA6CA2306010083440500354793874A
:1096D000F4FF93F7F70F636AF70C37D702008A0796
:1096E00013070791BA979C4382870C08EFF01FD0AD
:1096F000C9476312F50299472306F1000355240078
:109700006C00EFF01FB1F6406644D64425618280BC
:109710000C08EFF07FEB29C98347C100E5F303553F
:109720002400EFF04FF5C5B70C08EFF05FEEE5B79A
:109730000C08EFF01FECC5B70C08EFF0BFDCE1BF81
:109740000C08EFF0BFE4C1BF0C08EFF09FE1E1B7F8
:109750000C08EFF0DFDDC1B70C08EFF0FFED65BFDF
:10976000834715002308F10003552400EFF04F9DB7
:10977000A1470DC10347C500631BF702B7270020AF
:1097800003A707C09D4719C7184309C71008A68536
:109790000297AA872306F10041B70C08EFF07FEC8F
:1097A0009DBF0C08EFF0BFEEBDB79D47B1B7B7271F
:1097B000002003A7C7BFF9B7011122CC06CE26CAE5
:1097C0004AC84EC603470500930720092A84631C34
:1097D000F7128347150039476395E70A835645001A
:1097E0000967610781476398E610B729002003A540
:1097F00009C1CE84630105100C4403C90500631F31
:1098000009008347050085052146A9CF29059770E2
:10981000FE1FE780E0A083A704C1B5C34945EF4020
:10982000AFB82A841DC5930710FC2300F500A300E0
:10983000250183A504C10905414689059770FE1FCE
:10984000E780009E83A704C1A28503C51700EF40EF
:10985000AFC403A504C19770FE1FE780E08C23A866
:1098600004C031A809059770FE1FE780609BEF30A8
:10987000403A05494DF183A709C123802701854757
:109880009DA81307E003639EE7080347250095475B
:10989000631FF70203554500EFF06FAC9147E310EB
:1098A000F5FEB727002083A7C7BFF1DB03A387001E
:1098B000E30703FC0356E4000355440093056400EA
:1098C0006244F240D2444249B24905610283A14751
:1098D000631EF70083456400035544006244F24070
:1098E000D2444249B24905616FF08FFD93060003EF
:1098F0008147E301D7FEF2406244D2444249B24973
:109900003E85056182809306000A8147E315D7FEF4
:10991000EFF09FDA084425D59770FE1FE780C080DE
:10992000B9BF8147C9BF011126CA06CE22CC8944DE
:109930001DCD95CDAA842E8468008D45EF607F8D66
:109940008347E1002685228693F7F70393E7070410
:109950006C002307F100EF200041AA8409E90D46BD
:109960006C00130534009770FE1FE780608BF24097
:1099700062442685D244056182805D714EDE86C6D2
:10998000A2C4A6C2CAC052DC56DA5AD85ED68949E9
:1099900045CD5DCA138B4500420B135B0B01AE8AAC
:1099A0002A8A930530055A85B2849760FE1FE780A6
:1099B00060692A84CD4949C9EF607FB72A895686F4
:1099C000D285935A8900135A0901937BF90F130525
:1099D000440093FAFA0F137AFA0F1359890197701A
:1099E000FE1FE7800096A301740123015401A30028
:1099F000440123002401EF60FFB2AA854146080814
:109A00009770FE1FE780E093214734005A86A285B5
:109A10000808EF20E05BAA891DE121462C00238085
:109A20007401A380540123814401A381240113857F
:109A300044009770FE1FE780C090EF601FB0228542
:109A40009760FE1FE780406EB64026444E859644E0
:109A50000649F259625AD25A425BB25B6161828016
:109A600001114AC82A892E8506CE22CC26CA2EC6C6
:109A7000EFE01FED71C5405971C483475400094799
:109A8000B24593F6B70F6387E60011471305E00F61
:109A90006392E708835704000945639DB706930462
:109AA00084004146CA8526859760FE1FE78040777F
:109AB0004146CA85130584019760FE1FE780407602
:109AC0000347340085469307F7FE93F7F70F63E9E2
:109AD000F6041306C4033285C14532C6EF606FF346
:109AE00032469306C402A6852285EFF0FF828347A3
:109AF000240089CB22856244F240D2444249056168
:109B00006F10A01903473400C947E305F7FEA3010E
:109B1000F4000145F2406244D2444249056182802A
:109B2000930710050145E317F7FE83472400FDD393
:109B300022856244F240D244424905616F10601CA4
:109B40000945C9BF4945F9B7397152D42A8A3285C6
:109B500026DA4ED606DE22DC4AD8AE8932C6EFE0DF
:109B60003FDEC94459C54059C94441C48357040024
:109B700032466390C70883475400A18BB1CB372985
:109B80000020832709DF9304E00FA5C79C47B5C3D6
:109B90009304840126854146D2859760FE1FE780A5
:109BA0002068832709DF8325040826869C47938540
:109BB0000504180881462E858297AA844146CE85E1
:109BC00008089760FE1FE780E07293F4F40F11E13C
:109BD0008944034734009307B005631CF7002285CE
:109BE000EF10E00E8347240091CF9307C005A30137
:109BF000F400F250625426854259D254B259225A86
:109C0000216182809307E005DDB729CD011126CAC5
:109C100006CE22CCAA840945A9C10D4628002E846F
:109C20008D059760FE1FE780A05F8347A10070004D
:109C30002C0093F7F70393E7070426852305F1002B
:109C4000EF20601219E90D46A28568009760FE1F9B
:109C5000E780406A7D153335A000F2406244D2446B
:109C60000561828009458280011152C42A8A3285A9
:109C70004EC656C25AC006CE22CC26CA4AC82E8B21
:109C8000B28AB689EFE0DFCB09ED8944F240624445
:109C900026854249D244B249224A924A024B056182
:109CA00082805C592A89C544F5F34D45EF70AF8F2A
:109CB0001374F50F5145EF700F8FE38809FC83C7CC
:109CC0008901E3E487FC1375F50FE360F5FC930568
:109CD0003005130540089760FE1FE780A036232A51
:109CE000A9022A84CD445DD11306400881459760BE
:109CF000FE1FE780005AA301040023014401230250
:109D00006401231054012326340723240402A302F0
:109D100004008144E30C0AF62285EF001072AA8445
:109D200035D54A85EFF0CFA295B7397122DC06DE32
:109D300026DA4AD84ED652D456D25AD05ECE62CC0B
:109D400066CA0944630B061063090710AA8B3A8997
:109D5000368BB28A2E8CEFE0BFBE2A8A5144630E46
:109D6000050E9305300541459760FE1FE780802D65
:109D7000AA894D447DC18344190083472900A20468
:109D8000C207BE9483470900BE9483473900E207A7
:109D9000BE9483278A0263E697007D57094463993E
:109DA000E70A63070C0083474A000544898BCDC34B
:109DB000930C4B00214681450A85C20C9760FE1F1B
:109DC000E780204D93DC0C01930530056685976094
:109DD000FE1FE78020272A8C4D443DC95A86D68530
:109DE00011059760FE1FE780C0551146CA85628540
:109DF0009760FE1FE780E054414693058A014E8537
:109E00009760FE1FE780E05321478A866686E285D9
:109E10004E85EF20E01B2A841DE521468A85280017
:109E20009760FE1FE780E051214693054900280016
:109E30009760FE1FE780004C8547631EF502A685EC
:109E40005E85EF708FAC62859760FE1FE780C02D46
:109E50004E859760FE1FE780202D2285F2506254C8
:109E6000D2544259B259225A925A025BF24B624C76
:109E7000D24C216182800544F9B77971939705012D
:109E800022D406D626D24AD04ECEC1872E8463D5A0
:109E90000704B7240020938404C203C53400EF30C4
:109EA000BFD72AC611CDEFF03F91B24519E503C5E2
:109EB00024009307F00F631EF5002E85EF30BFC915
:109EC0002165218DB250225492540259F2494561C4
:109ED0008280EF307FDCEDB793F7150091C7EFF08C
:109EE0004F9813451400F9BFA1E10145E1BF850476
:109EF00093F4F40FEFE0BFBEE3F9A4FE33959900AD
:109F00001319050113590901B3772401EDD34A85CB
:109F1000EFE01FE7C167FD176305F500DD45EFF0D2
:109F20000F8B3345240179BF85448549E1B7B727B5
:109F3000002023A807C0B727002023A007C037A709
:109F40000100B72700201307E75423AE07BEB72749
:109F5000002023AAE7C037A70100938747C1130752
:109F6000A725D8C337970100130707EB98C737B762
:109F70000100B72700201307874E23A2E7C037B799
:109F80000100938747C013070705D8C337B70100FF
:109F90001307473398C78280B727002083C747C27B
:109FA000918B89C7B7270020938747C037270020A8
:109FB000232EF7BE01458280011106CE2AC6EFF09E
:109FC0001FF73245B72700209945A381A7C2EFD0DC
:109FD000CFA4F240379501001305E50205616FE05B
:109FE000BFB01C5581C7A1473E858280011122CC9C
:109FF00026CA2A84AE84130500049305300506CED4
:10A000009760FE1FE780000408D46305051013065F
:10A010000004A6859760FE1FE78080207854834760
:10A02000270193F68700638E0610145483C626001A
:10A03000A18A6388061083270408E9EF9305300599
:10A04000130500109760FE1FE780C0FF2320A408BF
:10A050008D4771C1A3020400785483C7140083465E
:10A06000170081EF81EE83C72400918BDDEB8347DE
:10A070002701918BDDE7854711A889C62147A302F7
:10A08000E40099C78347540093E70701A302F40053
:10A090006C5483C72501858B91CF1C54054783C71A
:10A0A00027008D8B6398E7008347640093E71700D0
:10A0B0002303F4008327040899C78347640093E7C8
:10A0C00087002303F4008347540005476398E70C97
:10A0D000930484004146814526859760FE1FE780F2
:10A0E000401B41468145130584019760FE1FE780B0
:10A0F000401A1306C4033285C14532C6EF606F9122
:10A10000832704083246BDC72285EF00903F93079E
:10A11000000525CDA147F2406244D2443E85056149
:10A12000828083C70400834607001547B387E70290
:10A1300037D7020013074796BA97B69783C7070029
:10A14000B1B783C6140091C68346170099C2E14790
:10A1500035BF83C62400D58F918B91DF83C7040060
:10A16000834607001547B387E70237D70200130776
:10A170008794D9B722859306C402A685EFF0CF99BC
:10A180002285EF00903159F5C14703550400A30122
:10A19000F4008145EF60DFE18147B5BF13F7870128
:10A1A00049C3C18B930484004146A9CB8905268508
:10A1B0009760FE1FE780C006414681451305840174
:10A1C0009760FE1FE780E00C834764001306C4031A
:10A1D000328593E747002303F400C14532C6EF60A0
:10A1E0004F838327040832468DC32285EF007031E8
:10A1F0009307200505F1A301F40079BF8145268569
:10A200009760FE1FE780E00845BF9306C402A6855D
:10A210002285EFF06F902285EF003028CD4761DD79
:10A22000D5BD094785456388E70093F7D70F1147E8
:10A230006397E700894503550400EF607FD78347A4
:10A24000640093E747002303F4008327040881C7D1
:10A25000930710054DB7C54779BF83472500638332
:10A260000726797122D406D626D24AD083473500F4
:10A27000130750052A84639FE706034975001306F8
:10A28000C503C14593573900AA97328583C4870017
:10A2900032C6EF501FF8B727002083A707DFA9C7F2
:10A2A0009C47B9C30325040893767900B3D6D440FC
:10A2B0003246858A93050504180893E606081305B7
:10A2C000050882971375F50F05E141460C08130543
:10A2D000C4029760FE1FE780A0F42285EF00F01B08
:10A2E00093076005A301F400B2502254925402591E
:10A2F00045618280130710026395E7021C5503270E
:10A30000050883D7470069EB13F7071071C7785525
:10A31000035747011377071061C393077002A30126
:10A32000F4008347340013077002639FE70C3C5826
:10A3300085E39305300571459760FE1FE78080D067
:10A3400028D819C5714681459760FE1FE78060F4E3
:10A350002458B9C883C7A40191E72285EFF00F877D
:10A36000238DA4002858814541469760FE1FE78051
:10A3700040F228583D478345A5019387F5FF93F7A1
:10A38000F70F6364F700EF50DFE8EF301FAB3C5886
:10A39000A1452398A70013852701EF509FE72C586C
:10A3A00003550400EF00D0409307800203550400DA
:10A3B000A301F400EFE0CFD8414611C58357E50073
:10A3C00013D617003E96B727002003C537C20606EE
:10A3D0008545EF30FFE509BF13F7072011CB78540F
:10A3E000035747011377072001C79307900205BF62
:10A3F00093F707409DD77C5483D7470193F70740D5
:10A400008DD39307B00221BF13078002639BE7023D
:10A410003C5889CB83D507010355040013862701D7
:10A42000EF00903E1C5483D7470013F707202DC33D
:10A430007854035747011377072039CB93079002CD
:10A44000B5B713079002639CE700EF600F8DAA85F4
:10A4500003550400EF00503A9307A00281BF130791
:10A46000A0026393E704EF60AF8AAA8585470145A0
:10A470006384F500814505452EC6EF606F872A8607
:10A48000B24503550400EF00B0331C5483D7470096
:10A4900093F707408DC77C5483D7470193F7074054
:10A4A00099CF9307B00219B71307B0026399E70079
:10A4B000EF604F87AA8503550400EF0070389307BB
:10A4C000F0020DB58280411122C4405926C206C651
:10A4D0007C54AA8483D7470113F7071019C718546F
:10A4E00003574700137707101DE313F7072019C719
:10A4F0001854035747001377072011EB93F70740D1
:10A500008DCF1C5483D7470093F707409DC793070F
:10A510001002A301F4002285EFF03FD4034734007A
:10A520009307F0026310F702224403D52400B240DF
:10A530009244814541016FE09FA99307F002A30176
:10A54000F400DDB7B2402244924441018280397167
:10A5500022DC405926DA4AD84ED606DEAA89AE84D5
:10A560003289630F043C035525008357040063843C
:10A57000A700A14429A08347240091EB9D44F250F9
:10A58000625426854259D254B25921618280938700
:10A59000E5FF93F7F70F2D47E362F7FE37D7020089
:10A5A0008A0713070798BA979C438287B28522854A
:10A5B000EFF03FA3AA84E1B74146CA851305C4045E
:10A5C0009760FE1FE780C0C522851127AA8411C1AC
:10A5D000A14483473400130740056397E7009307BE
:10A5E0009005A301F40061BF130760056395E700C0
:10A5F0009307A005FDB7D147EDB79309C4054E8574
:10A600004146CA859760FE1FE78080C10325040884
:10A6100055C983473400130790056399E7002285E5
:10A6200091279307E005A301F40059A81307A0059B
:10A630006394E7088347740013D737002297834653
:10A6400087009D8BB3D6F640B727002083A707DF8E
:10A65000858A93E606F893F6F60F81DF9C4791DB37
:10A660009305050818084E86130505048297937410
:10A67000F50FE39004F041460C081305C4049760FD
:10A68000FE1FE78020C7834774004D47850793F777
:10A69000F70FA303F4006377F7002285E125930702
:10A6A000E00581B7B727002003C537C28545EF30E5
:10A6B0005F999307500535B71307C005E381E7F6A7
:10A6C000814475BD130984004E86CA85228514080D
:10A6D000EFE09FC441469305C40408089760FE1F3D
:10A6E000E78040C1E30D05E88A861306C403CE85E2
:10A6F0004A85EF1090040DE12285EFE03FCDB727AA
:10A7000000202A8783A7C7C103550400814601465C
:10A710008A858297AA8411C1A14493072002D1B5EA
:10A7200083450600EFE0BF8A61BF0347340093070B
:10A730002002E315F7E47C5889EB93053005714559
:10A740009760FE1FE780009068D86858E30805E22C
:10A750004146CA859760FE1FE78080AC6458228519
:10A76000EFE0DFC6238DA400930730026DBD0347E1
:10A77000340093073002E313F7E08357060068586C
:10A780002146930529002318F50049059760FE1F0F
:10A79000E78000A97C5483D7470113F7270035CB06
:10A7A000185403574700098B2DC793074002A5BDD6
:10A7B0000347340093074002E312F7DC3C5C81EB73
:10A7C00085455D459760FE1FE780C08728DC285CD3
:10A7D000E30805EE834709004146CA85230BF500CF
:10A7E0009760FE1FE780C0A3930750022DBD03476B
:10A7F000340093075002E313F7D8285C19469305F9
:10A80000190041059760FE1FE78080A17C5483D723
:10A810004701918B9DCF1C5483D74700918B95CBDB
:10A820009307600209B57C5C89EB930530055145BF
:10A830009760FE1FE780008168DC685CE30B05D24F
:10A840004146CA859760FE1FE780809D7C5C7D57EE
:10A8500098CB4E85EFF03FC7A5B503250408130636
:10A860000004CA85130505049760FE1FE780409B1E
:10A870002285EFE0BFA683473400130700056395E8
:10A88000E7009307400545B313071005639CE700F5
:10A89000B727002003C537C28545EF308FFA9307ED
:10A8A000500551B313072005E39CE7E0B7270020CC
:10A8B00083A707DFE38F07CA9C47E38C07CA83257A
:10A8C00004089304840018089385050881462686A9
:10A8D0002E858297035504001008A685EF602FF699
:10A8E0009307B00589B3034734009307E005E317E6
:10A8F000F7C88325040841464A859760FE1FE78014
:10A90000609FAD44E30D05C6032504084146CA8592
:10A910009760FE1FE780C0902285EFE03FABB7272E
:10A9200000202A8783A7C7C12C58035504008146FD
:10A9300001468297AA8411C1A1449307100255B120
:10A94000AD47E39FF5D683460600835525001306E1
:10A95000650003450500EF50DFF29DB3894761C2F2
:10A96000DDCD2300A60083C70500A300F60083C742
:10A9700015002301F60083C72500A301F60083C755
:10A980003500A30206002302F60083D74500A18309
:10A99000858BA302F60003D745001377072009C76C
:10A9A00093E72700A302F60083D7450093F70740FB
:10A9B00099C78347560093E74700A302F60083D761
:10A9C000450013974701635807008347560093E7F4
:10A9D0008700A302F6002303060083C74500858B8A
:10A9E0002303F60003D74500098B09C793E7270027
:10A9F0002303F60083D74500918B99C783476600F0
:10AA000093E747002303F60003D745008147218BD6
:10AA100019C703476600136787002303E6003E85D6
:10AA200082802E86AA8505456FF05FF32E86AA8563
:10AA300009456FF0BFF289478DC505C5411106C6AE
:10AA4000AE870D47AA852380E7001385170041468E
:10AA50009750FE1FE780C07CB24081473E85410190
:10AA600082803E85828089478DC505C5411106C615
:10AA7000AE871147AA852380E7001385170041465A
:10AA80009750FE1FE780C079B24081473E85410163
:10AA900082803E85828089478DC505C5411106C6E5
:10AAA000AE871947AA852380E70013851700414622
:10AAB0009750FE1FE780C076B24081473E85410136
:10AAC00082803E85828089479DCD15CD411106C685
:10AAD0001D472380E50003570500AE872146A3806C
:10AAE000E5000357050021832381E5009305250038
:10AAF000138537009750FE1FE7808072B240814770
:10AB00003E85410182803E85828089478DC505C58D
:10AB1000411106C6AE872147AA852380E700138529
:10AB2000170041469750FE1FE780806FB240814773
:10AB30003E85410182803E858280894795C90DC945
:10AB4000411106C625472380E50003470500AE876F
:10AB50001946A380E500930515001385270097503B
:10AB6000FE1FE780E06BB24081473E854101828055
:10AB70003E85828089478DC505C5411106C6AE87D1
:10AB80002947AA852380E70013851700414697507F
:10AB9000FE1FE780E068B24081473E854101828028
:10ABA0003E858280894795C50DC5411106C6AE8791
:10ABB0003147AA852380E700138517001306000498
:10ABC0009750FE1FE780C065B24081473E85410136
:10ABD00082803E85828089478DC505C5411106C6A4
:10ABE000AE873547AA852380E700138517004146C5
:10ABF0009750FE1FE780C062B24081473E85410109
:10AC000082803E858280894791C909C99547238002
:10AC1000F50083470500A380F50081473E858280CB
:10AC2000894791C909C9AD472380F50083470500CD
:10AC3000A380F50081473E85828015C55D718A85B8
:10AC400086C6A2C42A84EFE02FE403550400B7B6F9
:10AC500001000A86938626A29D45EFE0CFD5B64037
:10AC60002644616182800545828015C55D718A85B3
:10AC700086C6A2C42A84EFE02FE103550400B7B6CC
:10AC800001000A869386C6A29D45EFE0CFD2B6406A
:10AC9000264461618280054582805D71A2C493056E
:10ACA000C5022A8441460A8586C69750FE1FE78062
:10ACB000205703550400B7B601000A86938666A3A1
:10ACC000C545EFE04FCFB6402644616182805D719B
:10ACD000A2C49305C5032A8441460A8586C69750B7
:10ACE000FE1FE780E05303550400B7B601000A8653
:10ACF000938666A6C545EFE00FCCB6402644616159
:10AD00008280B727002083A707DFB1CB9C435D710A
:10AD1000A2C486C62A841305E00F95CF0325040834
:10AD20009305050C1305050882978325040813066F
:10AD300000040A85938505089750FE1FE780404E62
:10AD400003550400B7B60100938646BA0A869305F8
:10AD50001004EFE04FC6B6402644616182801305BF
:10AD6000E00F8280317122DD2A840355050026DB45
:10AD700006DF4AD94ED752D556D35AD15ECF62CDCF
:10AD8000EFD01FBC3C58AA8489EB93053005714570
:10AD90009750FE1FE780002B28D82858CD470DC9B3
:10ADA000714681459750FE1FE780A04E0329040796
:10ADB0002285EFE0AFE1230DA90083472400372966
:10ADC0000020638A0712832709DF85E39307E00FDA
:10ADD000FA506A54DA544A59BA592A5A9A5A0A5BAA
:10ADE000FA4B6A4C3E852961828083AB0701E38F71
:10ADF0000BFC032B0408EF50AFF12A8C0145EF50F8
:10AE00002FEF83C754003858130B0B029309C40368
:10AE1000130AC405938A64003AC0B337F0002A8746
:10AE2000930801045688B33680015286CE855A8530
:10AE3000829B1C5403C727002307E10203C71700A6
:10AE4000A306E10283C707002306F102832709DF77
:10AE5000B5DF03AB4701E30B0BF683C75400B337F1
:10AE6000F0003ECEEF50CFEAAA8B0145EF504FE8FD
:10AE700003270408F2472AC03AC2B3387001568843
:10AE80007810930684004E86D2858800029B7C54FD
:10AE900003C727012305E10203C71700A304E1024A
:10AEA00083C707002304F102832709DF03A94701B1
:10AEB000EF500FE62A8B0145EF508FE383C8540013
:10AEC0009C082A883EC2B3381001B337600138109D
:10AED000930684015286CE8556C088000299035598
:10AEE0000400B7B60100938666BD9008C545EFE043
:10AEF0008FACAA87F1BD83C65400832709DF032BDB
:10AF00000408B336D00083AB070136CEEF504FE0D4
:10AF10002A8C0145EF50CFDD3C58F246130B0B0253
:10AF2000130AC4059309C403938A64002A8893080A
:10AF300001044E86D2853EC05687B33780015A85BC
:10AF4000829B1C54130B010303C727002307E10254
:10AF500003C71700A306E10283C707002306F10217
:10AF6000832709DF83AB470183C75400B337F00061
:10AF70003ECEEF50EFD92A8C0145EF506FD7F24704
:10AF80002AC0B338800156887810930684004E8614
:10AF9000D2855AC28800829B8325040841465A857F
:10AFA0009750FE1FE7800035AD47E31205EE0DB563
:10AFB000B7B601002E86938666A9C5456FE0AF9FA0
:10AFC0005D71B287A2C42300B1002A84BE85130537
:10AFD0001100194686C69750FE1FE7806024B7B659
:10AFE00001000A8622859386A6B3A145EFE0AF9CB7
:10AFF000B640264461618280B7B601002E869386F2
:10B00000A6B0C5456FE02F9B5D71B287A2C4231027
:10B01000B1002A84BE8513052100214686C69750BB
:10B02000FE1FE780E01FB7B601000A8622859386DF
:10B0300066ACAD45EFE02F98B64026446161828052
:10B04000B7B601002E86938646B7C5456FE0AF962A
:10B05000797122D406D626D28347350013073005EE
:10B060002A846384E708130750056396E70893076B
:10B07000A005A301F50083477500C14513D737002C
:10B080002A97834687009D8B1305C503B3D6F640E8
:10B09000858A93E606F893F6F60F36C6EF506F975B
:10B0A000B246B727002083A707DF9DCB9C478DCBF7
:10B0B0000325040818081306C403930505041305A3
:10B0C000050882971375F50F01ED1305C40241467B
:10B0D0000C089750FE1FE780A0142285EFF0FFBBFD
:10B0E000B250225492544561828093079005A30187
:10B0F000F50081467DB7130710026396E7027C5581
:10B100000327050883D747016316070E13F71700B7
:10B110006302070E185503574700058B61CF93074D
:10B120002002A301F4008347340013072002639D2B
:10B13000E70E3C5889EB9305300571459750FE1F8B
:10B14000E78040F028D82458C9C02285EFE00FA836
:10B15000238DA4002858814541469750FE1FE78063
:10B16000401328583D478345A5019387F5FF93F782
:10B17000F70F636DF702B727002083C7B7DFD5C38A
:10B180004146814508089750FE1FE7808010B7258B
:10B1900000201946938545AF08089750FE1FE780A9
:10B1A000200830580C082E85EF90401FEF20FFC874
:10B1B0003C58A1452398A70013852701EF506F85C0
:10B1C0002C5803550400EFF0BFDE930730020355FF
:10B1D0000400A301F400EFD0AFF6414619C10356B5
:10B1E000E500B727002003C537C206068545EF30C6
:10B1F0002F84FDB513F7270009CB185403574700D8
:10B20000098B01C79307400229BF918BE38D07F09B
:10B210001C5483D74700918BE38707F093076002A4
:10B2200009B7EF401FFF59B713073002639AE702CF
:10B230003C5889CB83D507010355040013862701A9
:10B24000EFF09FDC7C5483D7470113F7270021CF11
:10B25000185403574700098B39C79307400285BF2D
:10B2600013074002639CE700EF502FABAA850355FC
:10B270000400EFF07FD89307500291BF13075002EC
:10B280006390E704EF50CFA80DE9814505452EC630
:10B29000EF500FA62A86B24503550400EFF05FD2A7
:10B2A0007C5483D74701918B9DC71C5483D747009B
:10B2B000918B95C39307600219BF85450145C1BFB6
:10B2C000130760026399E700EF50CFA5AA850355E5
:10B2D0000400EFF0FFD67C540327040883D747010E
:10B2E00019EF13F7071001CF1854035747001377CE
:10B2F000071011C793077002A301F400D5B313F729
:10B30000072011CB1854035747001377072001C7B4
:10B3100093079002D5B793F7074091CB1C5483D77E
:10B32000470093F7074081C79307B002F1B793072F
:10B33000F002D9B7397122DC26DA4ED652D406DEB5
:10B340004AD8AE89328AAA84EFD08FDF405941466D
:10B3500081450A859750FE1FE780A0F325C8035951
:10B360000400631599060347340093071002631F16
:10B37000F7028327040899CF2C58A9C94A85EF10F2
:10B38000900A0545F2506254D2544259B259225A99
:10B39000216182808A861306C4059305C4031305C0
:10B3A0008400EF0090391DE18A85C9BF2C5899CDE2
:10B3B00083D70501639C47012146C9054E859750F7
:10B3C000FE1FE78020F319C12C584DBF2685EFD012
:10B3D0002FD72A8405455DD44C54A1C983D70501D4
:10B3E000639547052146C9054E859750FE1FE780A6
:10B3F00060F08547631BF502B727002083C7B78E2F
:10B4000091C74C5483C7B501639BA70CBD452685E6
:10B41000EF10E07BB727002083A787AA0145BDD3A3
:10B420001D45894582970145B1BFB727002003C755
:10B43000C7DFB7290020938989A7058B3E8931C3CF
:10B44000B72700200347540083C747DF631BF70279
:10B45000B72500201946938555DF130564009750E2
:10B46000FE1FE78020E98547631DF50083A70903D8
:10B4700081C791451D458297BD452685EF102075F2
:10B4800009B7372700200347B7DF83A7090331CB6C
:10B490000347C9DF098B09CB81C795451D458297B5
:10B4A0002685EF108078F1BD81C78D451D458297B7
:10B4B0004146814508089750FE1FE78080DDB7258B
:10B4C00000201946938545AF08089750FE1FE78076
:10B4D00020D50C082E850A86EF80506C8A8526853B
:10B4E00079BD8545C5FF6DBF797122D440594AD0D9
:10B4F0004ECE52CC06D626D2AA892E8A3289630D28
:10B50000046A0355250083570400638CA700A144F7
:10B51000B2502254268502599254F249624A45613A
:10B5200082808344240099C09D44DDB79387F5FF52
:10B5300093F7F70F3147E369F7FE37D702008A0721
:10B540001307079BBA979C4382871C54E9F3930522
:10B550003005130500049750FE1FE780A0AE08D405
:10B560005DD503470900914763F4E7008D444DB76B
:10B57000034719008547E3EBE7FE13060004CA857D
:10B580009750FE1FE780C0C90C547054A3020400FA
:10B59000D4415C4A858AFD8E83574601F99BD58F3D
:10B5A000231AF600D841544AF59B0583058B858202
:10B5B000F98E8606DD8E231AD600DC41584AED9AB4
:10B5C0008983858B09837D8F0A07558F231AE600AF
:10B5D000D4415C4A5D9B8D82858A8D83F58F8E0771
:10B5E000D98F231AF600D841544A93F7F7EF2183F5
:10B5F000058BA182F98EA206DD8E231AD600DC41CE
:10B60000584AA583858B25837D8F9317970013F761
:10B61000F6DF5D8F231AE600D4415C4AA982858A51
:10B62000A983F58F9396A7009377F7BFD58F231A39
:10B63000F600D441584AAD82858A2D83758FFD76F8
:10B640009386F67F2E07F58FD98F231AF60083474E
:10B65000260103250408A18B6387071083C72500F3
:10B66000A18B63820710E31405EA930530051305E7
:10B6700000109750FE1FE780E09C2320A408E307FA
:10B6800005EE7C54A30204000347190083C617008B
:10B6900089EA45C38347540093E70701A302F400F6
:10B6A00029A0A147A302F40075F72285EFF0EFDB94
:10B6B0006C5483C72501858B81CF1C5483C7270019
:10B6C0008D8B99C78347640093E717002303F40029
:10B6D0008327040899C78347640093E787002303FF
:10B6E000F4008347540005476393E70C41468145C6
:10B6F000130584009750FE1FE780A0B9414681459D
:10B70000130584019750FE1FE780A0B8C1451305BB
:10B71000C403EF401FB0032704089307000511E39B
:10B72000C14703550400A301F4008145EF505F8831
:10B73000C5B303C72701118B19E703472900118BF4
:10B7400019E38547A1BF83C7070015478346090052
:10B75000B387E70237D7020013074796BA97B69721
:10B7600083C7070025BF19C59750FE1FE780C09B00
:10B77000232004087C5403C7170011C7034719008E
:10B7800019C3E14721BF03C72701118B09E703470D
:10B790002900118B5DD783C7070015478346090031
:10B7A000B387E70237D702001307879445BF13F723
:10B7B000870131CFC18B130584004146A9C3890598
:10B7C0009750FE1FE780C0A54146814513058401BF
:10B7D0009750FE1FE780E0AB83476400C145130527
:10B7E000C40393E747002303F400EF409FA283279D
:10B7F000040881CF93072005A301F40011BB814504
:10B800009750FE1FE780E0A8C1B7CD47F5B70947BD
:10B8100089456386E70011476398E700854503552E
:10B820000400EF50EFF821A01947E389E7FE8347B2
:10B83000640093E747002303F4008327040881C7CB
:10B840009307100555BFC54745BF4146CA85130537
:10B85000C4049750FE1FE780A09C83473400130761
:10B860006005639CE700B727002003C537C2854504
:10B87000EF202FFD9307500541B745476383E7024B
:10B880009306C4021306C403930584002285EFD0F7
:10B89000BFA82285EFF06FC0AA8411C1A144D1478F
:10B8A000A1BFC94791BF9309C4054E854146CA85CA
:10B8B0009750FE1FE780C0960325040861CD83479B
:10B8C0003400130790056398E7002285EFF02FC03E
:10B8D0009307E00515B71307A005639EE706B72792
:10B8E000002083A707DFE38107C403A88700E30DD7
:10B8F00008C283477400930505084E8613D73700A6
:10B900002297834687009D8B0A87B3D6F640858AA7
:10B9100093E6060813050504029841468A85130537
:10B92000C4049750FE1FE780E09C11E1D284228579
:10B93000EFF0EFB983477400CD461307E0058507A4
:10B9400093F7F70FA303F40063E4F6001307600511
:10B95000A301E40075BE1307C005E39BE7BAB72750
:10B96000002083A707DFE38107BC9C47E38E07BA6B
:10B9700093050508130984000A8781464A862E85A7
:10B980008297035504000A86CA85EF504FEB930750
:10B99000B0059DB58A864E86930584002285EFD03A
:10B9A000BF9741469305C4040A859750FE1FE78060
:10B9B00060948547D284E31DF5B42285EFF02FB162
:10B9C000AA84E31605B4930710023DB5034734007B
:10B9D00093077002E31AF7B47C5889EB930530059E
:10B9E00071459740FE1FE780E06568D86858E30D11
:10B9F00005B2CA8541469750FE1FE7806082032941
:10BA000044072285EFD09F9C230DA9009307800255
:10BA1000E5B30347340093078002E317F7B0835779
:10BA2000060068582146930529002318F5004905AA
:10BA30009740FE1FE780C07E7C5483D7470113F7F1
:10BA4000072025CF1854035747001377072035C721
:10BA50009307900255B30347340093079002E31510
:10BA6000F7AC3C5C89EB930530055D459740FE1FC4
:10BA7000E780405D28DC285CE30805AA4146CA85CA
:10BA80009740FE1FE780C0799307A002B5B3034734
:10BA900034009307A002E319F7A883470600285C47
:10BAA000194693051900230BF50041059740FE1F29
:10BAB000E78000777C5483D7470193F70740B1C7ED
:10BAC0001C5483D7470093F70740A1C39307B002E4
:10BAD00025B3034734009307B002E317F7A47C5C57
:10BAE00089EB9305300551459740FE1FE78080554F
:10BAF00068DC685CE30D05A04146CA859740FE1FDF
:10BB0000E78000727C5C7D5798CB03D52900814586
:10BB1000EFD0EFCBF5BA034734009307F004E3F816
:10BB2000E79E03250408E304059E13060004CA8566
:10BB3000130505049740FE1FE780806E2285EFF015
:10BB40004F9CAA842285EFD06FF9834734001307F6
:10BB50000005639FE700B727002003D6E90003C56F
:10BB600037C285450606EF20AFEC9307300569B173
:10BB7000130710056395E70093076005B5B9130730
:10BB80002005E397E7989307C005BDB1034734004C
:10BB90009307E005E31DF796032504084146CA858F
:10BBA0009740FE1FE780C0672285EFF0AF9BAA8415
:10BBB00019BD83450600A9BF85478144E39AF594E2
:10BBC00003284600834736000347260083461600B5
:10BBD00083552500034606000145EF403FC10DBADD
:10BBE0008147C1463307F500B388F50003470700D6
:10BBF00083C808003308F600850733471701230080
:10BC0000E800E391D7FE82800147BD471308F00F9B
:10BC10003306F50083460600B388F500FD17860657
:10BC2000558F2380E8000347060093F7F70F1D8325
:10BC3000E39007FF82808147930800F8414893F61C
:10BC4000F70F3387F50063FCC600B306F50083C623
:10BC500006002300D7008507E39307FF82806395E2
:10BC6000C60023001701C5BF23000700EDB701116F
:10BC70004AC856C22E89AA8A93053005414506CE88
:10BC800022CC26CA4EC652C4328A9740FE1FE78095
:10BC9000603BAA849305300541459740FE1FE7802D
:10BCA000603A2A84CD49A5C431CD414681459740AB
:10BCB000FE1FE780005E2686A2855685EF80006E17
:10BCC000AA8929E18387040063D30706A285268514
:10BCD000EFF09FF3B7D502004A869385459E2285F3
:10BCE000EFF01FF08307090063D80704A2854A8597
:10BCF000EFF09FF1B7D5020052869385459E2285CD
:10BD0000EFF01FEE26859740FE1FE780E04111C44B
:10BD100022859740FE1FE7802041F24062444E8515
:10BD2000D2444249B249224A924A05618280CA8578
:10BD30002685EFF07FED7DB7D2854A85EFF0DFEC09
:10BD4000D1B781474146B306F5003387F500034775
:10BD5000070003C806008507334707012380E60074
:10BD6000E393C7FE8280011126CA4EC6AE84AA891B
:10BD700093053005130500034AC806CE22CC32894C
:10BD80009740FE1FE780002C2DC513060003814558
:10BD90002A849740FE1FE780C04F4146CE8522850A
:10BDA0009740FE1FE780E059A6850D461305D40194
:10BDB0009740FE1FE780E058130604029305040134
:10BDC0002285EF80A05DAA840D469305D4024A85A2
:10BDD0009740FE1FE780E05622859740FE1FE780D0
:10BDE000A034F240624426854249D244B2490561FA
:10BDF0008280CD44FDB75D714EDE62D4AE892A8C5F
:10BE00009305300513050003A6C2CAC052DC56DAFA
:10BE10005AD85ED686C6A2C4B28B368BBA84BE8A86
:10BE20004289468A9740FE1FE780C02163050510BE
:10BE30001306000381452A849740FE1FE780604572
:10BE40004146E28522859740FE1FE780804F4146AC
:10BE500081450A859740FE1FE780A0431D46DE8589
:10BE60000A859740FE1FE780C04D1D46DA85130501
:10BE700071009740FE1FE780C04C33392001B33476
:10BE8000900041468145080823072101A30791003E
:10BE90009740FE1FE780E03F1946D6854808974047
:10BEA000FE1FE780004A1946D2851305A10197407D
:10BEB000FE1FE7800049930404014146CE85268594
:10BEC0009740FE1FE780E0478A852685EFF07FE7F1
:10BED000930904024E86A6852285EF80204C2A898C
:10BEE0000DE94146CE8526859740FE1FE780403309
:10BEF0000C082685EFF0FFE44E86A6852285EF80AC
:10BF0000E0492A8946454146CE859740FE1FE78095
:10BF1000404322859740FE1FE7800021B64026441B
:10BF20004A8596440649F259625AD25A425BB25B3C
:10BF3000225C616182804D49D5B7011126CA52C485
:10BF4000AA842E8A13050003930530054AC84EC6FD
:10BF500006CE22CC3289B6899740FE1FE780800E3C
:10BF600035C52A84A68541469740FE1FE780603D7F
:10BF7000930404012146D28526859740FE1FE78061
:10BF8000403CCA852146130584019740FE1FE78087
:10BF9000403B13090402A6854A862285EF800040B3
:10BFA000AA844146CA854E859740FE1FE7806039C6
:10BFB00022859740FE1FE7802017F24062442685C5
:10BFC0004249D244B249224A05618280CD44F5B744
:10BFD00039715AD05ECE2A8BAE8B41459305300520
:10BFE00006DE26DA52D456D262CC66CA6AC8368CCD
:10BFF000328DBA8C22DC4AD84ED69740FE1FE7809D
:10C000006004AA8A9305300541459740FE1FE780EA
:10C0100060032A8ACD44638E0A0859C52A86D685CC
:10C020005A85EFF0DFC4AA8441E19305300541450C
:10C030009740FE1FE78000012A899305300541459E
:10C040009740FE1FE7800000AA89630A090E630675
:10C05000050E1304FD0011841376FD0049C07D1404
:10C060004204418035EE131544004E86D6855E9518
:10C07000EFF01FB7414681454A859740FE1FE78094
:10C080004021014D93170D01C18363F48708BDC0A2
:10C090004A859740FE1FE7802009638709004E8587
:10C0A0009740FE1FE780400856859740FE1FE780B7
:10C0B000A00763070A0052859740FE1FE780C0066D
:10C0C000F250625426854259D254B259225A925A99
:10C0D000025BF24B624CD24C424D216182800144A2
:10C0E000131544008A855E95EFF0FFB44E86D28525
:10C0F0000A85BDBF93154D000A86DE954A85EFF08F
:10C100003FAE4A868A855A85EF804029AA84050D6C
:10C1100095BFBDFC0A86CE854A85EFF07FAC4A8686
:10C120008A855A85EF808027AA846686CA856285BB
:10C130009740FE1FE780C00EA1BFCD4491BFCD4404
:10C14000A9BF397162CC2A8C594526DA4AD84ED615
:10C1500052D456D25AD05ECE06DE22DCAE8B328B63
:10C16000B68A3AC63E8AC289468983440104EF10E2
:10C17000BFA349C19167938717E92310F50085474D
:10C180002301F5002A8432472105630C0C04930730
:10C190001003A301F400194681459740FE1FE78074
:10C1A000400F23036401A3035401230A94002312C4
:10C1B0007401231744012318340123192401A28593
:10C1C000B72700206254F250D2544259B259225A31
:10C1D000925A025BF24B624C03C507C221616F1099
:10C1E000BFABA30104001946BA859740FE1FE78044
:10C1F000200345BFF2506254D2544259B259225AD8
:10C20000925A025BF24B624C21618280011122CC76
:10C210002A84314506CE2EC632C436C23AC0EF104B
:10C22000BF9829C19167938717E92310F500B2459C
:10C230002246924602478D472301F500A30185005F
:10C240006244B72700202312B5002313C50023142E
:10C25000D5002315E500F240AA8503C507C2056194
:10C260006F109FA3F24062440561828001114AC8A9
:10C270002A89394526CA06CE22CC2EC6B284EF10B2
:10C28000BF9231C1B2459167938727E92310F5002A
:10C2900091472301F500A30125012312B5002A844B
:10C2A000A685190521469740FE1FE78060F7A28505
:10C2B000B72700206244F240D244424903C507C276
:10C2C00005616F107F9DF2406244D244424905618E
:10C2D000828001114AC82A89414526CA06CE22CC4D
:10C2E0002EC6B284EF105F8C29C19167B245938747
:10C2F00027E92310F50095472A842301F50023122E
:10C300002501214619059740FE1FE78060F1A285AF
:10C3100023179400B72700206244F240D2444249D8
:10C3200003C537C205616F103F97F2406244D244A3
:10C33000424905618280011122CC2A84394506CE0A
:10C340002EC632C436C23AC0EF101F8629C191678B
:10C35000938717E92310F500B2452246924602471B
:10C3600099472301F50023128500B7270020624476
:10C370002313B5002314C5002315D5002316E500AB
:10C38000F240AA8503C507C205616F10FF90F24015
:10C39000624405618280797122D406D62A842EC631
:10C3A00032C436C23AC0EFC0AFD91DC1B245224631
:10C3B00092460247231CB100231DC1002C0813061E
:10C3C000F00F2285231ED100231FE100EFC04FC7CD
:10C3D000B250225445618280011122CC2A84394511
:10C3E00006CE2EC632C436C23AC0EF10EFFB29C1CA
:10C3F0009167938717E92310F500B24522469246CC
:10C4000002479D472301F50023128500B72700202E
:10C4100062442313B5002314C5002315D500231649
:10C42000E500F240AA8503C507C205616F10DF86EB
:10C43000F2406244056182805D712AC613052002C4
:10C44000CAC04EDE52DC56DA5AD85ED662D466D204
:10C450006AD086C6A2C4A6C26ECE2E8CB28B368B94
:10C460003AC43E8DC28CC68A035A010583594105E0
:10C4700003498105EF104FF369C5916632439386F6
:10C4800016E9A9472A842310D5002301F500930D4E
:10C49000E4002105930444012247630D030693073A
:10C4A0001003A301F400194681459740FE1FE78061
:10C4B00040DE194681456E859740FE1FE78060DDAE
:10C4C0001946814526859740FE1FE78080DC2303BF
:10C4D0007401A30364012300240323128401231D98
:10C4E0005401231E4401231F3401A285B7270020D5
:10C4F0002644B64096440649F259625AD25A425BE3
:10C50000B25B225C925C025DF24D03C507C26161C1
:10C510006F108FF8BA85A301040019469740FE1FDB
:10C52000E78000D0EA856E8519469740FE1FE780B8
:10C5300020CF1946E68526859740FE1FE78040CE2E
:10C5400079B7B640264496440649F259625AD25AFF
:10C55000425BB25B225C925C025DF24D6161828063
:10C56000011122CC2A84214506CE2EC632C436C201
:10C57000EF108FE315CD224692469167938717E916
:10C580002310F500B245B1472301F500A301850052
:10C590002303C500A303D5006244B727002023125C
:10C5A000B500F240AA8503C507C205616F10CFEE42
:10C5B000F24062440561828041110D4506C6EF10CC
:10C5C000AFDE0DC5930710F92300F5009307E003D4
:10C5D000A300F500C5472301F500B7270020B240AE
:10C5E000AA8503C507C241016F100FEBB24041019C
:10C5F0008280011122CC2A84294506CE2EC632C45F
:10C6000036C2EF106FDA15CDB24592469167938727
:10C6100017E92310F5002246C9472301F50023023C
:10C62000B500A30185002304D5006244B72700208C
:10C630002313C500F240AA8503C507C205616F1028
:10C64000AFE5F24062440561828001114AC82A893F
:10C650002D4526CA06CE22CC2EC6B284EF10CFD4EA
:10C6600029C5B245930710F92300F5009307E003AD
:10C67000A300F500CD472301F500A3012501230206
:10C68000B5002A84A685150519469740FE1FE78048
:10C6900020B9A285B72700206244F240D244424923
:10C6A00003C507C205616F102FDFF2406244D24418
:10C6B000424905618280011122CC2A84214506CE9F
:10C6C0002EC6EF106FCE05C9B2459167938717E963
:10C6D0002310F500D1472301F5002303B5002312F1
:10C6E0008500B72700206244F240AA8503C507C22F
:10C6F00005616F106FDAF2406244056182800111BA
:10C7000022CC2A84214506CE2EC632C4EF10CFC9D2
:10C710001DC52246B245930710592310F500230189
:10C7200085002303C5006244B72700202312B5000B
:10C73000F240AA8503C507C205616F10EFD5F2402C
:10C74000624405618280011122CC2A84214506CEF3
:10C750002EC632C4EF104FC51DC92246916793877C
:10C7600027E92310F500B245A1472301F500230373
:10C770008500A303C5006244B72700202312B5003B
:10C78000F240AA8503C537C205616F10EFD0F240B1
:10C79000624405618280011122CC2A84314506CE93
:10C7A0002EC632C436C23AC0EF100FC015CD224695
:10C7B0008567B24592460247938717C92310F50053
:10C7C000230185002303C5006244B72700202312FC
:10C7D000B5002314D5002315E500F240AA8503C552
:10C7E00007C205616F104FCBF24062440561828041
:10C7F000011126CAAE844AC82A891385C40006CE10
:10C8000022CC32C6EF104FBA1DCD8567938717E94A
:10C81000B2452310F50023019500231225012A8437
:10C82000310508C426869740FE1FE780609FA285D9
:10C83000B72700206244F240D244424903C507C2F0
:10C8400005616F106FC5F2406244D24442490561F0
:10C850008280011122CC2A84194506CE2EC6EF1003
:10C86000AFB405C98567938717F92310F500B24562
:10C870008547A301F500230185006244B727002006
:10C880002312B500F240AA8503C507C205616F10E7
:10C89000AFC0F240624405618280411122C42A8403
:10C8A0000D4506C6EF104FB005C5930710F92300DC
:10C8B000F500E947A300F500230185002244B727CE
:10C8C0000020B240AA8503C507C241016F10CFBC4A
:10C8D000B240224441018280011122CC2A842145A8
:10C8E00006CE2EC6EF104FAC0DC99167938727E98E
:10C8F0002310F500B245930700032301F50023033D
:10C9000085006244B72700202312B500F240AA85B3
:10C9100003C537C205616F102FB8F240624405614C
:10C9200082800111214506CE2EC632C4EF10CFA75A
:10C9300005C98567B2452246938707392310F5005C
:10C9400085472301F500B72700202312B5002313E4
:10C95000C500F240AA8503C587B805616F10CFB343
:10C96000F24005618280397122DC1304F5FF4AD858
:10C9700052D456D25ECE420406DE26DA4ED65AD0C5
:10C98000894B2A8A3289B68A418063967515B72BFE
:10C99000002083C78B975E8B89448DCF83C9160097
:10C9A00083C706009144A209B3E9F900B727002024
:10C9B00083D787A8F51763DFF9009307C6FF639D48
:10C9C000F90831452EC6EF102F9E2A84B24519ED85
:10C9D0009304F00FF250625426854259D254B25952
:10C9E000225A925A025BF24B21618280420913590A
:10C9F00009012302B50023132501930700F9150946
:10CA0000A1652310F5002311450185054A8597305E
:10CA1000FE1FE780206308C415C983C78B979385E1
:10CA2000EAFF13562900FD17238CFB969740FE1F43
:10CA3000E780E0821C44A28589071CC4B727002038
:10CA400003C587B8EF104FA5814469B72285973099
:10CA5000FE1FE780606DADBF9307D6FFE3CAF9F60E
:10CA6000B1473304F402B724002083A7C4B8A297C7
:10CA700003C7A70019C7884309C59730FE1FE78081
:10CA8000A06A13854900A16542058505418103AA75
:10CA9000C4B89730FE1FE780E05A83A7C4B8229A33
:10CAA0002320AA00A297884305D505472385E700E0
:10CAB00083478B974A86D685FD17230CFB969730C4
:10CAC000FE1FE780E07583A7C4B83E9423132401BA
:10CAD0002312340195BF8547E39CF5EEB14733043B
:10CAE000F402372B00208327CBB8DA89A29703D72B
:10CAF0006700884345CB83D74700B306C70091073B
:10CB000063C2D70A3A95D6859730FE1FE7804071F9
:10CB10000327CBB88144229783576700CA97C2077F
:10CB2000C1832313F700035747001107E394E7EA93
:10CB30003145EF106F87AA8521C1930700F92310B3
:10CB4000F5008327CBB82302750123114501A29775
:10CB500003D767009C432313E5001CC5B7270020BB
:10CB600003C587B8EF104F938327CBB83E942313A8
:10CB7000040023050400B9BD8327CBB8A2978843DE
:10CB800011C99730FE1FE780205A8327CBB8A297A0
:10CB900023A0070083A7C9B83E94231304002305EC
:10CBA00004005DB511C99730FE1FE780E05783A7E9
:10CBB000C9B8A29723A0070083A7C9B885443E94AB
:10CBC000231304002305040031B56FA050196FA092
:10CBD000901A6FA03043054582800545828041113F
:10CBE00006C6EFA09019B2400145410182806FA0B6
:10CBF000101C6FA0301E6FA070216FA090236FA03B
:10CC000090256FA090276FA090296FA0902B6FA008
:10CC1000302D6FA0302F8347160003460600A20771
:10CC20005D8E6FA070306FA0B0316FA070346FA0B8
:10CC300030376FA0103A6FA010406FA030426FA045
:10CC400050446FA070466FA090486FA0B04A034355
:10CC50000100030E4100834E8100034FC100834F4A
:10CC6000010183424101834381017EC816CA1ECC63
:10CC70007AC676C472C21AC06FA0D0496FA0D04ED7
:10CC80006FA0F0506FA0105305458280054582804B
:10CC9000054582806FC0A05D054582800545828084
:10CCA0006FC0C063B7D6020081479386469F1308C2
:10CCB000F00F3387F6000346070013170601418380
:10CCC0006364E50063130601828003D60500636593
:10CCD000C7002390E5008280850793F7F70FD1BF47
:10CCE00041119397050122C406C626C2C1872E842E
:10CCF00063D50702EF005FF2AA8409CD83470500E0
:10CD0000054793C707086364F700EF503034268562
:10CD1000EF007FE42165218D21A893F7150091CFC5
:10CD2000B727002083A747C991C3829713451400F2
:10CD3000B240224492444101828093F7250091CB76
:10CD4000B727002083A787C991C382971345240082
:10CD5000C5B793F7850099CBB727002083A747CAAB
:10CD6000FC5791C3829713458400D9B793F74500C8
:10CD700099CBB727002083A747CABC5791C3829796
:10CD80001345440075B793F7050281CFB7270020FC
:10CD900083A787CB83A7070991C382971345040212
:10CDA00041BF93F7050181CFB727002083A787CB29
:10CDB00083A7C70891C382971345040195BF939732
:10CDC00025010145E3D607F6B7270020938707C35F
:10CDD00083C6770003C6670083C5570003C54700B5
:10CDE000EFA0104A096505BF411126C2B7240020F3
:10CDF000B727002013060012814522C42A84138518
:10CE000004C306C623AA07D44AC09730FE1FE78092
:10CE100040480145EF20400B0145EF202012B72785
:10CE20000020A38187A2B707D707138404C3B107E3
:10CE30005CC8B7C70C0C938717131CCCB7C7D707B0
:10CE4000938717135CCCF177938717132310F402A1
:10CE500081477D47232EF40C8327840C232CE40C7C
:10CE60005D671307F71F37290020D98F130989A79A
:10CE70002324F40C2328F40C8347E9000327C40C73
:10CE8000A30C0402A30AF40AA30EF40AF977FD170F
:10CE9000231FF40E2310F410FD472301F410930711
:10CEA0003030231DF402231EF402232AE40CEF1079
:10CEB0001FBD9307C01C2319F4068357490003576D
:10CEC0000901A301A400A983A30EF4069306B00FE1
:10CED000938704C363F4E6001307B00F93150701AB
:10CEE000C1811386E50093163600C206C1822395E0
:10CEF000E7022397E7022396D7022398D7026D45CE
:10CF0000938404C363F3A5006D472391E402930562
:10CF10008014368763F4B600130780142392E70267
:10CF20002394E7020547A38FE7023707030013079F
:10CF3000C71CB8C3370716000E061307079023A2B5
:10CF400007042393C702D8DBEF703055EF30B02FC2
:10CF5000EF70600B2244B2409244024941016F508D
:10CF6000D067397122DC3704400026DA4ED6AE8411
:10CF7000AA899305E4FF054506DE4AD8EF101FB9DC
:10CF8000498C13170401418321839317840013599B
:10CF90000401D98F231601001379F90F10088A852F
:10CFA0004E852317F100A306210102C002C202C46C
:10CFB00002C802CA02CC02CEEF70403E8347E101B4
:10CFC0000347D101A3818400A2074207BA97034710
:10CFD000F101218023828400BA97F25062542380A9
:10CFE000F40013D78700C183A3822401A380E40047
:10CFF0002381F4004259D254B25921618280B7256D
:10D0000000203725002001111946938505A9130535
:10D0100005D106CE22CC26CA4AC891644EC69730A6
:10D02000FE1FE780E01F9385F4FF0145EF10DFABA3
:10D030002A84FD550145EF107FADA287FD147D596F
:10D0400033F79700B366E500D5CA6314250163077B
:10D05000970A37240020130704C32308F70EA1837F
:10D0600093E707FC9169C1642326A70EA308F70E76
:10D07000130404C3FD19FD14CE850145EF10DFA68E
:10D080002A89FD550145EF107FA8B3672501EDD72B
:10D09000FD576314F500E30139FF93570501230A97
:10D0A000F40E93578501A30AF40E8317040E231977
:10D0B000A40E230B240F4205135989001379F90399
:10D0C0004185A30B240F658DE58F6312F5020317CD
:10D0D000440F8317240E658FE58F631AF70003173B
:10D0E000640F8317440E658FE58FE307F7F8F2406E
:10D0F0006244D2444249B24905618280A685014515
:10D10000EF109F9E2A84FD550145EF103FA0A28796
:10D1100005BF411126C2B724002006C622C44AC05A
:10D12000938704C303C7E70383C7F703636AF70062
:10D1300001442285B2402244924402494101828046
:10D140002A8993051020130580079730FE1FE7807A
:10D1500060EF2A8471DD130680078145938404C340
:10D160009730FE1FE780E01263150900C1572302C4
:10D17000F400BC48A1EFE0C4A0C8E0C8232004002C
:10D180008547238FF4028547A302F400930700F933
:10D19000A303F400B72700209387C7D69853DC5326
:10D1A00038C47CC4FD572309F400B727002003C509
:10D1B000C7A82302A406EF70004583472406A308EE
:10D1C000A40093E737002301F406A5B7FC4880C309
:10D1D000E0C82320040083C7E40385075DB78347C5
:10D1E000A501411122C406C69907A306F5003C45D6
:10D1F00011472306E5002380E7003C450347D5009F
:10D200002A84A380E70083471503858B91E70347B2
:10D21000050389476319F70038448347070093E7FC
:10D2200007042300F7002844930524031946090541
:10D230009730FE1FE780C0FE28440356A4010C541B
:10D2400021059730FE1FE780A0FD930730F9A30367
:10D25000F400B24022444101828041114AC0372982
:10D260000020930709C383A7C70A06C622C426C2A3
:10D2700099E3054515AAAA84130909C3EF70C05D97
:10D280008327C90A8297EF30C0572A847DD19C50EA
:10D29000EC442324F50803C774009307A009631B1B
:10D2A000F71085472300F51483C7F4052303F5140D
:10D2B000A303F51483C7F50003C705010148A207BE
:10D2C0004207BA9703C7E5001546F905BA9703C7A1
:10D2D00035FF130584136207BA97232CF40883C71C
:10D2E00055FF03C765FFA2074207BA9703C745FF6B
:10D2F000BA97232EF40883C775FFA30BF40283C7E4
:10D3000095FF03C785FFA207D98F231CF40283C7AB
:10D31000B5FF03C7A5FFA207D98F231DF40283C75A
:10D32000D5FF03C7C5FFA207D98F231EF40283C709
:10D33000F5FF03C7E5FF232E0413A207D98F231F90
:10D34000F4028147232CF4129730FE1FE78040ED52
:10D35000F84483473702FD8BA30AF40203473702E0
:10D36000ED1793F7F70F15832308E4022D47636841
:10D37000F7028357A40305679306A7C7E917C207F7
:10D38000C18363EEF6008356C4039307301F63E83E
:10D39000D7008357E403130707C8637EF7020355DA
:10D3A0008400EF3080620145B24022449244024939
:10D3B000410182808327090D13971701E35C07EE73
:10D3C000BC4403C7070083C70500F98F9583858B8D
:10D3D0002300F514C5B58327090B2285829783277F
:10D3E000890D03558400294693F7072091E30546EC
:10D3F00093050008EF50005F8327090D139717016D
:10D400006359070003558400514693050008EF5007
:10D41000605D8327C904BC4B13974700E35B07E4B7
:10D4200003C54400A3890400494693050008EF5052
:10D43000605B81B5B727002083C717C3411122C4A1
:10D4400006C626C24AC02A848DEB0347C40085471E
:10D450006316F70E8347940303471404858B631DFB
:10D46000F70C1946930524041305A4039730FE1FF7
:10D47000E78040E8B334A00091A883471504CDC7E6
:10D48000834775041307000493F7070C639EE708AE
:10D49000485521C513092404CA851305A502EF5078
:10D4A00080668547AA84631AF50248548947230099
:10D4B000F404834735001946CA8593E72700A30083
:10D4C000F40451059730FE1FE78080D5B240224416
:10D4D000268502499244410182800347C400854762
:10D4E0006304F7048347C405918B9DEF834784034E
:10D4F00085EF130504049740FE1FE78000B648D46B
:10D5000005C589472300F404834735001946930570
:10D51000240493E72700A300F40451059730FE1F6D
:10D52000E78000D085445DB783478403898B91DF12
:10D530005C5483C7170091FB814449BF8347C405EE
:10D54000918B89FB8347940013F717000DC3834623
:10D55000F4000D47639DE60028406C402244B24031
:10D560009244024941011743FE1F6700C3B6898BED
:10D57000D5DB0347F4009547E316F7FAF1BF4111F5
:10D58000B727002022C406C6938707C3238807064F
:10D59000930710F9A303F500B727002003A407D5CC
:10D5A0000DC0B727002003C537A28545EF00FFFF58
:10D5B000930710273305F50222832244B24041012C
:10D5C0000283B2402244410182808347650199C7AA
:10D5D000034765006314F7006FF07FFA03475501B6
:10D5E00011CF834665006382E6022303E500B72777
:10D5F000002003C537A289456F00BFA4F1DF0347B0
:10D60000650079FB2303F500DDB7F9D7E5BF6C456D
:10D61000314783C7150093F7F7032307F5006386A7
:10D62000E700930700083E85828083C705000D4709
:10D63000BD8BA307F500E396E7FE41114AC013092D
:10D64000250322C419462A84A1054A8506C626C296
:10D650009730FE1FE78000CA91470DC56C44130543
:10D660002404194683C7050089059987858BA30083
:10D67000F4049730FE1FE780A0BA2285EFF09FDB0D
:10D6800009E9A147B2402244924402493E85410142
:10D6900082801305000483040401EF30CFF062059B
:10D6A0006185E3C0A4FE24449D472306F400238043
:10D6B000F40085472381F400A381F4001946CA854C
:10D6C000138544009730FE1FE78080B583C7240090
:10D6D00003C73400990793F7F70F13678700238177
:10D6E000F400A381E4003844BA9703578406A38169
:10D6F000E70083C7240038448346D4053E97835708
:10D7000084069206A183BD8BD58F2302F70003C741
:10D710002400814709071377F70F2381E40003569C
:10D72000A4018346C40501CA93F70604DDEFF95747
:10D73000998F93F7F70F93F6060495C203C634004A
:10D74000344413660604A381C4003697834614014B
:10D75000A301D70003C7240005072381E400035673
:10D76000A401014719CE63EEC70083C724002844F3
:10D770000C548D073E959730FE1FE78060AA034743
:10D78000A40183C6240093F7F60385073E97A306FA
:10D79000E4002381D40083471403858B91E703477A
:10D7A000040389476319F70038448347070093E768
:10D7B00007042300F7003C448345D400A380B7004E
:10D7C0000345F405930790F9A303F400EF6010708C
:10D7D0000346D4008345F4050D459740FE1FE780BE
:10D7E000E0C4EF706007814771BDF55791B76C4594
:10D7F0001307200283C7150093F7F7032307F500EB
:10D800006399E716411122C406C626C24AC083C7DF
:10D81000050015472A84BD8BA307F500639CE7022A
:10D820001946A105130525039730FE1FE78080AC3C
:10D830009147630905126C4419461305240483C7F4
:10D84000050089059987858BA300F4049730FE1F96
:10D85000E780009D2285EFF0FFBDA147630405101E
:10D8600037270020130947AC8357890093040032FF
:10D8700093870719B3D49702832747AC82978326EF
:10D880004900B30795003E8763E4A70063E4D7002F
:10D890003387D7402444A1472306F40018D02380BF
:10D8A000F40085472381F400A381F4001946930511
:10D8B0002403138544009730FE1FE780609683C7DA
:10D8C000240099072381F40083C7340093E72700DD
:10D8D000A381F4008347140481CB384483470700B5
:10D8E00093E707F82300F7001946930524041385EE
:10D8F000A4009730FE1FE780A09283C724009907F9
:10D9000093F7F70F13F7F7030507A306E400238146
:10D91000F40083471403858B91E703470403894789
:10D920006319F70038448347070093E7070423008F
:10D93000F7003C448345D400A380B7000345F405B9
:10D940009307A0F9A303F400EF6050580346D400F6
:10D950008345F4050D459740FE1FE78020ADEF603D
:10D96000B06F8147B2402244924402493E85410152
:10D970008280930700083E85828041114AC0372982
:10D980000020032649D922C426C206C69307800771
:10D990007CD2B727002083A787D6B70533002A8417
:10D9A000D857719B13671700D8D798431377F7CFD1
:10D9B00098C398431377F7CF1367072098C3372787
:10D9C0000020032787DE1447CD8E14C7B706030057
:10D9D0009386862534CA5457F59A54D70347E505EC
:10D9E0009376F7079843137707F8558F98C3244524
:10D9F0009D472306F50085462380F400A38104009B
:10DA00002381D4008347B5050D476385E700194797
:10DA1000639BE71E8547A381F40019469305240301
:10DA2000138544009720FE1FE780807F83C7240072
:10DA300099072381F4000347B40599476316F70457
:10DA400083C734001385A40093E72700A381F40063
:10DA500083471403898B638507164C5483C72501BC
:10DA6000638007161946D1059720FE1FE780407B8B
:10DA700038448347070093E707F82300F70083C77C
:10DA8000240099072381F40083C7340003C72400CE
:10DA900093E78700A381F4003C44BA9703578406B8
:10DAA000A381E70083C7240038448346D4053E970A
:10DAB000835784069206A183BD8BD58F2302F7007E
:10DAC00003C72400814709071377F70F2381E40078
:10DAD000035684018346C40509CA93F70604639379
:10DAE0000710F957998F93F7F70F93F6060495C22D
:10DAF00003C63400344413660604A381C400369779
:10DB000083461401A301D70003C72400050723811E
:10DB1000E4000356840169EA014703C624008347F1
:10DB2000A4059376F603850636979A07D18FA30648
:10DB3000E4002381F40083471403858B91E70347B6
:10DB4000040389476319F70038448347070093E7C4
:10DB500007042300F7003C440347D400A380E700F8
:10DB6000930760F9A303F4003844832749D9B8DF49
:10DB7000B727002083C707AD81EB37E5010081455A
:10DB80001305A57AEF00BFB8B7270020032749D9AE
:10DB90009387C7D6A3810700238207005C43014512
:10DBA00093E717005CC30346D4008345F405224481
:10DBB000B2409244024941011743FE1F67000387A8
:10DBC0008347940381CB38448347070093E707F8E2
:10DBD0002300F70019469305A4039720FE1FE78052
:10DBE000206471BDF557FDBDE3E8C7F283C724008B
:10DBF00028444C508D073E959720FE1FE7804062D9
